:10D74C002020434153202000204259452E2E2E00EC
:10D75C00204D4F44454C20002020454E44202000B5
:10D76C002530376C6400204320412053200043496E
:10D77C002D353031300043492D35303030005531A6
:10D78C002E30303130004349353030300053455263
:10D79C0049455300202020202020002043482030E1
:10D7AC00322000204348203033200066006500649E
:10D7BC000063006200610060007200710070006F15
:10D7CC00006E006D006C006B006A006900680067F9
:10D7DC0000FF40FF792464656667FFFFFFDFBF7FB2
:10D7EC00FFC0F9A4B0999282D88090B88FD4B74872
:10D7FC0000888883C6A1868E4789F9F2F3C7AAAB45
:10D80C00A38C98AF9287C1FCFDFE91A40000000090
:10D81C000805020000000B07040100000046090681
:01D82C0003F8
:10E39000014F001350FFFFFFFFFFFFFFFFFFFFFFD5
:10E3A000FFFFFFFFFFFFFFFF024D000004223F8041
:10E3B0000000C10BC10CC10AC10D4107220020267B
:10E3C0002600000000000000000000000000000027
:10E3D000000000000000000000000000000000003D
:07E3E0000000000000000036
:108EC900E490073AF012D4517BFF7AD7794C12E536
:108ED9006912ABAB129C7D125B218F4CE54CF4708F
:108EE90003028FA0E54C1424FD500724BE602A021A
:108EF9008F99E54CB4030512AFB28012E54CB40268
:108F090005124B918008E54CB4010312CEE47BFFB6
:108F19007AD7795412E569807790073B127DA700CB
:108F29000000007BFF7AD7795C12E56990003B74F9
:108F390013F0A37488F012DB4A125B218F4CE54CC5
:108F4900F46035E54C24FE600B04700D90071D7428
:108F590001F08005E490071DF0E490003BF0A3F0D8
:108F690090071DE0FFE4FCFDFE900842127D9B7D09
:108F79004F7C007F0112B986D390003CE0940190A8
:108F8900003BE0940050AF7BFF7AD7796412E56922
:108F99007FA07E0F12E52FE4900739F0900739E0A2
:108FA900FFC39432400302909AEF75F004A424C8D9
:108FB900FDE435F0FC7F0412BDC8900739E0FB25BC
:108FC900E025E02450F582E43406F583127D9BEB1D
:108FD90075F004A424F4FDE5F03401FC7F0412BD0E
:108FE900C8900739E0FB25E025E0244AF582E434FE
:108FF90000F583127D9BEB75F004A42420FDE5F0B8
:109009003403FC7F0412BDC8900739E0FB25E02535
:10901900E024F8F582E43401F583127D9BEB75F0C9
:1090290004A4244CFDE5F03404FC7F0412BDC8906F
:109039000739E025E025E0247AF582E43405F58353
:10904900127D9B90084274FFF0A374D7F0A3746C4F
:10905900F0900739E075F00584FFC374099FFFE4B8
:109069009400FEE4FCFD7B477AF47910F8127C2326
:10907900900845127D9B7B017A07793112A77F7B86
:10908900017A07793112E569900739E004F0028F16
:10909900A5129C7D12E6E87BFF7AD7797212E56901
:1090A9007F587E1B12E52F90071DE0600B7BFF7A2E
:1090B900D7797A12E56980097BFF7AD7798212E537
:1090C900697F587E1B12E52F7BFF7AD7798A12E5D3
:1090D900697F587E1B12E52F7BFF7AD7799212E5BB
:1090E9009F7BFF7AD7799912E5D57F107E2712E504
:1090F9002F7BFF7AD779A012E59F7BFF7AD779A0DA
:1091090012E5D57F107E2712E52FE4900739F090FC
:109119000739E0FFC39407501674502FF8E4F6EFAF
:1091290025E02426F87620087600E004F080E09017
:1091390007397407F0900739E0FFC3940D500B7499
:10914900502FF8E4F6E004F080EB900739740DF045
:10915900900739E0FFC39413500B74502FF8E4F6CD
:10916900E004F080EB7F207E4E12E52F12E70AE43F
:10917900900739F0900739E0FFC39407500FEF25A6
:10918900E02426F8E4F608F6E004F080E7E47F0A34
:10919900FEFDFC90002BE0F8A3E0F9A3E0FAA3E0C0
:1091A900FBC3127D6440197F407E427D0F7C009095
:1091B900002BE0F8A3E0A3E0A3E0D3127D64400311
:1091C90012AFB212DF117F647E0012E52F9001F217
:1091D900E0FD7C007F0A7E0012E1BE900020E0F8ED
:1091E900A3E0F9A3E0FAA3E0FB127C23C004C005C5
:1091F900C006C00790003FE0FEA3E0FFE4FCFDF8D5
:10920900F9AA06AB07D007D006D005D004127CAE68
:10921900900649127D9BE47F14FEFDFC900649E00F
:10922900F8A3E0F9A3E0FAA3E0FB127C2390071E60
:10923900127D9B12C9C7900469127D9BE47F0AFEC7
:10924900FDFC900469E0F8A3E0F9A3E0FAA3E0FBD0
:10925900C3127D6440197F407E427D0F7C009004DB
:1092690069E0F8A3E0A3E0A3E0D3127D6440577B53
:10927900FF7AD779A712E5697FC47E0912E7877F4C
:10928900A07E0F12E52F90FE437482F090FE407489
:10929900FFF090FE42E4F07F0AFE12E52F90FE03F4
:1092A9007488F090FE027402F07F327E0012E52F7E
:1092B90012DF117F647E0012E52F12C9C79004697D
:1092C900127D9B0292459001F2E0FD7C007F0A7EAF
:1092D9000012E1BE900037EEF0A3EFF09001F2E04A
:1092E900FD7C007F0A7E0012E1BE900020E0F8A319
:1092F900E0F9A3E0FAA3E0FB127C2390074B127D6F
:109309009B90003FE0FEA3E0FFE4FCFDF8F9AA060C
:10931900AB0790074BE0FCA3E0FDA3E0FEA3E0FF51
:1093290012E4A9E47B14FAF9F8127C2390074B1292
:109339007D9B90074BE0FCA3E0FDA3E0FEA3E0FFCB
:10934900E47B0AFAF9F812E4A990074B127D9BE431
:10935900900739F09001F0E02403FFE433FE900711
:1093690039E0C39FEE6480F8748098501112CB2EB7
:1093790090073F127D9B900739E004F080D6900654
:109389004EE0600302960D90073FE0FCA3E0FDA3C9
:10939900E0FEA3E0FFEC1277B1AB25AA24A923A82C
:1093A9002212759E1277EF900743127D9B90074317
:1093B900E0FCA3E0FDA3E0FEA3E0FF90073B127DE4
:1093C9009B90002BE0FCA3E0FDA3E0FEA3E0FFE4FB
:1093D9001277B1AB25AA24A923A82212759E127768
:1093E900EF900747127D9BE4900739F0900739E029
:1093F900FFC39407501B74502FF8769C7FD07E07CB
:1094090012E52F900739E02450F876FFE004F08048
:10941900DBE4900739F0900739E0FFC39407502344
:10942900C374069F2450F876A37FD07E0712E52FD8
:10943900900739E0FFC374069F2450F876FFE004D3
:10944900F080D3900747E0FCA3E0FDA3E0FEA3E092
:10945900FF900743E0F8A3E0F9A3E0FAA3E0FBD308
:10946900127D4E402E900747E0F8A3E0F9A3E0FAF9
:10947900A3E0FB900743E0FCA3E0FDA3E0FEA3E02B
:109489009BFFEE9AFEED99FDEC98FC90074F127D3B
:109499009B802B900743E0F8A3E0F9A3E0FAA3E04F
:1094A900FBA3E0FCA3E0FDA3E0FEA3E0C39BFFEE6A
:1094B9009AFEED99FDEC98FC90074F127D9B900761
:1094C9004BE0FCA3E0FDA3E0FEA3E0FFA3E0F8A3CB
:1094D900E0F9A3E0FAA3E0FBD3127D4E5003029515
:1094E900937BFF7AD779AF12E5697FC47E0912E7CA
:1094F9008790FE437482F090FE4074FFF090FE4224
:10950900E4F07F0AFE12E52F90FE037488F090FEC6
:10951900027402F07F327E0012E52F12DF117F64A0
:109529007E0012E52F12C9C790073F127D9B900755
:109539003FE0FCA3E0FDA3E0FEA3E0FFEC1277B15E
:10954900AB25AA24A923A82212759E1277EF9007AA
:1095590043127D9B7FA07E0F12E52FE4900739F01F
:109569009001F0E02402FFE433FE900739E0C39F45
:10957900EE6480F8748098501112CB2E90073F1238
:109589007D9B900739E004F080D612CB2E90073FDF
:10959900127D9B90073FE0FCA3E0FDA3E0FEA3E062
:1095A900FFEC1277B1AB25AA24A923A82212759E34
:1095B9001277EF900743127D9BE4900024F090000E
:1095C90010127DA70000000090073FE0FCA3E0FD1A
:1095D900A3E0FEA3E0FF900460127D9B900743E0A7
:1095E900FCA3E0FDA3E0FEA3E0FF900046127D9BF3
:1095F900900046E0FCA3E0FDA3E0FEA3E0FF90039A
:109609007C127D9B90064EE06073E4FDFC7F0412A2
:10961900BDC890002B127D9B90002BE0FCA3E0FDC0
:10962900A3E0FEA3E0FFE41277B1AB25AA24A923A6
:10963900A82212759E1277EF90037C127D9B9003EE
:109649007CE0FCA3E0FDA3E0FEA3E0FF900046124E
:109659007D9B7D147C007F0412BDC8900010127D93
:109669009B7D5E7C007F0112BDC8900024EFF07DD8
:10967900717C007F0112BDC8900183EFF090017BDE
:10968900E06017C2AC124B917BFF7AD7795412E58F
:0F969900697FA07E0F12E52F80E312002680DE8E
:0196A800229F
:10D45100E4F54DF54E758CFD758A6575A8027589E3
:10D461000175881175B80275CBFF75CACC75CDFFF2
:10D4710075CCCC75C834759850758780D2AFC2B35E
:10D4810090FE437482F090FE4074FFF090FE42E4FF
:10D49100F0FFFE12E52F90FE037488F090FE0274F7
:10D4A10002F0E490017BF090018304F0E49001F23A
:10D4B100F0900116F090064F04F0E4900181F0A382
:10D4C100F09002D7F090003EF0900014F090002A06
:10D4D100F090038E743BF09001F174FFF090000F17
:10D4E1007401F0E490017BF090037BF090071CF055
:10D4F1009001F7F0900376F0900037F0A3F09000E0
:10D501000CF0A3F090003BF0A3F090001EF0A3F00C
:10D5110090003FF0A304F0E4900042F0A3F09000EB
:10D5210020127DA7000013889002D3127DA700006E
:10D531001388E4FF7F50900469E4F0A3DFFC9002BC
:10D54100C4127DA7000000009001F3127DA7000026
:07D551000000E4F54DF54E6A
:01D5580022B0
:03000B0002D82DEB
:0BD82D00C0E0C083C082C0D075D018DE
:10D83800758CFD758A65A292B3929290001FE004E0
:10D84800F0700690001EE004F0D390001FE09420D2
:10D8580090001EE0944E4004E4F0A3F090003BE0FA
:10D868007002A3E0600E90003CE024FFF090003BC3
:10D87800E034FFF090000DE004F0700690000CE03A
:10D8880004F0D390000DE0942090000CE0944E40FA
:10D8980004E4F0A3F0054FE54FD394124003754F0D
:10D8A80000E54F25E024B7F582E434D7F583E49307
:10D8B800654DFE740193654EFFE54F25E02426F87B
:10D8C800E6FC08E6FDEE6CF563EF6DF564E54D6486
:10D8D800796CF565E54E6DF566D2B3F5828565839D
:10D8E80074FFF07450254FF8E6856482856383F0F1
:02D8F800C2B3B9
:09D8FA00D0D0D082D083D0E032FE
:0300230002CDC744
:0BCDC700C0E0C083C082C0D075D0085F
:10CDD20020980302CEDBC298900390E0FEC36480E9
:10CDE200948B5003EE7010900390E4F0FF7F0B9051
:10CDF2000117E4F0A3DFFCAF99900648E06004EF6E
:10CE0200547FFF900390E0FE7005900117EFF090C1
:10CE1200000EE0B4051CD20DEEFD3395E0FC741754
:10CE22002DF58274013CF583EFF0900390E4F0025B
:10CE3200CEC2900117E0FDC394304072EDD3943915
:10CE4200506CEEFD3395E0FC74172DF58274013CB5
:10CE5200F583EFF0900390E004F0900119E0FE6496
:10CE62004D600EEE64526009EE644F6004EEB4450C
:10CE72001C900390E0C3648094874044E4F0FF7FF9
:10CE82000B900117E4F0A3DFFC7F0B8033EE6450BC
:10CE9200702E900390E0C3648094894023E4F0FFF5
:10CEA2007F0B900117E4F0A3DFFC7F0B801290034D
:10CEB20090E4F0FF7F0B900117E4F0A3DFFC7F0BFF
:10CEC20090011BE0640D600F90011DE0640D60078E
:09CED200900120E0B40D02D20D24
:09CEDB00D0D0D082D083D0E03227
:10E52F00C3EF943CEE940F5011E4FCFDC3ED9FEC50
:10E53F009E50260DBD00010C80F2E4FBFAE4FCFDB9
:10E54F00C3ED9FEC9E50070DBD00010C80F20BBB7D
:09E55F0000010AEB64064A70E4B5
:01E568002290
:0EE1BE00900815EEF0A3EFF0A3ECF0A3EDF047
:10E1CC0090081B127DA700000001900819E4F0A331
:10E1DC0004F0900817E0FEA3E0FFD390081AE09F2C
:10E1EC00EE6480F8900819E064809850359008151A
:10E1FC00E0FEA3E0FFEE3395E0FDFC90081BE0F899
:10E20C00A3E0F9A3E0FAA3E0FB127C2390081B1215
:10E21C007D9B90081AE004F07006900819E004F059
:10E22C0080B090081BE0FCA3E0FDA3E0FEA3E0FFA0
:01E23C0022BF
:0FE78700754D40754E0012E52FE4F54DF54E220D
:10E72600E4F97FD07E0712E7877FB87E0B12E52FCC
:05E7360009E9B407ED44
:01E73B0022BB
:080003002043482030322000A8
:10CB2E009007E5127DA7000000009001F0E024FFC1
:10CB3E00FEE434FF9007E9F0A3CEF09007E9E0FEA3
:10CB4E00A3E0FFD39400EE64809480405AEF780205
:10CB5E00C333CE33CED8F92465F58274043EF58303
:10CB6E00E0FCA3E0FDA3E0FEA3E0FFC004C005C00F
:10CB7E0006C0079007E9E0FEA3E07802C333CE3388
:10CB8E00CED8F92469F58274043EF583D007D00619
:10CB9E00D005D004127D9B9007EAE024FFF09007A9
:10CBAE00E9E034FFF0809412C9C7900469127D9BAE
:10CBBE00E49007E9F0A3F09001F0E0FFC39007EADC
:10CBCE00E09F7480F89007E9E064809850609007C9
:10CBDE00E5E0FCA3E0FDA3E0FEA3E0FFC004C0057A
:10CBEE00C006C007A3E0FEA3E07802C333CE33CE67
:10CBFE00D8F92469F58274043EF583E0F8A3E0F9D0
:10CC0E00A3E0FAA3E0D007D006D005D0042FFFEEA4
:10CC1E003AFEED39FDEC38FC9007E5127D9B90074E
:10CC2E00EAE004F070069007E9E004F080899007CE
:10CC3E00E5E0FCA3E0FDA3E0FEA3E0FFC004C00519
:10CC4E00C006C0079001F0E0FFE4FCFDFEF8F9FA23
:10CC5E00AB07D007D006D005D004127CAE9007E506
:10CC6E00127D9B9007E5E0FCA3E0FDA3E0FEA3E0B0
:01CC7E00FFB6
:01CC7F002292
:0BDD46009007F4EBF0A3EAF0A3E9F073
:10DD5100C296C295D294D293C296C295C294D293DE
:10DD6100E4FFE4FEC296C295C294D2939007F4E018
:10DD7100FBA3E0FAA3E0F98F82758300127B315493
:10DD810080FD6004D2978002C2979007F4E0FBA364
:10DD9100E0FAA3E02FF9E43AFA127B18FD25E0122C
:10DDA1007B5ED296C295C294D293E4FD0DEDB40A86
:10DDB100FB0EEEB408AE0FEFB403A7C296C295C234
:10DDC10094D2937F027E0012E52FC296C295D2941F
:10DDD100D2937F027E0012E52FC296D295D294D2C1
:08DDE100937F057E0012E52F7F
:01DDE9002217
:10DF1100E49007EFF09007F3F0900025E0FD7C001E
:10DF21007E4C7F4B127BD7AB07AA0690064FE0FFD2
:10DF3100C394004006EFD39403400690064F74014A
:10DF4100F090064FE0FFD394004009EF25E025E073
:10DF51009007EFF09007EFE04420A3F07C017D00F3
:10DF6100AF03AE02127BD7EF540F4490A3F090079A
:10DF710022E060079007F1E054EFF0AE02AF037CBE
:10DF8100017D00127BD79007F2EDF07B017A0779D2
:0BDF9100F012DD467F647E0012E52FD9
:01DF9C002262
:10C9C700E4F5679007EB127DA700000000D297E41B
:10C9D700F56AF56BF56C30B2779007EBE0FCA3E0F6
:10C9E700FDA3E0FEA3E02401FFE43EFEE43DFDE4F9
:10C9F7003CFC9007EB127D9BE47F507EC3FDFC90CF
:10CA070007EBE0F8A3E0F9A3E0FAA3E0FBC3127D8C
:10CA170064700312DF117F647E0012E52F7FA07E12
:10CA2700867D017C009007EBE0F8A3E0F9A3E0FA2C
:10CA3700A3E0FBC3127D64409D7BFF7A007903125C
:10CA4700E5697FE87E0312E7877F887E1312E52F6B
:10CA5700C296D295D294C293E4F568E4F567F56976
:10CA6700D296D295D294C293E56725E0F5673097C1
:10CA770003436701C296D295D294C2930569E569CB
:10CA8700B408DD746A2568F8A6670568E568B40325
:10CA9700CAC296D295D294D293AF6AE4FCFDFE90B7
:10CAA7000031127D9B900031E0FCA3E0FDA3E0FE86
:10CAB700A3E0FF7808127D88A804A905AA06AB079A
:10CAC700E4EB456BFFEAFEE9FDE8FC900031127DDF
:10CAD7009B900031E0FCA3E0FDA3E0FEA3E0FF781C
:10CAE70008127D88A804A905AA06AB07E4EB456CE4
:10CAF700FFEAFEE9FDE8FC900031127D9B900031D2
:10CB0700E0FCA3E0FDA3E0FEA3E0FF7804127D753F
:10CB1700900031127D9BD297900031E0FCA3E0FD9D
:06CB2700A3E0FEA3E0FF05
:01CB2D0022E5
:10CFFE0020205345414C2000204348203131200051
:10D00E0020434820313220002031202D20372000AF
:10D01E00202043414C20004D4F44452020004341E9
:10D02E004C20454E4400202020202020200020208F
:10D03E0020202020002020202025336C6400203D5D
:10D04E0025356C64002043414C3120004341504152
:10D05E002020002043414C322000444955492020D5
:10D06E00002043414C3320005350414E20200054A9
:10D07E003D2530356C640049443D202025326C64DA
:10D08E000020202530356C64002043414C372000B1
:10D09E00464143544F52002D202D202D202D00208F
:10D0AE002D202D202D2000204348203133200053E9
:10D0BE00554343455353002043482031342000202C
:10D0CE00203245524F2000324552302053004554F5
:10D0DE0054494E3600202020555020200020434138
:10D0EE004C3520004C4F414420200020554E4C4FD3
:10D0FE004144002043414C3420005A45524F2020D9
:09D10E0000FFFFFFFFFFFFFFFF20
:10AFB200E4900753F0A3F0A3F012DB4A12DF117FF3
:10AFC200647E0012E52F90FE02E030E7147BFF7AE8
:10AFD200CF79FE12E56912E7267F707E1712E52F00
:10AFE20022125B218F4CE54CF4700302B30D9001E9
:10AFF2007CE54CF0E490003EF0900020E0FCA3E001
:10B00200FDA3E0FEA3E0FF9002D3127D9B90003EE1
:10B01200E0600302B328900376F09001F2E0FD7C39
:10B02200007F0A7E0012E1BE900020E0F8A3E0F962
:10B03200A3E0FAA3E0FB127C23C004C005C006C053
:10B042000790003FE0FEA3E0FFE4FCFDF8F9AA064A
:10B05200AB07D007D006D005D004127CAE900649CB
:10B06200127D9BE47F14FEFDFC900649E0F8A3E00C
:10B07200F9A3E0FAA3E0FB127C2390071E127D9B4A
:10B0820090017CE024FE606E14700302B18914709A
:10B092000302B2A424FE700302B2CA14700302B205
:10B0A200DB24FC700302B2F224C5700302B2EA246C
:10B0B20045600302B2FE900020E0FCA3E0FDA3E0A5
:10B0C200FEA3E0FF9007E97401F0127E1E900020BB
:10B0D200127D9B900020E0FCA3E0FDA3E0FEA3E034
:10B0E200FF9002D3127D9B900376E0600990003EB0
:10B0F2007401F002B30790003FE0FEA3E0FFE4FC1E
:10B10200FD9007E97402F0127E1E90003FEEF0A35C
:10B11200EFF09001F2E0FD7C007F0A7E0012E1BEBA
:10B12200900020E0F8A3E0F9A3E0FAA3E0FB127C90
:10B1320023C004C005C006C00790003FE0FEA3E0A4
:10B14200FFE4FCFDF8F9AA06AB07D007D006D0054C
:10B15200D004127CAE900649127D9BE47F14FEFD62
:10B16200FC900649E0F8A3E0F9A3E0FAA3E0FB12A1
:10B172007C2390071E127D9B900376E0600990016C
:10B182007C7402F002B307E47F107E27FDFC900678
:10B1920049E0F8A3E0F9A3E0FAA3E0FBD3127D644F
:10B1A20040107BFF7AD0790612E5697F707E171214
:10B1B200E52F9002D3E0FCA3E0FDA3E0FEA3E0FFB5
:10B1C2009007E97403F0127E1E9002D3127D9BE475
:10B1D2007F64FEFDFC9002D3E0F8A3E0F9A3E0FA5D
:10B1E200A3E0FB127C23E41277B1C004C005C006C1
:10B1F200C007900020E0FCA3E0FDA3E0FEA3E0FF77
:10B20200E41277B1A804A905AA06AB07D007D006B5
:10B21200D005D0041276A7900756127D9BE4FFFE5C
:10B222007D207C41900756E0F8A3E0F9A3E0FAA361
:10B23200E0FB12774450127BFF7AD0790E12E56957
:10B242007F707E1712E52F802CE4FFFE7DC87C42C2
:10B25200900756E0F8A3E0F9A3E0FAA3E0FB127727
:10B2620044601240107BFF7AD0790E12E5697F703C
:10B272007E1712E52FE4FFFE7DC87C42900756E060
:10B28200F8A3E0F9A3E0FAA3E0FB127744600540DB
:10B292000302B1B4900376E0600890003E7401F0BE
:10B2A2008063E4FF1286B8900376E0600890003E67
:10B2B2007401F080507F011286B8900376E0600836
:10B2C20090003E7401F0803D1296A9900376E060F2
:10B2D2000890003E7401F0802C12D55990003E7403
:10B2E20001F0900753F0801D90017C7401F08015ED
:10B2F20090003E7401F0900753F0800912E7269007
:10B30200003E7401F012DB4A02B00F7BFF7AD07963
:10B312001612E5697BFF7AD0791E12E59F7BFF7AD0
:10B32200D0792512E5D5900753E0700302AFC87BB0
:10B33200FF7AD0792C12E5697BFF7AD0791E12E56B
:10B342009F7BFF7AD0792512E5D57FA07E0F12E58B
:10B352002F7BFF7AD0793412E5697BFF7AD0793C72
:0FB3620012E59F7BFF7AD0793C12E5D512D11707
:01B3710022B9
:10000E00E54CB4460790003E7401F02290017CE06E
:05001E007002EFF0226A
:067E1E009007E5127D9BB8
:107E2400E49007EAF0A37404F0A37409F0A37401C6
:107E3400F078FD7C07FD7BFF7AD1790F7E007F0807
:107E4400127AF2E4900807F0A3F0A3F0A3F012DB97
:107E54004A9007E5E0FCA3E0FDA3E0FEA3E0FF9069
:107E6400080D127D9B9007E9E0D3940A402D9008F9
:107E74004274FFF0A374D0F0A37443F090080DE0B3
:107E8400FCA3E0FDA3E0FEA3E0FF900845127D9B68
:107E94007B017A0779EE12A77F802B90084274FF4A
:107EA400F0A374D0F0A3744CF090080DE0FCA3E0B0
:107EB400FDA3E0FEA3E0FF900845127D9B7B017AC1
:107EC4000779EE12A77F9007E9E0127DF87F2F0172
:107ED4007F56027FAD037FD4047FDD057FE60780F4
:107EE4001A08804E0980BA0B80B00D80810E808103
:107EF4000F80D01080B011808F12808F1380B01447
:107F040080B01580A51680B017809A1880B01980AB
:107F1400B01A80C51E80D01F80D02280BA2380B0C2
:107F24002480E23580ED36000080F69007EE74433D
:107F3400F07BFF7AD0795312E59F7BFF7AD0795A90
:107F440012E5D590080374C6F090080274B7F002E5
:107F540080F69007EE7444F07BFF7AD0796112E5E5
:107F64009F7BFF7AD0796812E5D590080274B7F048
:107F74009001F2E0FFB401089007F37421F080202F
:107F8400EFB4020C9007F27421F0A37430F0801067
:107F9400EFB4030C9007F17421F0A37430F0A3F054
:107FA40090080374A1F00280F69007EE744CF07B05
:107FB400FF7AD0796F12E59F7BFF7AD0797612E54C
:107FC400D590080374C7F090080274B7F00280F6E5
:107FD4009007EB7406F00280F69007EB7403F0024E
:107FE40080F690084274FFF0A374D0F0A3747DF07F
:107FF40090080DE0FCA3E0FDA3E0FEA3E0FF9008E1
:1080040045127D9B7B017A0779EE12A77F9007EBDF
:108014007404F00280F690084274FFF0A374D0F068
:10802400A37485F090080DE0FCA3E0FDA3E0FEA39B
:10803400E0FF900845127D9B7B017A0779EE12A739
:108044007F9007EB7401F00280F690084274FFF011
:10805400A374D0F0A3748FF090080DE0FCA3E0FDAE
:10806400A3E0FEA3E0FF900845127D9B7B017A0705
:1080740079EE12A77F9007EB7404F08075E4900703
:10808400EBF0A37409F0E4A3F08067E49007EBF04D
:10809400A37404F0805CE49007EBF0A37405F08013
:1080A40051E49007EBF0A37406F08046E49007EBEC
:1080B400F0A304F0803CE49007EBF0A37402F0809A
:1080C40031E49007EBF0A37404F080269007F3E00A
:1080D400B420037430F09007EB7401F08014E49042
:1080E40007EBF0A37409F08009E49007EBF0A374A4
:1080F40006F09007E9E0B4051B7BFF7AD0793412CF
:10810400E5697BFF7AD0799712E59F7BFF7AD07976
:108114009E12E5D5E4900805F0A3F0900805E0FE72
:10812400A3E0FFC39407EE64809480502F74EE2F75
:10813400F58274073EF583E090D7BD93FF9008065F
:10814400E024EEF582E43407F583EFF0900806E0CE
:1081540004F07006900805E004F080BF9001F2E09E
:10816400FF60249007E9E0FE64076004EEB4091799
:10817400C374069FFFE49400FE74EE2FF582740727
:108184003EF583E0547FF09007E9E0FDB41F0790CB
:1081940007F3E0547FF0ED6404603CED6405603760
:1081A400E4900805F0A3F0900806E0FF24EEF582C1
:1081B400E43407F583E0FE74502FF8A60690080611
:1081C400E004F07006900805E004F0900805E07003
:1081D40004A3E0640770D0125B218F4CE54CF4706B
:1081E400030286A0E54C24BA70030284F62446B444
:1081F4000C00400302869A908202F82828730282B7
:108204003302825502825502822602822602825558
:1082140002822602822602822602822602869A028E
:1082240083169007E9E0B4020612E72602869D90C1
:1082340007E9E0C39404500E9007FDE0B4C007E4DE
:10824400900807F0A3F09007EDE0254C7003754CFF
:10825400019007EBE07006900807F0A3F09007E99F
:10826400E0B40221D3900808E09403900807E06486
:10827400809480401012E7269003767401F09007F2
:10828400EAF002869D9007EBE0FFD3900808E09F98
:108294007480F8900807E0648098400612E726028C
:1082A400869D9007ECE0FFE54CD39F40028F4C90F5
:1082B4000808E0FF24F5F582E43407F583E54CF083
:1082C40090D7ED93FE74FD2FF582E43407F583EE29
:1082D400F09007E9E0B41F18900807E07002A3E0EB
:1082E400700E74FD2FF582E43407F583E0547FF0BB
:1082F4009007E9E0B4050D74FD2FF582E43407F529
:108304008374BFF0900808E004F07006900807E05A
:1083140004F0E54C640B60030284359007E9E0FF48
:108324006402600DEF64076008EF6409600302846F
:1083340029C3900808E09401900807E064809480C1
:10834400500302869D900809E07002A3E0600612C3
:10835400E72602869D900807E0FFA3E0A3CFF0A3E1
:10836400EFF0900808E024FCF582E43407F583E09C
:10837400547FF0900805E4F0A37406F0900807E039
:10838400FEA3E0FFC3900806E09FEE6480F8900827
:1083940005E06480984033A3E0FF24FDF582E434D3
:1083A40007F583E0FEC374069F2450F8A60674F50F
:1083B4002FF582E43407F583E4F0900806E024FF07
:1083C400F0900805E034FFF080B2E4900805F0A3D3
:1083D400F0900807E0FEA3E0FF24FFFDEE34FFFC6D
:1083E400900805E0FAA3E0FBD39DEC6480F8EA640E
:1083F4008098400302869DC3EF9BFFEE9AFE74FCB7
:108404002FF58274073EF583E0FF900806E0FEC373
:1084140074069E2450F8A607E004F0700690080540
:10842400E004F080AC9003767401F09007EA7401E4
:10843400F0900805E4F0A37406F0900807E0FEA3AA
:10844400E0FFC3900806E09FEE6480F8900805E022
:108454006480984033A3E0FF24FDF582E43407F5FB
:1084640083E0FEC374069F2450F8A60674F52FF526
:1084740082E43407F583E4F0900806E024FFF090EA
:108484000805E034FFF080B2E4900805F0A3F09012
:108494000807E0FEA3E0FF24FFFDEE34FFFC900894
:1084A40005E0FAA3E0FBD39DEC6480F8EA648098CD
:1084B400502EC3EF9BFFEE9AFE74FC2FF5827407D7
:1084C4003EF583E0FF900806E0FEC374069E245048
:1084D400F8A607E004F07006900805E004F080AF09
:1084E400E54C640B600302869D900807F0A3F0023C
:1084F400869D900807E0FAA3E0FBD39400EA648029
:108504009480500302869290080D127DA70000000B
:1085140000EB24FFFEEA34FF900805F0A3CEF0C37D
:10852400900805E06480948050030285B190080DA2
:10853400E0F8A3E0F9A3E0FAA3E0FBC000C001C0A7
:1085440002C003900805E0FCA3E0FD7F0A7E001250
:10855400E1BEA804A905AA06AB07900805E0FEA39E
:10856400E0FFC3900808E09FFF900807E09EFE74B8
:10857400F42FF58274073EF583E0FFE4FCFDFE1260
:108584007C23D003D002D001D000EB2FFFEA3EFEC3
:10859400E93DFDE83CFC90080D127D9B900806E047
:1085A40024FFF0900805E034FFF00285239007E9EA
:1085B400E0FCB40220900809E07002A3E06011908E
:1085C400080AE0FE900808E0C39E9001F2F08005DE
:1085D400E49001F2F0EC64076008EC6409600302C3
:1085E4008692900809E07002A3E0700D900807E0FD
:1085F400FFA3E0A3CFF0A3EFF0900809E0FEA3E00F
:10860400FFC3900808E09FFF900807E09EFE9001DA
:10861400F2E0FDC3EF9DFFEE9400FE90080BF0A383
:10862400EFF0D39400EE64809480401C12E7267F20
:10863400B87E0B12E52F90080D127DA700000000F4
:108644009007EA7401F08051900809E0FEA3E0FF6E
:10865400C3900808E09FFF900807E09EFE9001F297
:10866400E0C39FFFE49EFE90080BF0FCA3EFF0FD37
:108674007F0A7E0012E1BE90080DE0F8A3E0F9A3A2
:10868400E0FAA3E0FB127C2390080D127D9B900777
:10869400EA7401F0800312E72612DB4A9007EAE04D
:1086A40070030281DB90080DE0FCA3E0FDA3E0FE73
:0386B400A3E0FF41
:0186B70022A0
:0586B80090075AEFF0ED
:1086BD00E4900762F012DB4A125B218F4CE54CF41B
:1086CD007003028E81E54C64466003028E007BFFD1
:1086DD007AD0793412E569E490075BF090075BE09E
:1086ED00FFC364809483400302894190064FEFF0ED
:1086FD0012DF11900763127DA700000000E49007C0
:10870D005DF09001F0E075F002A4FF90075DE0FDD3
:10871D003395E0FCC3ED9FE5F06480F8EC64809840
:10872D00501112CB2E900773127D9B90075DE004C4
:10873D00F080CF90075BE070097BFF7AD079A512AE
:10874D00E56990075BE0B401097BFF7AD079AD1242
:10875D00E56990075BE0B402097BFF7AD079A51239
:10876D00E569E490075CF090075CE0C36480949445
:10877D0040030288F212CB2EC004C005C006C0070C
:10878D0090075BE0FF3395E0FEEF7802C333CE3305
:10879D00CED8F9FBAA062467F58274073AF583D083
:1087AD0007D006D005D004127D9B74672BF582741B
:1087BD00073AF583E0FCA3E0FDA3E0FEA3E0FF9004
:1087CD000773E0F8A3E0F9A3E0FAA3E0FBD3127D71
:1087DD0064404690075BE0FF3395E0FEEF7802C3FF
:1087ED0033CE33CED8F92467F58274073EF583E096
:1087FD00F8A3E0F9A3E0FAA3E0FB900773E0FCA374
:10880D00E0FDA3E0FEA3E0C39BFFEE9AFEED99FD14
:10881D00EC98FCA3127D9B804690075BE0FF33959F
:10882D00E0FEEF7802C333CE33CED8F92467F5825C
:10883D0074073EF583E0FCA3E0FDA3E0FEA3E0FF9B
:10884D00900773E0F8A3E0F9A3E0FAA3E0FBC3EF10
:10885D009BFFEE9AFEED99FDEC98FCA3127D9BE437
:10886D007FC47E09FDFC900777E0F8A3E0F9A3E053
:10887D00FAA3E0FBD3127D64400D12E7267FA07EA4
:10888D000F12E52F0286C2900763E0FCA3E0FDA363
:10889D00E0FEA3E0FFC004C005C006C00790075B63
:1088AD00E0FF3395E0FEEF7802C333CE33CED8F937
:1088BD002467F58274073EF583E0F8A3E0F9A3E0A1
:1088CD00FAA3E0D007D006D005D0042FFFEE3AFE74
:1088DD00ED39FDEC38FC900763127D9B90075CE051
:1088ED0004F0028774E47B14FAF9F8900763E0FC56
:1088FD00A3E0FDA3E0FEA3E0FF127CAEC004C00523
:10890D00C006C00790075BE0FF3395E0FEEF7802ED
:10891D00C333CE33CED8F92467F58274073EF58381
:10892D00D007D006D005D004127D9B90075BE004E4
:10893D00F00286E990075AE07003028CE19002D3B1
:10894D00E0F8A3E0F9A3E0FAA3E0FB900020E0FC3F
:10895D00A3E0FDA3E0FEA3E0FF127CAEA804A905F1
:10896D00AA06AB0790071EE0FCA3E0FDA3E0FEA363
:10897D00E0FF127CAE90077B127D9BE490075BF0CD
:10898D0090075BE0FFC3648094834003028C25EF66
:10899D003395E0FEEF7802C333CE33CED8F924679A
:1089AD00F58274073EF583E0FCA3E0FDA3E0FEA392
:1089BD00E0FFC004C005C006C00790075BE0FF33B1
:1089CD0095E0FEEF7802C333CE33CED8F9FBAA067D
:1089DD00248BF58274073AF583D007D006D005D0E5
:1089ED0004127D9B747F2BF58274073AF583E0F8B2
:1089FD00A3E0F9A3E0FAA3E0FBC000C001C002C0F0
:108A0D000390075BE0FF3395E0FEEF7802C333CEB2
:108A1D0033CED8F9248BF58274073EF583E0FCA3A1
:108A2D00E0FDA3E0FEA3E0D003D002D001D000C34F
:108A3D009BFFEE9AFEED99FDEC98FC90077BE0F81C
:108A4D00A3E0F9A3E0FAA3E0FBD3127D64402190EB
:108A5D00075BE064026003028C1C7BFF7AD079B562
:108A6D0012E56912E7267FA07E0F12E52F0286C25E
:108A7D0090075BE0FF3395E0FEEF7802C333CE3312
:108A8D00CED8F9247FF58274073EF583E0F8A3E094
:108A9D00F9A3E0FAA3E0FBC000C001C002C003903F
:108AAD00075BE0FF3395E0FEEF7802C333CE33CEA4
:108ABD00D8F9248BF58274073EF583E0FCA3E0FD25
:108ACD00A3E0FEA3E0D003D002D001D000C39BFFF2
:108ADD00EE9AFEED99FDEC98FCC004C005C006C0F1
:108AED00079002D3E0F8A3E0F9A3E0FAA3E0FB902E
:108AFD000020E0FCA3E0FDA3E0FEA3E0FF127CAEAE
:108B0D00D003D002D001D000127C23C004C005C018
:108B1D0006C00790075BE0FF3395E0FEEF7802C3D8
:108B2D0033CE33CED8F9247FF58274073EF583E03A
:108B3D00F8A3E0F9A3E0FAA3E0D007D006D005D062
:108B4D00042FFFEA3EFEE93DFDE83CFC7B407A4206
:108B5D00790F7800C3127D64501F90075BE06003AE
:108B6D00028C1C7BFF7AD079B512E56912E7267F5E
:108B7D00A07E0F12E52F0286C27BFF7AD079BD123F
:108B8D00E56990075BE0FF3395E0FEEF7802C333B4
:108B9D00CE33CED8F9FBAA06247FF58274073AF5B9
:108BAD0083E0FCA3E0FDA3E0FEA3E0FF90002B1209
:108BBD007D9B748B2BF58274073AF583E0FCA3E063
:108BCD00FDA3E0FEA3E0FF90002BE0F8A3E0F9A3E6
:108BDD00E0FAA3E0FBC3EF9BFFEE9AFEED99FDECEF
:108BED0098FC90001A127D9B90075BE090064FF069
:108BFD0012DF1190075B7403F0900010127DA70037
:108C0D00000000E4900024F07FA07E0F12E52F906D
:108C1D00075BE004F002898D9002D3E0FCA3E0FD38
:108C2D00A3E0FEA3E0FFE41277B1C004C005C006C7
:108C3D00C007900020E0FCA3E0FDA3E0FEA3E0FF51
:108C4D00E41277B1D003D002D001D0001276A790F4
:108C5D00075E127D9B90001AE0FCA3E0FDA3E0FEF1
:108C6D00A3E0FFE41277B190075EE0F8A3E0F9A36B
:108C7D00E0FAA3E0FB12759EC004C005C006C00754
:108C8D0090071EE0FCA3E0FDA3E0FEA3E0FFE412CD
:108C9D0077B1D003D002D001D0001276A78F258EE8
:108CAD00248D238C22900460E0FCA3E0FDA3E0FE64
:108CBD00A3E0FFEC1277B1AB25AA24A923A82212B9
:108CCD00759E1277EF900046127D9B90076274019E
:108CDD00F0028EBFE490075BF090075BE0FFC3648A
:108CED008094834003028DE7EF3395E0FEEF780229
:108CFD00C333CE33CED8F92467F58274073EF5839E
:108D0D00E0FCA3E0FDA3E0FEA3E0FFE47B64FAF941
:108D1D00F8D3127D6440167BFF7AD079C512E569D0
:108D2D0012E7267FA07E0F12E52F0286C290075B09
:108D3D00E0FF7047EF3395E0FEEF7802C333CE339B
:108D4D00CED8F92467F58274073EF583E0FCA3E0E5
:108D5D00FDA3E0FEA3E0FF7B607AAE790A7800C345
:108D6D00127D6450167BFF7AD079C512E56912E742
:108D7D00267FA07E0F12E52F0286C290075BE0FFD3
:108D8D003395E0FEEF7802C333CE33CED8F92467A6
:108D9D00F58274073EF583E0FCA3E0FDA3E0FEA39E
:108DAD00E0FFC004C005C006C00790075BE0FF33BD
:108DBD0095E0FEEF7802C333CE33CED8F9247FF59C
:108DCD008274073EF583D007D006D005D004127DFE
:108DDD009B90075BE004F0028CE67BFF7AD079BDB7
:108DED0012E5697FA07E0F12E52F9007627401F0E6
:108DFD00028EBFE54CB40B0D9003767401F0900715
:108E0D0062F0028EBFE54C640170647BFF7AD0790D
:108E1D00CD12E5697BFF7AD079D512E59F7BFF7A7C
:108E2D00D079DC12E5D57FA07E0F12E52FE49007F7
:108E3D005DF09001F0E0240AFFE433FE90075DE061
:108E4D00FD3395E0FCC3ED9FEE6480F8EC648098F3
:108E5D00501112CB2E90002B127D9B90075DE004DC
:108E6D00F080CF9003767401F0900762F08043128A
:108E7D00E726803E90075AE0601D7BFF7AD079E3AC
:108E8D0012E5697BFF7AD079EB12E59F7BFF7AD0F3
:108E9D0079F212E5D5801B7BFF7AD079F912E5695D
:108EAD007BFF7AD1790112E59F7BFF7AD179081288
:0B8EBD00E5D5900762E070030286C557
:018EC8002287
:0EE7A5002043414C362000554552494659004C
:1096A900E490075AF0A3F090075EF0A37402F090DB
:1096B900002BE0FCA3E0FDA3E0FEA3E0FF90046023
:1096C900127D9B900460E0FCA3E0FDA3E0FEA3E013
:1096D900FFEC1277B1AB25AA24A923A82212759E03
:1096E9001277EF900046127D9B7BFF7AE779A512EE
:1096F900E59F7BFF7AE779AC12E5D59001F2E0FFAF
:1097090070089001167405F08022EFB401089001E9
:10971900167404F08016EFB402089001167403F071
:10972900800AEFB403069001167402F07F2C7E01C3
:1097390012E52F125B218F4CE54CF4700302993C22
:10974900E54C700302985B24F8604724FD7003021E
:10975900992A24C570030299222445600302993687
:1097690012CB2E900460127D9B900460E0FCA3E074
:10977900FDA3E0FEA3E0FFEC1277B1AB25AA24A973
:1097890023A82212759E1277EF900046127D9B0244
:10979900993912CB2E900768127D9B900768E0FCDF
:1097A900A3E0FDA3E0FEA3E0FFEC1277B1AB25AA8D
:1097B90024A923A82212759E1277EF900764127DBF
:1097C9009BAB25AA24A923A822C000C001C002C0BE
:1097D90003900460E0F8A3E0F9A3E0FAA3E0FB90AA
:1097E9000768E0FCA3E0FDA3E0FEA3E0C39BFFEE56
:1097F9009AFEED99FDEC98FC1277B1A804A905AA87
:1098090006AB07E4FFFE7D807C401276A7D003D02B
:1098190002D001D0001274AD8F258E248D238C22A5
:1098290012CB2E900768127D9B900768E0FCA3E09D
:10983900FDA3E0FEA3E0FFEC1277B1AB25AA24A9B2
:1098490023A82212759E1277EF900764127D9B025E
:10985900993912CB2E900768127D9B900768E0FC1E
:10986900A3E0FDA3E0FEA3E0FFEC1277B1AB25AACC
:1098790024A923A82212759E1277EF900764127DFE
:109889009BAF25AE24AD23AC22C004C005C006C0E1
:1098990007900460E0F8A3E0F9A3E0FAA3E0FB90E5
:1098A9000768E0FCA3E0FDA3E0FEA3E0C39BFFEE95
:1098B9009AFEED99FDEC98FC1277B1A804A905AAC6
:1098C90006AB07E4FFFE7D807C401276A7A804A9B9
:1098D90005AA06AB07D007D006D005D0041274A993
:1098E9008F258E248D238C2212CB2E900768127D12
:1098F9009B900768E0FCA3E0FDA3E0FEA3E0FFEC7A
:109909001277B1AB25AA24A923A82212759E127732
:10991900EF900764127D9B801790075A7401F080BD
:109929000F9003767401F090075AF0800312E7262E
:1099390012E45312CB2EE41277B1AB25AA24A92342
:10994900A82212759E1277EF900380127D9B9000DA
:1099590046E0F8A3E0F9A3E0FAA3E0FB900380E076
:10996900FCA3E0FDA3E0FEA3E0C39BFFEE9AFEED9E
:1099790099FDEC98FC9002C4127D9BE4FFFEFDFC6E
:109989009002C4E0F8A3E0F9A3E0FAA3E0FBC31254
:109999007D4E402F9002C4E0FCA3E0FDA3E0FEA3AE
:1099A900E0240AFFE43EFEE43DFDE43CFCE47B14D4
:1099B900FAF9F812E4A9900385127D9BE49000144A
:1099C900F080319002C4E0FCA3E0FDA3E0FEA3E037
:1099D90024F6FFEE34FFFEED34FFFDEC34FFFCE42A
:1099E9007B14FAF9F812E4A9900385127D9B900083
:1099F900147401F0900385E0FCA3E0FDA3E0FEA34D
:109A0900E0FF900389127D9B90075CE4F0A304F0CA
:109A190090003FE0FEA3E0FFC390075DE09F900741
:109A29005CE09E503E900389E0FCA3E0FDA3E0FECC
:109A3900A3E0FF900385E0F8A3E0F9A3E0FAA3E02F
:109A4900FBEF2BFFEE3AFEED39FDEC38FC90038974
:109A5900127D9B90075DE004F0700690075CE004BE
:109A6900F080AD900389E0FCA3E0FDA3E0FEA3E054
:109A7900FF9001F3127D9B9002C4E0FCA3E0FDA3DB
:109A8900E0FEA3E0FF900760127D9BE4FFFEFDFC72
:109A9900900760E0F8A3E0F9A3E0FAA3E0FBC312A2
:109AA9007D4E501D900760E0FCA3E0FDA3E0FEA3FE
:109AB900E0FF74FFFBFAF9F8127C23900760127D2E
:109AC9009B900760E0FCA3E0FDA3E0FEA3E0240A6D
:109AD900FFE43EFEE43DFDE43CFCE47B14FAF9F8C6
:109AE90012E4A9AC00AD01AE02AF03E47B02FAF9BE
:109AF900F812E4A990075EEEF0A3EFF0E4F526F57D
:109B090027F528F529F52AF52BF52CF52DF52EF550
:109B19002FF530F531F532F533EE7061EFB40A0007
:109B2900505B909B32F8282873029B50029B580285
:109B39009B60029B60029B68029B68029B70029B70
:109B490070029B78029B80752620752700802E75F0
:109B590028207529008026752A20752B00801E75FE
:109B69002C20752D008016752E20752F00800E75FE
:109B7900302075310080067532207533009001F36D
:109B8900E0FCA3E0FDA3E0FEA3E0FF12D9039007E8
:109B99005BE07003029C56C390075FE09404900752
:109BA9005EE0648094805043AF25AE24AD23AC229F
:109BB9007BBD7A37790678361274AD8F258E248D60
:109BC900238C22900460E0FCA3E0FDA3E0FEA3E067
:109BD900FFEC1277B1AB25AA24A923A82212759EFE
:109BE9001277EF900046127D9B806290075EE0FE3F
:109BF900A3E0FF64044E6006EF64054E700E7F2CEF
:109C09007E0112E787E490075BF08041AF25AE241F
:109C1900AD23AC227BBD7A37790678B61274AD8F45
:109C2900258E248D238C22900460E0FCA3E0FDA303
:109C3900E0FEA3E0FFEC1277B1AB25AA24A923A883
:109C49002212759E1277EF900046127D9B90075A5B
:109C5900E0700302973CE4F526F527F528F529F588
:109C69002AF52BF52CF52DF52EF52FF530F531F5D7
:039C790032F5338E
:019C7C0022C5
:10E66F009007E97405F07F007E007D007C00127E2C
:10E67F001EE47BC87A07F9F8C3127D64600EE54C7F
:0FE68F00B4110612E72612E7267F00227F012230
:10E73C002025303278253032782530327800203060
:06E74C00303030303000D7
:10E6E8007F0A7E0012E52F90FF0A742FF07F647E68
:10E6F8000012E52F90FF0B7402F07F647E0012E594
:02E708002F22BE
:10E1390090FF00E090038EF0D394594002E4F07F01
:10E14900057E0012E52F90FF02E0900579F0D39447
:10E15900594002E4F07F057E0012E52F90FF04E0AC
:10E16900900029F0D394244002E4F07F057E001248
:10E17900E52F90FF07E0900028F0D394314002E4A6
:10E18900F07F057E0012E52F90FF08E0900005F072
:10E19900D394124002E4F07F057E0012E52F90FF30
:10E1A90009E0900019F0D394994002E4F07F057ECC
:05E1B9000012E52F2219
:10E02900EF14604604600302E0B2900001127B31F4
:10E03900FF127B18FEC454F02F90FF09F0900002E4
:10E04900127B31FFC454F0FF900003127B312F90F3
:10E05900FF08F0900004127B31FFC454F0FF9000D8
:10E0690005127B312F90FF07F022900001127B31BE
:10E07900FF127B18FEC454F02F90FF04F0900002A9
:10E08900127B31FFC454F0FF900003127B312F90B3
:10E09900FF02F0900004127B31FFC454F0FF90009E
:0AE0A90005127B312F90FF00F022DA
:05B69A00900789EFF0AC
:10B69F00A3E4F0A304F0E4A3F0A3F012DB4A7F0AC3
:10B6AF007E0012E52F12E1397F0A7E0012E52F90FE
:10B6BF000789E014607A04600302B7B1900019E0C3
:10B6CF00FDC4540F90078EF0ED540FA3F0900005BA
:10B6DF00E0FFC4540F900790F0EF540FA3F09000C9
:10B6EF0028E0FEC4540F900792F0EE540FA3F09091
:10B6FF00084274FFF0A374E7F0A3743CF0A3E4F0E6
:10B70F00A3EDF0A3E4F0A3EFF0900028E0FF900882
:10B71F0049E4F0A3EFF07B017A07799412A77F7BBE
:10B72F00017A07799412E56953527F53547F8072DF
:10B73F00900029E0FDC4540F90078EF0ED540FA335
:10B74F00F0900579E0FFC4540F900790F0EF540F7D
:10B75F00A3F090038EE0FEC4540F900792F0EE54C6
:10B76F000FA3F090084274FFF0A374E7F0A3743CAA
:10B77F00F0A3E4F0A3EDF0A3E4F0A3EFF090038EB9
:10B78F00E0FF900849E4F0A3EFF07B017A0779948A
:10B79F0012A77F7B017A07799412E56953527F5381
:10B7AF00547F125B218F4CE54CF4700302B928E5EE
:10B7BF004C24F6500A14604924C5606402B92290E3
:10B7CF000789E014600604600302B92590078CE036
:10B7DF00FF248EF582E43407F583E54CF090D7ED26
:10B7EF0093FE74512FF8A60653527F53547F900740
:10B7FF008CE004F0D39405500302B925E4F002B9AC
:10B80F0025E4FF7F0690078EE4F0A3DFFC7F067B25
:10B81F00FF7AE7794A12E569E490078CF002B925BF
:10B82F00900789E014607004600302B90C90078ED2
:10B83F00E075F00AA4FFA3E02FFF900019F0900726
:10B84F0090E075F00AA4FEA3E02E900005F090079B
:10B85F0092E075F00AA4FEA3E02E900028F0EFD33B
:10B86F0094635013900005E0940C500B900028E067
:10B87F00941F500302B90CE490078EF0A304F0A3B9
:10B88F00F0E4A3F0A304F0A37403F012E7267F40C3
:10B89F007E1F12E52F806690078EE075F00AA4FFD9
:10B8AF00A3E02FFF900029F0900790E075F00AA415
:10B8BF00FEA3E02E900579F0900792E075F00AA4B0
:10B8CF00FEA3E02E90038EF0EFD394175010900547
:10B8DF0079E0943B500890038EE0943B401F900713
:10B8EF008E7401F0E4A3F0A304F0A37403F0E4A3B7
:10B8FF00F0A3F012E7267F407E1F12E52F900789F5
:10B90F00E0FF7B017A07798E12E02990078D740191
:10B91F00F0800312E72612DB4A90078CE0FF248E9B
:10B92F00F582E43407F583E0FE90078AE0FCA3E09C
:10B93F00D3943CEC9400400E74512FF876FF90078F
:10B94F008AE4F0A304F090078AE475F001127C0DED
:10B95F00FCD3E5F0941EEC94004012EE90D7ED93DB
:10B96F00FE74512FF8A60653527F53547F90078DC4
:06B97F00E0700302B7B105
:01B98500229F
:0DE7B300204348203031200025376C6400E1
:10ABAB00E4FDFC7F0412BDC890002B127D9B7D043D
:10ABBB007C007F0412BDC890001A127D9B7D147C13
:10ABCB00007F0412BDC8900010127D9B7D087C0095
:10ABDB007F0412BDC8900020127D9B7D0C7C007FF2
:10ABEB000412BDC890003FEEF0A3EFF07D107C0087
:10ABFB007F0412BDC8E41277B1C004C005C006C003
:10AC0B00077D097C007F0A7E0012E1BEE41277B15A
:10AC1B00A804A905AA06AB07D007D006D005D00417
:10AC2B001276A78F258E248D238C227D1C7C007F92
:10AC3B000412BDC890017D127D9B7D207C007F049A
:10AC4B0012BDC89001EA127D9B7D667C007F0112CC
:10AC5B00BDC89001F2EFF07D657C007F0112BDC88D
:10AC6B0090064FEFF07D627C007F0112BDC8900112
:10AC7B00F0EFF07D637C007F0112BDC89002C9EF3D
:10AC8B00F07D647C007F0112BDC890038DEFF07DD9
:10AC9B00617C007F0112BDC890000AEEF0A3EFF0BB
:10ACAB007D607C007F0112BDC8900044EEF0A3EFE5
:10ACBB00F07D5F7C007F0112BDC8900026EEF0A3F3
:10ACCB00EFF07D5D7C007F0112BDC890064EEFF06A
:10ACDB007D5C7C007F0112BDC89001EEEFF07D5BC7
:10ACEB007C007F0112BDC8900041EFF07D5A7C00C3
:10ACFB007F0112BDC89002D2EFF07D597C007F011D
:10AD0B0012BDC8900384EFF07D587C007F0112BD0B
:10AD1B00C890000EEFF07D577C007F0112BDC890EC
:10AD2B000018EFF07D567C007F0112BDC89002DD4C
:10AD3B00EFF07D557C007F0112BDC8900004EFF051
:10AD4B007D537C007F0112BDC8900017EFF07D5240
:10AD5B007C007F0112BDC8900392EFF07D517C0007
:10AD6B007F0112BDC89002C8EFF07D5E7C007F01B1
:10AD7B0012BDC8900024EFF07D507C007F0112BD06
:10AD8B00C890045FEFF07D697C007F0112BDC89015
:10AD9B000464E4F0A3EFF07D677C007F0112BDC873
:10ADAB00900646E4F0A3EFF07D687C007F0112BDB6
:10ADBB00C8900466EFF07D6A7C007F0112BDC890DD
:10ADCB00064DEFF07D727C007F0112BDC8900467C9
:10ADDB00EFF07D6B7C007F0112BDC8900025EFF07A
:10ADEB007D6C7C007F0112BDC8900722EFF07D7057
:10ADFB007C007F0112BDC8900391EFF07D6D7C004C
:10AE0B007F0112BDC8900648EFF07D6E7C007F017C
:10AE1B0012BDC890002FE4F0A3EFF07D547C007FAF
:10AE2B000112BDC8900035E4F0A3EFF07D6F7C00FC
:10AE3B007F0112BDC8900723EFF07D4F7C007F018F
:10AE4B0012BDC890071DEFF0E4900753F0A3F090EC
:10AE5B000753E0FEA3E0FFC39448EE9400502BEFA2
:10AE6B002478FDE43EFC7F0112BDC8900754E0241A
:10AE7B0031F582E43405F583EFF0900754E004F0EC
:10AE8B007006900753E004F080C5900646E0FEA3E1
:10AE9B00E07802C333CE33CED8F924C8FDE43EFCB0
:10AEAB007F0412BDC8C004C005C006C0079006468B
:10AEBB00E0FAA3E0FBAE027802C333CE33CED8F96F
:10AECB002450F58274063EF583D007D006D005D00A
:10AEDB0004127D9BEBAE027802C333CE33CED8F98E
:10AEEB0024F4FDEE3401FC7F0412BDC8C004C00580
:10AEFB00C006C007900646E0FAA3E0FBAE0278025C
:10AF0B00C333CE33CED8F9244AF58274003EF58391
:10AF1B00D007D006D005D004127D9BEBAE02780291
:10AF2B00C333CE33CED8F92420FDEE3403FC7F049B
:10AF3B0012BDC8C004C005C006C007900646E0FAA3
:10AF4B00A3E0FBAE027802C333CE33CED8F924F89C
:10AF5B00F58274013EF583D007D006D005D00412DC
:10AF6B007D9BEBAE027802C333CE33CED8F9244CA3
:10AF7B00FDEE3404FC7F0412BDC8C004C005C0063E
:10AF8B00C007900646E0FEA3E07802C333CE33CE73
:10AF9B00D8F9247AF58274053EF583D007D006D014
:06AFAB0005D004127D9B9D
:01AFB100227D
:10D1170090002BE0FCA3E0FDA3E0FEA3E0FF900856
:10D1270042127D9BE4FDFC7F0412B98690001AE051
:10D13700FCA3E0FDA3E0FEA3E0FF900842127D9B65
:10D147007D047C007F0412B986900020E0FCA3E0F8
:10D15700FDA3E0FEA3E0FF900842127D9B7D087CC3
:10D16700007F0412B98690003FE0FEA3E0FFE4FCD5
:10D17700FD900842127D9B7D0C7C007F0412B986CE
:10D187007D097C007F0A7E0012E1BEE41277B1AB15
:10D1970025AA24A923A82212759E1277EF90075A71
:10D1A700127D9B90075AE0FCA3E0FDA3E0FEA3E0FD
:10D1B700FF900842127D9B7D107C007F0412B98688
:10D1C700900010E0FCA3E0FDA3E0FEA3E0FF9008C1
:10D1D70042127D9B7D147C007F0412B98690002447
:10D1E700E0FFE4FCFDFE900842127D9B7D5E7C0023
:10D1F7007F0112B9869001F2E0FFE4FCFDFE900882
:10D2070042127D9B7D667C007F0112B98690064F96
:10D21700E0FFE4FCFDFE900842127D9B7D657C00EB
:05D227007F0112B98631
:01D22C0022DF
:109C7D00E4FFFEFDFCAB25AA24A923A822127744FC
:109C8D00601B4019E4FFFE7D207C41AB25AA24A971
:109C9D0023A82212774460025003029E187BFF7A9C
:109CAD00E779B312E5697FC47E0912E787E490076F
:109CBD0053F0900753E0F9C394334003029E18E923
:109CCD0025E025E02450F582E43406F583127DA7C6
:109CDD0000000000E925E025E0244AF582E4340087
:109CED00F583127DA700000000E925E025E024F8AA
:109CFD00F582E43401F583127DA700000000E9250B
:109D0D00E025E0247AF582E43405F583127DA70081
:109D1D00000000E975F004A424C8FDE435F0FCC092
:109D2D0004C005E925E025E02450F582E43406F56C
:109D3D0083E0FCA3E0FDA3E0FEA3E0FF9008421248
:109D4D007D9BD005D0047F0412B986900753E0FBAC
:109D5D0075F004A424F4FDE5F03401FCC004C00545
:109D6D00EB25E025E0244AF582E43400F583E0FCA0
:109D7D00A3E0FDA3E0FEA3E0FF900842127D9BD07F
:109D8D0005D0047F0412B986900753E0FB75F004EB
:109D9D00A42420FDE5F03403FCC004C005EB25E050
:109DAD0025E024F8F582E43401F583E0FCA3E0FD21
:109DBD00A3E0FEA3E0FF900842127D9BD005D004E6
:109DCD007F0412B986900753E0FB75F004A4244C70
:109DDD00FDE5F03404FCC004C005EB25E025E024CE
:109DED007AF582E43405F583E0FCA3E0FDA3E0FE03
:109DFD00A3E0FF900842127D9BD005D0047F041292
:109E0D00B986900753E004F0029CBF9001F2E0FD8B
:109E1D007C007F0A7E0012E1BE900020E0F8A3E0F6
:109E2D00F9A3E0FAA3E0FB127C23900010E0F8A365
:109E3D00E0F9A3E0FAA3E0FBD3127D645016E4FF32
:109E4D00FEFDFC900010E0F8A3E0A3E0A3E0C31238
:109E5D007D4E500A900010127DA700000000900664
:109E6D004FE0FFC394004006EFD394034005E49008
:109E7D00064FF07F9F7E867D017C00900020E0F8EC
:109E8D00A3E0F9A3E0FAA3E0FBD3127D64400A90AE
:109E9D000020127DA7000003E8D3900040E094F469
:109EAD0090003FE094014005E4F0A304F09001F22E
:109EBD00E0D394034002E4F0D3900647E09432904F
:109ECD000646E094004004E4F0A3F090064EE0D383
:109EDD0094014002E4F09002DDE0D394634002E48B
:109EED00F09002C9E0D394014002E4F09001F0E05B
:109EFD00C3940150037405F09001F0E0D394094030
:109F0D00037405F090064DE0C3940150037401F005
:109F1D0090064DE0D3940940037401F0900467E07E
:109F2D00D394014002E4F0D3900045E094099000F1
:109F3D0044E094004005E4F0A304F0D3900027E042
:109F4D009409900026E094004005E4F0A304F0D3BA
:109F5D0090000BE0940990000AE094004006E4F0B4
:109F6D00A37402F09001EEE0D394044002E4F0906B
:109F7D000041E0D3940440037403F0900384E0D3D4
:109F8D0094074002E4F0900466E0D394014002E4AB
:109F9D00F0900018E0D394014002E4F090000EE040
:109FAD00D394054002E4F09002C8E0D39406400239
:109FBD00E4F0D3900465E094E7900464E0940340EA
:109FCD0005E4F0A304F0900004E0D394044003747E
:109FDD0004F0900017E0D3940940037405F090034A
:109FED008DE0D394014002E4F09002D2E0D39401CD
:109FFD004002E4F0900392E0D394024002E4F0902A
:10A00D00045FE0D394014002E4F0900025E0D39486
:10A01D003240037414F0900025E0C3940A50037489
:10A02D0014F0900722E0D394014002E4F0900391E4
:10A03D00E0D394014002E4F0900648E0D39402404E
:10A04D0002E4F0D3900030E0946390002FE0940090
:10A05D004004E4F0A3F0D3900036E0946390003513
:10A06D00E094004004E4F0A3F09001F2E0FD7C00E8
:10A07D007F0A7E0012E1BE900020E0F8A3E0F9A374
:10A08D00E0FAA3E0FB127C23900377E0F8A3E0F95C
:10A09D00A3E0FAA3E0FBD3127D64400A900377128C
:10A0AD007DA7000000009001F2E0FD7C007F0A7E9C
:10A0BD000012E1BE900020E0F8A3E0F9A3E0FAA3BE
:10A0CD00E0FB127C239002CEE0F8A3E0F9A3E0FAC6
:10A0DD00A3E0FBD3127D64400A9002CE127DA7004F
:10A0ED000000009001F2E0FD7C007F0A7E0012E18D
:10A0FD00BE900020E0F8A3E0F9A3E0FAA3E0FB1284
:10A10D007C23900372E0F8A3E0F9A3E0FAA3E0FB4F
:10A11D00D3127D64400A900372127DA700000000E7
:10A12D009001F2E0FD7C007F0A7E0012E1BE9000FE
:10A13D0020E0F8A3E0F9A3E0FAA3E0FB127C239062
:10A14D0002CAE0F8A3E0F9A3E0FAA3E0FBD3127D85
:10A15D0064400A9002CA127DA700000000E47FC08F
:10A16D007E5DFDFC90017DE0F8A3E0F9A3E0FAA38C
:10A17D00E0FBD3127D64400A90017D127DA70000A3
:10A18D000FA0E47FC07E5DFDFC9001EAE0F8A3E046
:10A19D00F9A3E0FAA3E0FBD3127D64400A9001EA33
:10A1AD00127DA700004E20900723E0D394014003B9
:10A1BD007401F090071DE0D394014002E4F0E490A7
:10A1CD000753F0900753E0FB25E025E02493F5823B
:10A1DD00E43403F583127DA700000000EB25E02495
:10A1ED0084F582E43401F583E4F0A3F0900753E0A5
:10A1FD0004F0E0B433CD9002D9127DA70000000029
:07A20D00E4900039F0A3F01A
:01A214002227
:0DBDC8009007E5EFF0A3ECF0FAA3EDF0FB1F
:10BDD5009007EF127DA7000000009007EDEAF0A3A1
:10BDE500EBF09007E5E0FF9007E7E02FFF9007E60F
:10BDF500E03400FE9007EDE0FCA3E0FDC39FEC9E60
:10BE0500400302BFBA9007E974A0F0A304F0ECFF69
:10BE150025E0540EFF9007E8F09007ECEDF074A0D4
:10BE25004F9007E9F0D290D2917F0A7E0012E52F5C
:10BE3500C2917F0A7E0012E52FC290E49007EBF0D5
:10BE45009007E9E0FF30E704D2918002C291EF2527
:10BE5500E09007E9F0D2907F017E0012E52FC290B5
:10BE65007F017E0012E52F9007EBE004F0E0C3941C
:10BE75000840CDD2902091FDC2907F0A7E0012E548
:10BE85002FE49007EBF09007ECE0FF30E704D29148
:10BE95008002C291EF25E09007ECF0D2907F017E01
:10BEA5000012E52FC2907F017E0012E52F9007EB6F
:10BEB500E004F0E0C3940840CDD2902091FDC290FB
:10BEC5007F0A7E0012E52FD2917F027E0012E52FB8
:10BED500D2907F027E0012E52FC2917F027E001272
:10BEE500E52FC2907F027E0012E52F9007EAE0FF62
:10BEF5009007E8E0FEEF4E9007EAF0E4A3F0900724
:10BF0500EAE0FF30E704D2918002C291EF25E0908C
:10BF150007EAF0D2907F017E0012E52FC2907F01E3
:10BF25007E0012E52F9007EBE004F0E0C394084093
:10BF3500CDD2902091FDC2907F0A7E0012E52FE4BC
:10BF45009007EBF0D2909007EFE0FCA3E0FDA3E0B3
:10BF5500FEA3E0FF7801127D889007EF127D9B30EC
:10BF650091199007EFE0FCA3E0FDA3E0FEA3E044F8
:10BF750001FFEEEDEC9007EF127D9BC2909007EB71
:10BF8500E004F0E0B408BDC2907F027E0012E52F08
:10BF9500C2917F027E0012E52FD291D2907F647EFE
:10BFA5000012E52F9007EEE004F070069007EDE033
:10BFB50004F002BDE79007EFE0FCA3E0FDA3E0FE7F
:03BFC500A3E0FFF7
:01BFC8002256
:0BB9860090083FEFF0A3ECF0A3EDF001
:10B99100BF0119A3E0FCA3E0FDA3E0FEA3E0FF7853
:10B9A10018127D88900842127D9B802090083FE00C
:10B9B100B40219900842E0FCA3E0FDA3E0FEA3E07D
:10B9C100FF7810127D88900842127D9B900840E01C
:10B9D100FFA3E090084CCFF0A3EFF090083FE0FF09
:10B9E100900841E02FFF900840E03400FE90084CA1
:10B9F100E0FCA3E0FDC39FEC9E400302BBC29008A4
:10BA010048E4F0A374A0F0EC25E0FFE4337E00EFFE
:10BA1100540EFF900846E4F0A3EDF0E4A3F074A007
:10BA21004FA3F0D290D2917F0A12E52FC2917F02EB
:10BA31007E0012E52FC2907F0A7E0012E52FE4906E
:10BA4100084AF0A3F0900848E0FEA3E0FF30E704C5
:10BA5100D2918002C291EF25E0FFEE33900848F0C9
:10BA6100A3EFF0D2907F027E0012E52FC2907F02F9
:10BA71007E0012E52F90084BE004F0700690084A12
:10BA8100E004F0C390084BE0940890084AE0940069
:10BA910040B3D2902091FD7F027E0012E52FC2902B
:10BAA1007F087E0012E52FE490084AF0A3F0900889
:10BAB10046E0FEA3E0FF30E704D2918002C291EF9D
:10BAC10025E0FFEE33900846F0A3EFF0D2907F021D
:10BAD1007E0012E52FC2907F027E0012E52F9008B2
:10BAE1004BE004F0700690084AE004F0C390084B64
:10BAF100E0940890084AE0940040B3D2902091FD70
:10BB01007F027E0012E52FC2907F027E0012E52F98
:10BB1100E490084AF0A3F0900842E0FCA3E0FDA302
:10BB2100E0FEA3E0E4FFFEFDEC5480FC6004D29152
:10BB31008002C291900842E0FCA3E0FDA3E0FEA3D5
:10BB4100E0FF7801127D88900842127D9BD2907FA0
:10BB5100027E0012E52FC2907F027E0012E52F9037
:10BB6100084BE004F0700690084AE004F0C3900826
:10BB71004BE0940890084AE09400409BD2902091B9
:10BB8100FD7F027E0012E52FC291C2907F027E00EE
:10BB910012E52FC290C2917F027E0012E52FD29052
:10BBA1007F027E0012E52FD2917FF47E0112E52FF4
:10BBB10090084DE004F0700690084CE004F002B9E2
:01BBC100DCA7
:01BBC2002260
:10D5590012E66FEF700302D6527D077C007F0A7EC8
:10D569000012E1BEE41277B1AB25AA24A923A822AF
:10D5790012759E1277EF900762127D9B9008427494
:10D58900FFF0A374E7F0A374BBF0900762E0FCA37B
:10D59900E0FDA3E0FEA3E0FF900845127D9B7B011F
:10D5A9007A07795A12A77F7B017A07795A12E569B6
:10D5B9007FB87E0B12E52F900762E0FCA3E0FDA384
:10D5C900E0FEA3E0FF9007E97404F0127E1E9007C5
:10D5D90062127D9B7D077C007F0A7E0012E1BEE41A
:10D5E9001277B1C004C005C006C007900762E0FC0D
:10D5F900A3E0FDA3E0FEA3E0FFE41277B1D003D0DE
:10D6090002D001D0001276A78F258E248D238C227B
:10D619007B777ACC79AB78321274AD8F258E248DD5
:10D62900238C22900460E0FCA3E0FDA3E0FEA3E0CC
:10D63900FFEC1277B1AB25AA24A923A82212759E63
:09D649001277EF900046127D9B60
:01D6520022B5
:0FE79600202020202020200020202020202000D4
:03E3E70001100022
:10E56900900849EBF0A3EAF0A3E9F0E4F51090086C
:10E5790049E0FBA3E0FAA3E0F98510827583001254
:10E589007B3190D7BD93FF74502510F8A60705106D
:06E59900E510B407D922D1
:0BD34000900757EBF0A3EAF0A3E9F020
:10D34B0012DB4A900757E0FBA3E0FAA3E0F912E7E0
:10D35B005290075EEEF0A3EFF090075A74FFF0A324
:10D36B0074F9F090075EE0FEA3E0FFD390075BE05B
:10D37B009FEE6480F890075AE0648098400302D4D3
:10D38B00507FB87E0B12E52F90075AE0FFA3E0A366
:10D39B00CFF0A3EFF090075BE02406FF90075AE075
:10D3AB003400FE90075CE0FCA3E0FDD39FEE6480AD
:10D3BB00F8EC6480985077C3EC64809480500890AC
:10D3CB00076074FFF0804490075FE024FFFF900735
:10D3DB005EE034FFFED3ED9FEE6480F8EC64809842
:10D3EB00400890076074FFF08021900757E0FBA383
:10D3FB00E0FAA3E0F990075CE0FEA3E0F5828E83F0
:10D40B00127B3190D7BD93900760F0900760E0FFDF
:10D41B0090075BE0FE90075DE0C39E2450F8A607E3
:10D42B00E004F0700690075CE004F002D3A0125BFE
:10D43B0021BFFF1190075BE004F0700690075AE0E4
:05D44B0004F002D36EA5
:01D4500022B9
:06D903009007E5127D9B78
:10D909009007E97407F0E47B0AFAF9F89007E5E073
:10D91900FCA3E0FDA3E0FEA3E0FF12E4A9AF03EF3F
:10D9290090D7ED93FE9007EAF0900116E0F96405AF
:10D939006017E92402FDE433FC9007E9E0B5050925
:10D94900E4B50405EE547FA3F0E92402FFE433FEB5
:10D959009007E9E0C39FEE6480F8748098501FE453
:10D96900FFFEFDFC9007E5E0F8A3E0F9A3E0FAA3C8
:10D97900E0FBC3127D4E70069007EA74FFF0900732
:10D98900E9E0FFB40111900014E0600B9002D7E0C8
:10D9990070057550BF800B9007EAE0FE744F2FF8B1
:10D9A900A6069007E5E0FCA3E0FDA3E0FEA3E0FFE7
:10D9B900E47B0AFAF9F812E4A99007E5127D9B9035
:0BD9C90007E9E014F0E0600302D90F52
:01D9D4002230
:10E59F00900811EBF0A3EAF0A3E9F0E4F51090086E
:10E5AF0011E0FBA3E0FAA3E0F98510827583001256
:10E5BF007B3190D7BD93FF74572510F8A607051030
:06E5CF00E510B406D9229C
:10E5D500900811EBF0A3EAF0A3E9F0E4F510900838
:10E5E50011E0FBA3E0FAA3E0F98510827583001220
:10E5F5007B3190D7BD93FF745D2510F8A6070510F4
:06E60500E510B406D92265
:06DBF400900815127D9B54
:10DBFA00900819740CF0E47B0AFAF9F8900815E019
:10DC0A00FCA3E0FDA3E0FEA3E0FF127CAEAF03EFAE
:10DC1A0090D7ED93FE90081AF0900116E0FD640586
:10DC2A00600E900819E024F9B50505EE547FA3F0BB
:10DC3A00900819E024F9C39D501FE4FFFEFDFC90F3
:10DC4A000815E0F8A3E0F9A3E0FAA3E0FBC3127D0C
:10DC5A0064700690081A74FFF090081AE0FF9008A2
:10DC6A0019E02450F8A607900815E0FCA3E0FDA3EC
:10DC7A00E0FEA3E0FFE47B0AFAF9F8127CAE900812
:10DC8A0015127D9B900819E014F0E0640660030207
:02DC9A00DC00AC
:01DC9C002265
:06DC9D00900815127D9BAA
:10DCA3009008197412F0E47B0AFAF9F8900815E069
:10DCB300FCA3E0FDA3E0FEA3E0FF127CAEAF03EF05
:10DCC30090D7ED93FE90081AF0900116E0FD6405DD
:10DCD300600E900819E024F3B50505EE547FA3F018
:10DCE300900819E024F3C39D501FE4FFFEFDFC9050
:10DCF3000815E0F8A3E0F9A3E0FAA3E0FBC3127D63
:10DD030064700690081A74FFF090081AE0FF9008F8
:10DD130019E02450F8A607900815E0FCA3E0FDA342
:10DD2300E0FEA3E0FFE47B0AFAF9F8127CAE900868
:10DD330015127D9B900819E014F0E0640C60030257
:02DD4300DCA959
:01DD450022BB
:10E70A007BFF7AE7799612E5697BFF7AE7799E12B1
:0CE71A00E59F7BFF7AE7799E12E5D5228F
:10E767002043482030342000202020202020200073
:105B2100900811127DA700000000200D03026827D4
:105B3100C20DE4900390F090000EE0640360030254
:105B410067FD9002DDE0FF75F00A842430FDE43347
:105B5100FC900117E06D7001EC60030267FDEF75C9
:105B6100F00A84E5F02430FFE433FEA3E06F700116
:105B7100EE60030267FDA3E024BB607524FD7003A2
:105B8100025EDC24FC700302637E14604024FE602C
:105B91005214606B24FE60030267EE9002DDE0FFA9
:105BA10012E4ED7F0D12E4ED7F0A12E4ED9001178E
:105BB100E0FF12E4ED7F0D12E4ED7F0A12E4ED90B7
:105BC100011AE0645760030267EE7F652290011AB3
:105BD100E0FEB45A037F6622EE645460030267EE6E
:105BE1007F672290011AE0645060030267EE7F68CC
:105BF1002290011AE0644D60030267EE7F692290F2
:105C0100011AE0644E6003025ED9A3E024D075F06E
:105C11000AA4FFAEF0E4FCFD900811127D9B9008F0
:105C210011E0F8A3E0F9A3E0FAA3E0FB90011CE086
:105C310024D0FFE434FFFEE4FCFDEB2FFFEA3EFE3F
:105C4100ED39FDEC38FC900811127D9BE47F32FEAA
:105C5100FDFC900811E0F8A3E0F9A3E0FAA3E0FB52
:105C6100D3127D4E400612E7777FFF22900813E0A2
:105C7100FFA3E0900646CFF0A3EFF09002DDE075C0
:105C8100F00A842430FF12E4ED9002DDE075F00AA1
:105C910084E5F02430FF12E4ED7F5012E4ED7F4EF5
:105CA10012E4ED900646E0FEA3E0FF7C007D0A12BF
:105CB1007B82EF2430FF12E4ED900646E0FEA3E084
:105CC100FF7C007D0A127B82ED2430FF12E4ED7F20
:105CD1000D12E4ED7F0A12E4ED900646E0FEA3E02A
:105CE1007802C333CE33CED8F9FBAA062450F5820D
:105CF10074063AF583E0FCA3E0FDA3E0FEA3E0FF18
:105D0100900377127D9B74F82BF58274013AF58329
:105D1100E0FCA3E0FDA3E0FEA3E0FF900372127D8F
:105D21009B900646E0FEA3E07802C333CE33CED883
:105D3100F9FBAA06244AF58274003AF583E0FCA334
:105D4100E0FDA3E0FEA3E0FF9002CE127D9B747AFA
:105D51002BF58274053AF583E0FCA3E0FDA3E0FE98
:105D6100A3E0FF9002CA127D9B900646E0FAA3E0F1
:105D7100FBAE027802C333CE33CED8F924C8FDE49A
:105D81003EFCC004C005EBAE027802C333CE33CE75
:105D9100D8F92450F58274063EF583E0FCA3E0FDBA
:105DA100A3E0FEA3E0FF900842127D9BD005D00442
:105DB1007F0412B986900646E0FAA3E0FBAE0278B2
:105DC10002C333CE33CED8F924F4FDEE3401FCC046
:105DD10004C005EBAE027802C333CE33CED8F9242A
:105DE1004AF58274003EF583E0FCA3E0FDA3E0FEEA
:105DF100A3E0FF900842127D9BD005D0047F0412DE
:105E0100B986900646E0FAA3E0FBAE027802C333FE
:105E1100CE33CED8F92420FDEE3403FCC004C005F6
:105E2100EBAE027802C333CE33CED8F924F8F58233
:105E310074013EF583E0FCA3E0FDA3E0FEA3E0FFD7
:105E4100900842127D9BD005D0047F0412B9869040
:105E51000646E0FAA3E0FBAE027802C333CE33CEAE
:105E6100D8F9244CFDEE3404FCC004C005EBAE02AD
:105E71007802C333CE33CED8F9247AF58274053E45
:105E8100F583E0FCA3E0FDA3E0FEA3E0FF90084260
:105E9100127D9BD005D0047F0412B986900646E09E
:105EA100FEA3E0FFE4FCFD900842127D9B7D677C30
:105EB100007F0112B986900377E0FCA3E0FDA3E027
:105EC100FEA3E0FF12DBF49002CEE0FCA3E0FDA311
:105ED100E0FEA3E0FF12DC9D7FFF2290011AE06447
:105EE10049600302614D12D653900811127D9B90B7
:105EF10001F2E0FD7C007F0A7E0012E1BE900020ED
:105F0100E0F8A3E0F9A3E0FAA3E0FB127C239008F8
:105F110011E0F8A3E0F9A3E0FAA3E0FBD3127D645A
:105F21005038900646E0FEA3E07802C333CE33CE6C
:105F3100D8F9244AF58274003EF583E0FCA3E0FD24
:105F4100A3E0FEA3E0FF900811E0F8A3E0F9A3E0CD
:105F5100FAA3E0FBC3127D64500612E7777FFF22AC
:105F6100900811E0FCA3E0FDA3E0FEA3E0FFC00464
:105F7100C005C006C007900646E0FEA3E07802C354
:105F810033CE33CED8F9FBAA062450F58274063AF3
:105F9100F583D007D006D005D004127D9B74502B19
:105FA100F58274063AF583E0FCA3E0FDA3E0FEA3CD
:105FB100E0FF900377127D9B9002DDE075F00A848B
:105FC1002430FF12E4ED9002DDE075F00A84E5F083
:105FD1002430FF12E4ED7F4812E4ED7F4912E4ED35
:105FE100E47B107A27F9F8900811E0FCA3E0FDA307
:105FF100E0FEA3E0FF12E4A9EF2430FF12E4ED90EC
:106001000811E0FCA3E0FDA3E0FEA3E0FFE47B10A8
:106011007A27F9F812E4A9AC00AD01AE02AF039002
:106021000811127D9BE47BE87A03F9F8900811E0EE
:10603100FCA3E0FDA3E0FEA3E0FF12E4A9EF2430FE
:10604100FF12E4ED900811E0FCA3E0FDA3E0FEA344
:10605100E0FFE47BE87A03F9F812E4A9AC00AD01B2
:10606100AE02AF03900811127D9BE47B64FAF9F84C
:10607100900811E0FCA3E0FDA3E0FEA3E0FF12E421
:10608100A9EF2430FF12E4ED900811E0FCA3E0FD3C
:10609100A3E0FEA3E0FFE47B64FAF9F812E4A9AC03
:1060A10000AD01AE02AF03900811127D9BE47B0AA3
:1060B100FAF9F8900811E0FCA3E0FDA3E0FEA3E0EB
:1060C100FF12E4A9EF2430FF12E4ED900811E0FC87
:1060D100A3E0FDA3E0FEA3E0FFE47B0AFAF9F812D6
:1060E100E4A9AC00AD01AE02AF03900811127D9B93
:1060F100900814E02430FF12E4ED7F0D12E4ED7FEF
:106101000A12E4ED900646E0FEA3E07802C333CE26
:1061110033CED8F924C8FDE43EFCC004C005900389
:1061210077E0FCA3E0FDA3E0FEA3E0FF90084212AC
:106131007D9BD005D0047F0412B986900377E0FCE3
:10614100A3E0FDA3E0FEA3E0FF12DBF490011AE05F
:106151006445600302637B12D653900811127D9B44
:10616100900646E0FEA3E07802C333CE33CED8F9E1
:106171002450F58274063EF583E0FCA3E0FDA3E024
:10618100FEA3E0FF900811E0F8A3E0F9A3E0FAA371
:10619100E0FBD3127D64400612E7777FFF2290086F
:1061A10011E0FCA3E0FDA3E0FEA3E0FFC004C005F5
:1061B100C006C007900646E0FEA3E07802C333CED6
:1061C10033CED8F9FBAA0624F8F58274013AF58397
:1061D100D007D006D005D004127D9B74F82BF58230
:1061E10074013AF583E0FCA3E0FDA3E0FEA3E0FF28
:1061F100900372127D9B9002DDE075F00A842430D9
:10620100FF12E4ED9002DDE075F00A84E5F0243040
:10621100FF12E4ED7F4812E4ED7F4512E4EDE47BEB
:10622100107A27F9F8900811E0FCA3E0FDA3E0FE45
:10623100A3E0FF12E4A9EF2430FF12E4ED9008116E
:10624100E0FCA3E0FDA3E0FEA3E0FFE47B107A27DE
:10625100F9F812E4A9AC00AD01AE02AF0390081148
:10626100127D9BE47BE87A03F9F8900811E0FCA326
:10627100E0FDA3E0FEA3E0FF12E4A9EF2430FF124A
:10628100E4ED900811E0FCA3E0FDA3E0FEA3E0FF34
:10629100E47BE87A03F9F812E4A9AC00AD01AE029F
:1062A100AF03900811127D9BE47B64FAF9F8900822
:1062B10011E0FCA3E0FDA3E0FEA3E0FF12E4A9EFDF
:1062C1002430FF12E4ED900811E0FCA3E0FDA3E00F
:1062D100FEA3E0FFE47B64FAF9F812E4A9AC00AD97
:1062E10001AE02AF03900811127D9BE47B0AFAF91B
:1062F100F8900811E0FCA3E0FDA3E0FEA3E0FF128B
:10630100E4A9EF2430FF12E4ED900811E0FCA3E0D2
:10631100FDA3E0FEA3E0FFE47B0AFAF9F812E4A989
:10632100AC00AD01AE02AF03900811127D9B900845
:1063310014E02430FF12E4ED7F0D12E4ED7F0A1228
:10634100E4ED900646E0FEA3E07802C333CE33CEFF
:10635100D8F92420FDEE3403FCC004C0059003727B
:10636100E0FCA3E0FDA3E0FEA3E0FF900842127D64
:106371009BD005D0047F0412B9867FFF2290011AB9
:10638100E0644F60030265BD12D653900811127D7F
:106391009B900646E0FEA3E07802C333CE33CED80D
:1063A100F92450F58274063EF583E0FCA3E0FDA3D9
:1063B100E0FEA3E0FF900811E0F8A3E0F9A3E0FA02
:1063C100A3E0FBD3127D64400612E7777FFF2290A2
:1063D1000811E0FCA3E0FDA3E0FEA3E0FFC004C0C0
:1063E10005C006C007900646E0FEA3E07802C3336D
:1063F100CE33CED8F9FBAA06244AF58274003AF5C9
:1064010083D007D006D005D004127D9B744A2BF5AA
:106411008274003AF583E0FCA3E0FDA3E0FEA3E073
:10642100FF9002CE127D9B9002DDE075F00A84247C
:1064310030FF12E4ED9002DDE075F00A84E5F0240E
:1064410030FF12E4ED7F4C12E4ED7F4F12E4EDE4F6
:106451007B107A27F9F8900811E0FCA3E0FDA3E096
:10646100FEA3E0FF12E4A9EF2430FF12E4ED90084F
:1064710011E0FCA3E0FDA3E0FEA3E0FFE47B107AC2
:1064810027F9F812E4A9AC00AD01AE02AF03900800
:1064910011127D9BE47BE87A03F9F8900811E0FC86
:1064A100A3E0FDA3E0FEA3E0FF12E4A9EF2430FF87
:1064B10012E4ED900811E0FCA3E0FDA3E0FEA3E0EF
:1064C100FFE47BE87A03F9F812E4A9AC00AD01AE70
:1064D10002AF03900811127D9BE47B64FAF9F890F6
:1064E1000811E0FCA3E0FDA3E0FEA3E0FF12E4A994
:1064F100EF2430FF12E4ED900811E0FCA3E0FDA3CE
:10650100E0FEA3E0FFE47B64FAF9F812E4A9AC0031
:10651100AD01AE02AF03900811127D9BE47B0AFA34
:10652100F9F8900811E0FCA3E0FDA3E0FEA3E0FF71
:1065310012E4A9EF2430FF12E4ED900811E0FCA36E
:10654100E0FDA3E0FEA3E0FFE47B0AFAF9F812E420
:10655100A9AC00AD01AE02AF03900811127D9B9072
:106561000814E02430FF12E4ED7F0D12E4ED7F0A00
:1065710012E4ED900646E0FEA3E07802C333CE3389
:10658100CED8F924F4FDEE3401FCC004C00590021C
:10659100CEE0FCA3E0FDA3E0FEA3E0FF90084212E1
:1065A1007D9BD005D0047F0412B9869002CEE0FC19
:1065B100A3E0FDA3E0FEA3E0FF12DC9D90011AE041
:1065C100644560030267EB12D653900811127D9B5C
:1065D100900646E0FEA3E07802C333CE33CED8F96D
:1065E100244AF58274003EF583E0FCA3E0FDA3E0BC
:1065F100FEA3E0FF900811E0F8A3E0F9A3E0FAA3FD
:10660100E0FBD3127D64400612E7777FFF229008FA
:1066110011E0FCA3E0FDA3E0FEA3E0FFC004C00580
:10662100C006C007900646E0FEA3E07802C333CE61
:1066310033CED8F9FBAA06247AF58274053AF5839C
:10664100D007D006D005D004127D9B747A2BF58239
:1066510074053AF583E0FCA3E0FDA3E0FEA3E0FFAF
:106661009002CA127D9B9002DDE075F00A8424300D
:10667100FF12E4ED9002DDE075F00A84E5F02430CC
:10668100FF12E4ED7F4C12E4ED7F4512E4EDE47B73
:10669100107A27F9F8900811E0FCA3E0FDA3E0FED1
:1066A100A3E0FF12E4A9EF2430FF12E4ED900811FA
:1066B100E0FCA3E0FDA3E0FEA3E0FFE47B107A276A
:1066C100F9F812E4A9AC00AD01AE02AF03900811D4
:1066D100127D9BE47BE87A03F9F8900811E0FCA3B2
:1066E100E0FDA3E0FEA3E0FF12E4A9EF2430FF12D6
:1066F100E4ED900811E0FCA3E0FDA3E0FEA3E0FFC0
:10670100E47BE87A03F9F812E4A9AC00AD01AE022A
:10671100AF03900811127D9BE47B64FAF9F89008AD
:1067210011E0FCA3E0FDA3E0FEA3E0FF12E4A9EF6A
:106731002430FF12E4ED900811E0FCA3E0FDA3E09A
:10674100FEA3E0FFE47B64FAF9F812E4A9AC00AD22
:1067510001AE02AF03900811127D9BE47B0AFAF9A6
:10676100F8900811E0FCA3E0FDA3E0FEA3E0FF1216
:10677100E4A9EF2430FF12E4ED900811E0FCA3E05E
:10678100FDA3E0FEA3E0FFE47B0AFAF9F812E4A915
:10679100AC00AD01AE02AF03900811127D9B9008D1
:1067A10014E02430FF12E4ED7F0D12E4ED7F0A12B4
:1067B100E4ED900646E0FEA3E07802C333CE33CE8B
:1067C100D8F9244CFDEE3404FCC004C0059002CA83
:1067D100E0FCA3E0FDA3E0FEA3E0FF900842127DF0
:1067E1009BD005D0047F0412B9867FFF227F3F1220
:1067F100E4ED7F0D12E4ED7F0A12E4ED90000EE06E
:106801006405701F9002DDE0F568900117E0B5683E
:10681100037F65227F3F12E4ED7F0D12E4ED7F0AD5
:1068210012E4ED7FFF2212E4538F67E567B4FF03A3
:0C6831007FFF227FC47E0912E787AF675B
:01683D002238
:10E45300E54F640360FAE54FB403FB7F03EFB54F69
:10E46300FC90FE80E0FD5407FDAE4F0FD3940050A7
:10E4730005E54FB406E7ED70037FFF22ED24FE6050
:10E483001024FE601424037018EE90D81893FE80B5
:10E4930012EE90D81F93FE800AEE90D82693FE804A
:05E4A300027EFFAF0640
:01E4A8002251
:10DB4A00E4900812F0A3127DA700000000E54F64DC
:10DB5A000360FAE54FB403FBE4FBEBB54FFC90FE20
:10DB6A0080E0900811F05407F00BD394004023A3EF
:10DB7A00E004F0A3E0FCA3E0FDA3E0FEA3E024019F
:10DB8A00FFE43EFEE43DFDE43CFC900813127D9B5D
:10DB9A008005E54FB406C3900811E0604C90081266
:10DBAA00E06046E4900812F07FF47E01FDFCA3E0F9
:10DBBA00F8A3E0F9A3E0FAA3E0FBD3127D64408D59
:10DBCA007BFF7AE7796712E56912E7267FA07E0F65
:10DBDA0012E52F7BFF7AE7796F12E5699008131235
:09DBEA007DA70000000002DB57DA
:01DBF300220F
:10E60B00EFB40206752A20752B00EFB403067528AC
:10E61B0020752900C374059FFF14FF7401A8070818
:10E62B008002C333D8FCFFF4FF9001F1E05FF09060
:03E63B00FE40F0AE
:01E63E0022B9
:10E63F00EFB40205E4F52AF52BEFB40305E4F52852
:10E64F00F529C374059FFF14FF7401A80708800202
:0FE65F00C333D8FCFF9001F1E04FF090FE40F084
:01E66E002289
:10D65300900815127DA70000000090011BE024D064
:10D66300FFE434FFFE7C277D10127B70E4FCFD9009
:10D673000815127D9B900815E0F8A3E0F9A3E0FAE2
:10D68300A3E0FBC00090011CE024D0FFE434FFFEC4
:10D693007C037DE8127B70E4FCFDD000EB2FFFEAF6
:10D6A3003EFEED39FDEC38FC900815127D9B900889
:10D6B30015E0F8A3E0F9A3E0FAA3E0FB90011DE075
:10D6C30024D075F064A4FFE4FCFDEB2FFFEA35F0F2
:10D6D300FEED39FDEC38FC900815127D9B90081582
:10D6E300E0F8A3E0F9A3E0FAA3E0FB90011EE02435
:10D6F300D075F00AA4FFE4FCFDEB2FFFEA35F0FE42
:10D70300ED39FDEC38FC900815127D9B900815E06F
:10D71300F8A3E0F9A3E0FAA3E0FB90011FE024D013
:10D72300FFE434FFFEE4FCFDEB2FFFEA3EFEED39A0
:10D73300FDEC38FC900815127D9B900815E0FCA3C6
:08D74300E0FDA3E0FEA3E0FFFE
:01D74B0022BB
:10E0B300204348203032200020434C454152200069
:10E0C300202053455450004F494E542020005020E7
:10E0D300484F4C4420002020484F4C4420004944E2
:10E0E30020434F44450020205441524520004849D5
:10E0F3002046414C4C004C4F2046414C4C0020489C
:10E10300492020202000204C4F20202020002020C8
:10E1130053544F5020002053544152542000205454
:10E123004152452020002020202020202000204F85
:06E13300554552202000BA
:07E3EA0044086F0000000071
:10002600C200E4900753F0A304F0E4900757F09061
:10003600075904F0E4A3F090075FF0A304F0E4A3EB
:10004600F0A3F0900767F0A3F0A3F0A3F090078663
:10005600127DA700000000E490078AF0A3F0900745
:1000660090F074FFA3F0A3F0A3127DA70000000098
:10007600E4900797F0A3F0A3F0A3F0A3F0A3F09009
:1000860007B9127DA7000000009007BD127DA700EA
:100096000000009007C1127DA7000000009007CD68
:1000A600127DA700000000E49007D5F0A3F0A3F0AE
:1000B600A3F0A3F0A3F09007DCF0A3127DA7000045
:1000C60000009007E1127DA7000000007F0112E604
:1000D6003F7F0212E63F7F0312E63F7F0412E63FB0
:1000E6009001F2E0FF70089001167405F08022EF8F
:1000F600B401089001167404F08016EFB40208905B
:1001060001167403F0800AEFB40306900116740218
:10011600F0E490076CF0A3F09001F0E02402FFE415
:1001260033FEC390076DE09FEE6480F890076CE0A5
:10013600648098501912CB2E90078C127D9B9007E5
:100146006DE004F0700690076CE004F080CAE47F6E
:100156000AFEFDFC90078CE0F8A3E0F9A3E0FAA301
:10016600E0FBC3127D6440197F407E427D0F7C0018
:1001760090078CE0F8A3E0A3E0A3E0D3127D6440EF
:10018600187BFF7AE079B312E5697FC47E0912E72E
:10019600877F887E1312E52F229001F2E0FD7C0016
:1001A6007F0A7E0012E1BE900020E0F8A3E0F9A3EA
:1001B600E0FAA3E0FB127C2390077E127D9B900061
:1001C6002BE0FCA3E0FDA3E0FEA3E0FFE41277B181
:1001D600AB25AA24A923A82212759E1277EF9007B1
:1001E600C5127D9B90003FE0FEA3E0FFE4FCFD7B93
:1001F60009FAF9F8127C2390077EE0F8A3E0F9A348
:10020600E0FAA3E02FFFEA3EFEE93DFDE83CFC9064
:100216000776127D9B90003FE0FEA3E0FFE4FCFD25
:10022600F8F9AA06AB0790077EE0FCA3E0FDA3E081
:10023600FEA3E0FF12E4A9E47B0AFAF9F8127C2394
:1002460090077A127D9B900466E0601F90077AE023
:10025600FCA3E0FDA3E0FEA3E0FFE47B05FAF9F8CA
:1002660012E4A990077A127D9B801D90077AE0FC24
:10027600A3E0FDA3E0FEA3E0FFE47B19FAF9F81280
:10028600E4A990077A127D9B900045E075F00AA4D8
:100296009001EFF0900026E0FEA3E0FF4E700C9078
:1002A60007657407F0A374D0F0800F7C077DD01229
:1002B6007B70900765EEF0A3EFF090000BE075F011
:1002C60014A490003DF07003740EF012E3F2900057
:1002D60040E0FF900017E0FEEF8EF0A490076BF071
:1002E600900015E4F0A304F0C200900006127DA76A
:1002F6000000000090000EE0600312D9D59006467B
:10030600E0FEA3E07802C333CE33CED8F9FBAA06CB
:100316002450F58274063AF583E0FCA3E0FDA3E0E1
:10032600FEA3E0FF900377127D9B744A2BF582743F
:10033600003AF583E0FCA3E0FDA3E0FEA3E0FF9016
:1003460002CE127D9B900646E0FEA3E07802C33300
:10035600CE33CED8F9FBAA0624F8F58274013AF515
:1003660083E0FCA3E0FDA3E0FEA3E0FF900372128E
:100376007D9B747A2BF58274053AF583E0FCA3E045
:10038600FDA3E0FEA3E0FF9002CA127D9B900377D7
:10039600E0FCA3E0FDA3E0FEA3E0FF12DBF4900285
:1003A600CEE0FCA3E0FDA3E0FEA3E0FF12DC9D127D
:1003B600E139900389127DA700000000E490071C34
:1003C600F09001F7F090001EF0A3F09001F2E0FD2E
:1003D600700790079AE054E3F0EDB4010790079A8E
:1003E600E04404F0EDB4020790079AE04408F0ED0B
:1003F600B4030790079AE04410F090FE41E090079E
:1004060056F0540FF0125B218F4C900391E070066A
:1004160090071DE06010E54CB40803754C0AE54CE6
:10042600B40903754C0CE54CB4FF0B900756E06419
:100436000F7003021CAB900756E024F5700302050B
:100446001F24FE70030205761470030205DC147087
:10045600030206462408600302064E9002C8E02402
:10046600FB500B60191470030204F902050F900784
:10047600557401F07FC47E0912E787020654900086
:1004860010127DA700000000E4900024F0F530F57E
:100496003190018304F0900010E0FCA3E0FDA3E09E
:1004A600FEA3E0FF900842127D9B7D147C007F0432
:1004B60012B986900024E0FFE4FCFDFE900842128B
:1004C6007D9B7D5E7C007F0112B986900183E0FFF3
:1004D600E4FCFDFE900842127D9B7D717C007F014D
:1004E60012B9869007557428F07FC47E0912E787F3
:1004F6000206549001837401F09007557428F07F2A
:10050600C47E0912E7870206549007557428F07FC7
:10051600C47E0912E7870206549002C8E024FC60F4
:100526000A240424FA501460228035900755740773
:10053600F07FC47E0912E7870206549007557403BC
:10054600F07FC47E0912E787020654E4900183F027
:100556009007557428F07FC47E0912E78702065477
:100566009007557428F07FC47E0912E78702065467
:100576009002C8E0603C14602914601624FB500207
:1005860080459007557408F07FC47E0912E78702FC
:100596000654900755740AF07FC47E0912E7870255
:1005A60006549007557407F07FC47E0912E7870248
:1005B6000654E4900183F09007557428F07FC47EBA
:1005C6000912E7870206549007557428F07FC47E07
:1005D6000912E78780789002C8E0604014602E1404
:1005E600601424FB500280499007557409F07FC4BB
:1005F600FE12E7878058E49002D7F090075404F083
:10060600A37428F07FC47E0912E7878041900755BE
:100616007402F07FC47E0912E787803290018374EA
:1006260001F09007557428F07FC47E0912E7878091
:100636001D9007557428F07FC47E0912E787800E47
:10064600900755E54CF080069007557428F0900702
:1006560056E0640F602F7F647E0012E52FD390076B
:10066600D6E094C89007D5E09400500CA3E004F0BF
:1006760070069007D5E004F090FE41E0900756F032
:10068600540FF080C9E49007D5F0A3F0900755E029
:100696006402600302074390000CF0A3F0E54F608C
:1006A600FCE54F70FCE49007DBF09007DBE0B54F0C
:1006B600F990FE80E0FF3395E090076CF0A3EFF031
:1006C6007E005407FF90076CEEF0A3EFF09007DB77
:1006D600E004F0D3EF9400748094804006A3E00415
:1006E600F08005E54FB412C290076CE07002A3E0FB
:1006F600604B9007DCE06045E49007DCF0D39000A7
:100706000DE094A090000CE0940F40917FC47E0908
:1007160012E78790017B7401F0E490000CF0A3F0DF
:10072600F526F527F528F529F52AF52BF52CF52DCF
:10073600F52EF52FF530F531F532F53322900755C4
:10074600E060030209EB90000CF0A3F0E54F60FCBB
:10075600E54F70FCE49007DBF09007DBE0B54FF95E
:1007660090FE80E0FF3395E090076CF0A3EFF07EFB
:10077600005407FF90076CEEF0A3EFF09007DBE064
:1007860004F0D3EF9400748094804006A3E004F054
:100796008005E54FB412C290076CE07002A3E070CA
:1007A600030209EB9007DCE070030209EBE4900713
:1007B600DCF0D390000DE094A090000CE0940F4084
:1007C6008B7FC47E0912E787E490000CF0A3F0F556
:1007D60026F527F528F529F52AF52BF52CF52DF51F
:1007E6002EF52FF530F531F532F5337BFF7AE079CA
:1007F600BB12E5697BFF7AE079C312E59F7BFF7A3E
:10080600E079CA12E5D5E490076CF0A3F090076C86
:10081600E0FEA3E0FFC39433EE64809480400302BD
:10082600099AEF7802C333CE33CED8F9FBAA062451
:1008360050F58274063AF583127DA7000000007415
:100846004A2BF58274003AF583127DA7000000005A
:1008560090076CE0FEA3E07802C333CE33CED8F91E
:10086600FBAA0624F8F58274013AF583127DA700E7
:10087600000000747A2BF58274053AF583127DA781
:100886000000000090076CE0FEA3E07802C333CEC0
:1008960033CED8F9FF24C8FDE43EFCC004C005747D
:1008A600502FF58274063EF583E0FCA3E0FDA3E03D
:1008B600FEA3E0FF900842127D9BD005D0047F0482
:1008C60012B98690076CE0FEA3E07802C333CE33FC
:1008D600CED8F9FF24F4FDEE3401FCC004C0057443
:1008E6004A2FF58274003EF583E0FCA3E0FDA3E009
:1008F600FEA3E0FF900842127D9BD005D0047F0442
:1009060012B98690076CE0FEA3E07802C333CE33BB
:10091600CED8F9FF2420FDEE3403FCC004C00574D4
:10092600F82FF58274013EF583E0FCA3E0FDA3E019
:10093600FEA3E0FF900842127D9BD005D0047F0401
:1009460012B98690076CE0FEA3E07802C333CE337B
:10095600CED8F9FF244CFDEE3404FCC004C0057467
:100966007A2FF58274053EF583E0FCA3E0FDA3E053
:10097600FEA3E0FF900842127D9BD005D0047F04C1
:1009860012B98690076DE004F0700690076CE004DB
:10099600F0020813900646E0FEA3E07802C333CEC9
:1009A60033CED8F9FBAA062450F58274063AF583AD
:1009B600E0FCA3E0FDA3E0FEA3E0FF900377127D39
:1009C6009B744A2BF58274003AF583E0FCA3E0FDA4
:1009D600A3E0FEA3E0FF9002CE127D9B9007557424
:1009E6006FF0020752900755E0127DF80F05000AD6
:1009F60057011386020CCA0313F00413F00513F013
:100A060006131E071BD6081B51090C570A13C60BE3
:100A160011780C13DB461CA1650A57660CCA671BC6
:100A2600D6681B51690A326F00001CA8900377E054
:100A3600FCA3E0FDA3E0FEA3E0FF12DBF49002CEF0
:100A4600E0FCA3E0FDA3E0FEA3E0FF12DC9D021C98
:100A5600A89002D7E0600EE54CB4660312E7771261
:100A6600E726021CA8900018E070389002D8E070C3
:100A760032E54CB4660312E777E4F526F527F52848
:100A8600F529F52AF52BF52CF52DF52EF52FF53054
:100A9600F531F532F53312E7267FA07E0F12E52FEA
:100AA600021CA8900024E0600612E726021CA8900B
:100AB600078CE0FCA3E0FDA3E0FEA3E0FF9007C9DE
:100AC600127D9B9007C9E0FCA3E0FDA3E0FEA3E036
:100AD600FFEC1277B1AB25AA24A923A82212759E92
:100AE6001277EF9007C9127D9B90037CE0FCA3E090
:100AF600FDA3E0FEA3E0FF9007C9E0F8A3E0F9A399
:100B0600E0FAA3E0FBD3127D4E402E90037CE0F882
:100B1600A3E0F9A3E0FAA3E0FB9007C9E0FCA3E099
:100B2600FDA3E0FEA3E09BFFEE9AFEED99FDEC9897
:100B3600FC90076E127D9B802D9007C9E0F8A3E01C
:100B4600F9A3E0FAA3E0FB90037CE0FCA3E0FDA39D
:100B5600E0FEA3E0C39BFFEE9AFEED99FDEC98FC48
:100B660090076E127D9B90077AE0FCA3E0FDA3E060
:100B7600FEA3E0FF90076EE0F8A3E0F9A3E0FAA376
:100B8600E0FBD3127D4E4003020C2590078CE0FC5F
:100B9600A3E0FDA3E0FEA3E0FF900046127D9B903C
:100BA6000046E0FCA3E0FDA3E0FEA3E0FF900842C0
:100BB600127D9BE4FDFC7F0412B986900046E0FCA2
:100BC600A3E0FDA3E0FEA3E0FFEC1277B1AB25AAFC
:100BD60024A923A82212759E1277EF900046127D53
:100BE6009BE54C64666003021CA89002DDE075F08C
:100BF6000A842430FF12E4ED9002DDE075F00A84E9
:100C0600E5F02430FF12E4ED7F4D12E4ED7F5A1239
:100C1600E4ED7F0D12E4ED7F0A12E4ED021CA8E577
:100C26004CB4660312E777E4F526F527F528F5298F
:0C0C3600F52AF52BF52CF52DF52EF52FE9
:100C4200F530F531F532F5337FA07E0F12E52F1224
:100C5200E726021CA8900024E0600C900183E0606B
:100C62000612E726021CA89002D7E0700B04F0E4FB
:100C720090000CF0A3F0800AE49002D7F0900754A1
:100C820004F09002D7E060229002D2E0B4010B7B24
:100C9200FF7AE079D112E56980097BFF7AE079D9A0
:100CA20012E5697FA07E0F12E52F90086F127DA7D3
:100CB20000000000E4900767F0A3F0900793127D14
:100CC200A700000000021CA89002D7E0600EE54CCD
:100CD200B4670312E77712E726021CA8900018E017
:100CE20070389002D8E07032E54CB4670312E777AF
:100CF200E4F526F527F528F529F52AF52BF52CF547
:100D02002DF52EF52FF530F531F532F53312E726B4
:100D12007FA07E0F12E52F021CA890076AE0600EEA
:100D2200E54CB4670312E77712E726021CA8E4FF3A
:100D3200FEFDFC900389E0F8A3E0F9A3E0FAA3E04A
:100D4200FBC3127D4E7051900010127DA70000006F
:100D520000E4900024F090018304F0E4F530F531D2
:100D6200900010E0FCA3E0FDA3E0FEA3E0FF9008EA
:100D720042127D9B7D147C007F0412B98690002470
:100D8200E0FFE4FCFDFE900842127D9B7D5E7C004C
:100D92007F0112B986021CA89001F2E0FD7C007F5F
:100DA2000A7E0012E1BE900020E0F8A3E0F9A3E081
:100DB200FAA3E0FB127C23900389E0F8A3E0F9A3F5
:100DC200E0FAA3E0FBD3127D64400EE54CB4670366
:100DD20012E77712E726021CA8900046E0FCA3E087
:100DE200FDA3E0FEA3E0FF900380E0F8A3E0F9A3F7
:100DF200E0FAA3E0FBD3127D4E505CE54CB46703EE
:100E020012E77712E726900010127DA7000000007B
:100E1200E4900024F090018304F0E4F530F5319081
:100E22000010E0FCA3E0FDA3E0FEA3E0FF90084277
:100E3200127D9B7D147C007F0412B986900024E011
:100E4200FFE4FCFDFE900842127D9B7D5E7C007FEC
:100E52000112B986021CA8900389E0FCA3E0FDA35D
:100E6200E0FEA3E0FF900010127D9B90002474012D
:100E7200F0E4900183F0F530753110E54C64677051
:100E8200329002DDE075F00A842430FF12E4ED9026
:100E920002DDE075F00A84E5F02430FF12E4ED7F14
:100EA2004D12E4ED7F5412E4ED7F0D12E4ED7F0A62
:100EB20012E4ED900010E0FCA3E0FDA3E0FEA3E04D
:100EC200FF900842127D9B7D147C007F0412B9863C
:100ED200900024E0FFE4FCFDFE900842127D9B7D21
:100EE2005E7C007F0112B986900183E0FFE4FCFD85
:100EF200FE900842127D9B7D717C007F0112B986B3
:100F0200021CA89002D7E0600612E726021CA8E4A1
:100F1200F526F527F528F529F52AF52BF52CF52DDB
:100F2200F52EF52FF530F531F532F5337BFF7AE00A
:100F320079E112E5697FA07E0F12E52F900646E067
:100F4200FAA3E0FBFFAE02E4FCFD9007E1127D9BF9
:100F5200AF03AE02E4FCFD9007E97408F0127E1EB6
:100F6200900646EEF0A3EFF0D39432EE9400401CCC
:100F720012E7267FA07E0F12E52F9007E3E0FFA382
:100F8200E0900646CFF0A3EFF0021CA8900646E0E0
:100F9200FEA3E07802C333CE33CED8F924C8FDE4F1
:100FA2003EFC7F0412BDC8C004C005C006C0079045
:100FB2000646E0FAA3E0FBAE027802C333CE33CE9C
:100FC200D8F92450F58274063EF583D007D006D0B6
:100FD20005D004127D9BEBAE027802C333CE33CE32
:100FE200D8F924F4FDEE3401FC7F0412BDC8C0041C
:100FF200C005C006C007900646E0FAA3E0FBAE02B9
:101002007802C333CE33CED8F9244AF58274003E37
:10101200F583D007D006D005D004127D9BEBAE023B
:101022007802C333CE33CED8F92420FDEE3403FC4C
:101032007F0412BDC8C004C005C006C007900646A2
:10104200E0FAA3E0FBAE027802C333CE33CED8F986
:1010520024F8F58274013EF583D007D006D005D07E
:1010620004127D9BEBAE027802C333CE33CED8F9A5
:10107200244CFDEE3404FC7F0412BDC8C004C0053C
:10108200C006C007900646E0FEA3E07802C333CE56
:1010920033CED8F9FBAA06247AF58274053AF58391
:1010A200D007D006D005D004127D9B74502BF58258
:1010B20074063AF583E0FCA3E0FDA3E0FEA3E0FFA3
:1010C200900377127D9B900646E0FEA3E07802C370
:1010D20033CE33CED8F9FBAA0624F8F58274013A4E
:1010E200F583E0FCA3E0FDA3E0FEA3E0FF90037222
:1010F200127D9B744A2BF58274003AF583E0FCA3BF
:10110200E0FDA3E0FEA3E0FF9002CE127D9B9006DD
:1011120046E0FAA3E0FBAE027802C333CE33CED868
:10112200F9247AF58274053EF583E0FCA3E0FDA381
:10113200E0FEA3E0FF9002CA127D9BAF03AE02E481
:10114200FCFD900842127D9B7D677C007F0112B9F5
:1011520086900377E0FCA3E0FDA3E0FEA3E0FF128C
:10116200DBF49002CEE0FCA3E0FDA3E0FEA3E0FFEF
:1011720012DC9D021CA89002D7E0600612E726024C
:101182001CA8E4F526F527F528F529F52AF52BF50F
:101192002CF52DF52EF52FF530F531F532F5337BA3
:1011A200FF7AE079E912E5697FA07E0F12E52F90C0
:1011B2000010E0FCA3E0FDA3E0FEA3E0FF9007E93E
:1011C2007407F0127E1E900782127D9B90003FE012
:1011D200FEA3E0FFE4FCFDF8F9AA06AB0790078244
:1011E200E0FCA3E0FDA3E0FEA3E0FF12E4A9AF034D
:1011F200900763EAF0A3EFF0900782E0FCA3E0FD22
:10120200A3E0FEA3E0FFC004C005C006C00790072C
:1012120063E0FEA3E0FFE4FCFDAA06AB07D007D023
:1012220006D005D004C3EF9BFFEE9AFEED9400FDBD
:10123200EC9400FC900782127D9B9001F2E0FD7C11
:10124200007F0A7E0012E1BE900020E0F8A3E0F9E0
:10125200A3E0FAA3E0FB127C23900782E0F8A3E06C
:10126200F9A3E0FAA3E0FBD3127D64401612E7264D
:101272007FA07E0F12E52F900782127DA70000004B
:10128200008049900782E0FCA3E0FDA3E0FEA3E01A
:10129200FF900010127D9B900010E0FCA3E0FDA3E4
:1012A200E0FEA3E0FFEC4D4E4F601390002474016A
:1012B200F0753020753100E4900183F0800EE490E7
:1012C2000024F0F530F53190018304F0900010E035
:1012D200FCA3E0FDA3E0FEA3E0FF900842127D9B89
:1012E2007D147C007F0412B986900024E0FFE4FCA8
:1012F200FDFE900842127D9B7D5E7C007F0112B94B
:1013020086900183E0FFE4FCFDFE900842127D9B83
:101312007D717C007F0112B986021CA89002D7E081
:10132200601B9002D2E0B4011490086FE0FCA3E0CD
:10133200FDA3E0FEA3E0FF9001F3127D9B9001EE7E
:10134200E0701590000EE064046003021CA8D2B4A1
:1013520012B372C2B4021CA812683EE490071CF0D9
:101362009001F7F0900467E060127F1B12E2B07FF9
:101372005012E2B07F0112E2B0021CA8E4900467AE
:10138200F0021CA89002D7E0600612E726021CA811
:10139200900024E07003021CA8900183E06004E442
:1013A200F080069001837401F0900183E0FFE4FC79
:1013B200FDFE900842127D9B7D717C007F0112B977
:1013C20086021CA89002D7E0600612E726021CA83B
:1013D20090071C7401F0021CA89002D7E06006126C
:1013E200E726021CA89001F77401F0021CA89002E3
:1013F200D7E0700690071DE0600612E726021CA8DF
:1014020090075AE0700302178C900755E06404605D
:10141200030215C990076CF0A3F090076DE025E078
:101422002426F8E4F608F6E004F0700690076CE073
:1014320004F090076CE07004A3E0640770DC7BFFAB
:101442007AE079F112E5697FA07E0F12E52F90060E
:1014520046E0FEA3E07802C333CE33CED8F924F8B7
:10146200F58274013EF583E0FCA3E0FDA3E0FEA358
:10147200E0FF9007E97409F0127E1E900782127D48
:101482009B90003FE0FEA3E0FFE4FCFDF8F9AA0612
:10149200AB07900782E0FCA3E0FDA3E0FEA3E0FF20
:1014A20012E4A9AF03900763EAF0A3EFF09007827A
:1014B200E0FCA3E0FDA3E0FEA3E0FFC004C005C082
:1014C20006C007900763E0FEA3E0FFE4FCFDAA0666
:1014D200AB07D007D006D005D004C3EF9BFFEE9A2E
:1014E200FEED9400FDEC9400FC900782127D9B902F
:1014F2000646E0FEA3E07802C333CE33CED8F92409
:1015020050F58274063EF583E0FCA3E0FDA3E0FE05
:10151200A3E0FF900782E0F8A3E0F9A3E0FAA3E0DA
:10152200FBD3127D64400D12E7267FA07E0F12E5E9
:101532002F021784900782E0FCA3E0FDA3E0FEA344
:10154200E0FFC004C005C006C007900646E0FEA347
:10155200E07802C333CE33CED8F9FBAA0624F8F5DD
:101562008274013AF583D007D006D005D004127DEB
:101572009B74F82BF58274013AF583E0FCA3E0FD3D
:10158200A3E0FEA3E0FF900372127D9B900646E06B
:10159200FEA3E07802C333CE33CED8F92420FDEE89
:1015A2003403FCC004C005900372E0FCA3E0FDA379
:1015B200E0FEA3E0FF900842127D9BD005D0047F9D
:1015C2000412B986021784900755E064056003028D
:1015D200178490076CF0A3F090076DE025E02426B5
:1015E200F8E4F608F6E004F0700690076CE004F008
:1015F20090076CE07004A3E0640770DC7BFF7AE084
:1016020079F912E5697FA07E0F12E52F900646E078
:10161200FEA3E07802C333CE33CED8F9247AF58222
:1016220074053EF583E0FCA3E0FDA3E0FEA3E0FF2A
:101632009007E97409F0127E1E900782127D9B903A
:10164200003FE0FEA3E0FFE4FCFDF8F9AA06AB07C9
:10165200900782E0FCA3E0FDA3E0FEA3E0FF12E41A
:10166200A9AF03900763EAF0A3EFF0900782E0FCD2
:10167200A3E0FDA3E0FEA3E0FFC004C005C006C0D6
:1016820007900763E0FEA3E0FFE4FCFDAA06AB07B8
:10169200D007D006D005D004C3EF9BFFEE9AFEED33
:1016A2009400FDEC9400FC900782127D9B9006460C
:1016B200E0FEA3E07802C333CE33CED8F9244AF554
:1016C2008274003EF583E0FCA3E0FDA3E0FEA3E00C
:1016D200FF900782E0F8A3E0F9A3E0FAA3E0FBD3CE
:1016E200127D64400D12E7267FA07E0F12E52F02C5
:1016F2001784900782E0FCA3E0FDA3E0FEA3E0FFD5
:10170200C004C005C006C007900646E0FEA3E0780C
:1017120002C333CE33CED8F9FBAA06247AF58274FB
:10172200053AF583D007D006D005D004127D9B740C
:101732007A2BF58274053AF583E0FCA3E0FDA3E081
:10174200FEA3E0FF9002CA127D9B900646E0FEA334
:10175200E07802C333CE33CED8F9244CFDEE340404
:10176200FCC004C0059002CAE0FCA3E0FDA3E0FEB9
:10177200A3E0FF900842127D9BD005D0047F0412A3
:10178200B986E490075AF0021B2C900755E06404D6
:10179200600302196990076CF0A3F090076DE025D1
:1017A200E02426F8E4F608F6E004F0700690076CF0
:1017B200E004F090076CE07004A3E0640770DC7B47
:1017C200FF7AE1790112E5697FA07E0F12E52F9081
:1017D2000646E0FEA3E07802C333CE33CED8F92426
:1017E20050F58274063EF583E0FCA3E0FDA3E0FE23
:1017F200A3E0FF9007E97409F0127E1E900782129F
:101802007D9B90003FE0FEA3E0FFE4FCFDF8F9AA17
:1018120006AB07900782E0FCA3E0FDA3E0FEA3E095
:10182200FF12E4A9AF03900763EAF0A3EFF0900779
:1018320082E0FCA3E0FDA3E0FEA3E0FFC004C0053C
:10184200C006C007900763E0FEA3E0FFE4FCFDAA28
:1018520006AB07D007D006D005D004C3EF9BFFEE3E
:101862009AFEED9400FDEC9400FC900782127D9BA1
:1018720090077EE0FCA3E0FDA3E0FEA3E0FFA3E06F
:10188200F8A3E0F9A3E0FAA3E0FBD3127D4E5038AF
:10189200900646E0FEA3E07802C333CE33CED8F9F9
:1018A200244AF58274003EF583E0FCA3E0FDA3E048
:1018B200FEA3E0FF900782E0F8A3E0F9A3E0FAA319
:1018C200E0FBC3127D64500D12E7267FA07E0F124B
:1018D200E52F021B2C900782E0FCA3E0FDA3E0FEB3
:1018E200A3E0FFC004C005C006C007900646E0FEA4
:1018F200A3E07802C333CE33CED8F9FBAA06245034
:10190200F58274063AF583D007D006D005D00412CA
:101912007D9B74502BF58274063AF583E0FCA3E0BC
:10192200FDA3E0FEA3E0FF900377127D9B900646A5
:10193200E0FEA3E07802C333CE33CED8F924C8FD4B
:10194200E43EFCC004C005900377E0FCA3E0FDA3E5
:10195200E0FEA3E0FF900842127D9BD005D0047FF9
:101962000412B986021B2C900755E064056003023D
:101972001B2690076CF0A3F090076DE025E024266B
:10198200F8E4F608F6E004F0700690076CE004F064
:1019920090076CE07004A3E0640770DC7BFF7AE1DF
:1019A200790912E5697FA07E0F12E52F900646E0C5
:1019B200FEA3E07802C333CE33CED8F9244AF582AF
:1019C20074003EF583E0FCA3E0FDA3E0FEA3E0FF8C
:0C19D2009007E97409F0127E1E90078255
:1019DE00127D9B90003FE0FEA3E0FFE4FCFDF8F9D2
:1019EE00AA06AB07900782E0FCA3E0FDA3E0FEA3EE
:1019FE00E0FF12E4A9AF03900763EAF0A3EFF090C3
:101A0E000782E0FCA3E0FDA3E0FEA3E0FFC004C05C
:101A1E0005C006C007900763E0FEA3E0FFE4FCFDEF
:101A2E00AA06AB07D007D006D005D004C3EF9BFFA4
:101A3E00EE9AFEED9400FDEC9400FC900782127D70
:101A4E009B900646E0FEA3E07802C333CE33CED899
:101A5E00F92450F58274063EF583E0FCA3E0FDA365
:101A6E00E0FEA3E0FF900782E0F8A3E0F9A3E0FA1E
:101A7E00A3E0FBD3127D64400D12E7267FA07E0FFC
:101A8E0012E52F021B2C900782E0FCA3E0FDA3E0E1
:101A9E00FEA3E0FFC004C005C006C007900646E0E6
:101AAE00FEA3E07802C333CE33CED8F9FBAA0624C8
:101ABE004AF58274003AF583D007D006D005D004DB
:101ACE00127D9B744A2BF58274003AF583E0FCA3D9
:101ADE00E0FDA3E0FEA3E0FF9002CE127D9B9006F8
:101AEE0046E0FEA3E07802C333CE33CED8F924F419
:101AFE00FDEE3401FCC004C0059002CEE0FCA3E074
:101B0E00FDA3E0FEA3E0FF900842127D9BD005D01E
:101B1E00047F0412B986800690075A7401F0900370
:101B2E0077E0FCA3E0FDA3E0FEA3E0FF12DBF49060
:101B3E0002CEE0FCA3E0FDA3E0FEA3E0FF12DC9DDD
:101B4E00021CA89002D7E0700690071DE0600EE51B
:101B5E004CB4690312E77712E726021CA890000422
:101B6E00E064037055E54C646970329002DDE075F7
:101B7E00F00A842430FF12E4ED9002DDE075F00AE5
:101B8E0084E5F02430FF12E4ED7F4512E4ED7F4D45
:101B9E0012E4ED7F0D12E4ED7F0A12E4ED7BFF7A85
:101BAE00E1791112E5697FA07E0F12E52F7F0212F7
:101BBE00E63F7F0312E63F021CA8E54CB469031210
:101BCE00E77712E726021CA89002D7E0700690076E
:101BDE001DE0600EE54CB4680312E77712E72602AB
:101BEE001CA8900004E064036003021C9490076B31
:101BFE00E0FFE4FCFDFE9001F3E0F8A3E0F9A3E0C2
:101C0E00FAA3E0FBD3127D4E505A9007D97401F01F
:101C1E00E54C646870329002DDE075F00A84243081
:101C2E00FF12E4ED9002DDE075F00A84E5F0243059
:101C3E00FF12E4ED7F4F12E4ED7F5012E4ED7F0DC5
:101C4E0012E4ED7F0A12E4ED7BFF7AE1791912E5D9
:101C5E00697FA07E0F12E52F7F0212E60B7F031223
:101C6E00E60B8036E54CB4680312E7777BFF7AE12A
:101C7E00792112E56912E7267FA07E0F12E52FE487
:101C8E009007D9F08014E54CB4680312E77712E799
:101C9E00268007D2B412B372C2B412DB4A90075434
:101CAE00E07049D3900762E09446900761E094009B
:101CBE00401D12E7267FA07E0F12E52F9007547469
:101CCE0001F0E4900761F0A3F090075AF0801DD365
:101CDE00900768E0940E900767E09400500E90070E
:101CEE0062E004F07006900761E004F012CB2E90D3
:101CFE00078C127D9B7F407E427D0F7C0090046995
:101D0E00E0F8A3E0F9A3E0FAA3E0FBD3127D645060
:101D1E001AE47F0AFEFDFC900469E0F8A3E0A3E05C
:101D2E00A3E0C3127D644003021DC0E490076CF073
:101D3E00A3F090076DE025E02426F8E4F608F6E01F
:101D4E0004F0700690076CE004F090076CE07004ED
:101D5E00A3E0640770DC7BFF7AE079B312E569904B
:101D6E00FE437482F090FE4074FFF090FE42E4F069
:101D7E007F0AFE12E52F90FE037488F090FE027427
:101D8E0002F07F327E0012E52F12DF1112E3F27F96
:101D9E00647E0012E52F12C9C7900469127D9B1252
:101DAE00CB2E90078C127D9B7F647E0012E52F0256
:101DBE001D0390078CE0FCA3E0FDA3E0FEA3E0FF73
:101DCE00E41277B190075B127D9B900754E070038D
:101DDE0002040090075BE0FCA3E0FDA3E0FEA3E09D
:101DEE00FFAB25AA24A923A82212759E1277EF9085
:101DFE000380127D9B900786E0FCA3E0FDA3E0FE2E
:101E0E00A3E0FFEC4D4E4F7014900380E0FCA3E076
:101E1E00FDA3E0FEA3E0FF900786127D9B90004697
:101E2E00E0FCA3E0FDA3E0FEA3E0FF900380E0F85A
:101E3E00A3E0F9A3E0FAA3E0FBD3127D4E402E906F
:101E4E000046E0F8A3E0F9A3E0FAA3E0FB900380DC
:101E5E00E0FCA3E0FDA3E0FEA3E09BFFEE9AFEED07
:101E6E0099FDEC98FC90076E127D9B802D9003805F
:101E7E00E0F8A3E0F9A3E0FAA3E0FB900046E0FC53
:101E8E00A3E0FDA3E0FEA3E0C39BFFEE9AFEED9957
:101E9E00FDEC98FC90076E127D9B900786E0FCA3EC
:101EAE00E0FDA3E0FEA3E0FF900380E0F8A3E0F9DD
:101EBE00A3E0FAA3E0FBD3127D4E402E900786E0FE
:101ECE00F8A3E0F9A3E0FAA3E0FB900380E0FCA303
:101EDE00E0FDA3E0FEA3E09BFFEE9AFEED99FDEC84
:101EEE0098FC900772127D9B802D900380E0F8A3E2
:101EFE00E0F9A3E0FAA3E0FB900786E0FCA3E0FD87
:101F0E00A3E0FEA3E0C39BFFEE9AFEED99FDEC98D5
:101F1E00FC900772127D9B9007CDE0FCA3E0FDA321
:101F2E00E0FEA3E0FF900380E0F8A3E0F9A3E0FA5F
:101F3E00A3E0FBD3127D4E402E9007CDE0F8A3E038
:101F4E00F9A3E0FAA3E0FB900380E0FCA3E0FDA37D
:101F5E00E0FEA3E09BFFEE9AFEED99FDEC98FC905F
:101F6E0007D1127D9B802B900380E0F8A3E0F9A3AC
:101F7E00E0FAA3E0FB9007CDE0FCA3E0FDA3E0FEBA
:101F8E00A3E0C39BFFEE9AFEED99FDEC98FCA31225
:101F9E007D9B900044E07002A3E070030220D69077
:101FAE000024E060030220D69001EFE0FFE4FCFD88
:101FBE00FE90076EE0F8A3E0F9A3E0FAA3E0FBD3EE
:101FCE00127D4E40030220CF9002D8E07003022013
:101FDE00CFE47B05FAF9F8900649E0FCA3E0FDA3F7
:101FEE00E0FEA3E0FF127CAEE47B02FAF9F8127C6D
:101FFE002390037CE0F8A3E0F9A3E0FAA3E02FFF1F
:10200E00EA3EFEE93DFDE83CFC900380E0F8A3E0EB
:10201E00F9A3E0FAA3E0FBC3127D6440030220C6DD
:10202E00E47B05FAF9F8900649E0FCA3E0FDA3E095
:10203E00FEA3E0FF127CAEE47B02FAF9F8127C23D9
:10204E00A804A905AA06AB0790037CE0FCA3E0FD5B
:10205E00A3E0FEA3E0C39BFFEE9AFEED99FDEC9884
:10206E00FC900380E0F8A3E0F9A3E0FAA3E0FBD331
:10207E00127D644043900765E0FEA3E0FFD390001D
:10208E001FE09F90001EE09E403EE4F0A3F0900300
:10209E0080E0FCA3E0FDA3E0FEA3E0FF900046126B
:1020AE007D9B900380E0FCA3E0FDA3E0FEA3E0FF98
:1020BE00900786127D9B8010E490001EF0A3F080A6
:1020CE0007E490001EF0A3F090003DE0FFE4FCFD5D
:1020DE00FE900772E0F8A3E0F9A3E0FAA3E0FBC3D9
:1020EE00127D4E400890075FE4F0A304F0C3900702
:1020FE0060E0940790075FE09400503790003DE059
:10210E00FFE4FCFDFE900772E0F8A3E0F9A3E0FA0D
:10211E00A3E0FBC3127D4E500E900760E004F070FA
:10212E000690075FE004F0E4F526F5279002D8F05C
:10213E000221E77526207527009002D87401F090D1
:10214E000380E0FCA3E0FDA3E0FEA3E0FF9007CD3B
:10215E00127D9B900769E060030221E790076BE018
:10216E00FFE4FCFDFE9001F3E0F8A3E0F9A3E0FA32
:10217E00A3E0FBD3127D4E406090000FE0705490B0
:10218E00000EE0B40207D2B412B372C2B49002D7FA
:10219E00E070109001EEE0600A9002C9E0B4010315
:1021AE001237559002D7E070259001EEE0601F9037
:1021BE0002C9E0B40118900467E0B401117F1B124C
:1021CE00E2B07F5012E2B07F0112E2B08005E490DF
:1021DE000467F090000F7401F0900046E0F8A3E061
:1021EE00F9A3E0FAA3E0FB900380E0FCA3E0FDA3DB
:1021FE00E0FEA3E0C39BFFEE9AFEED99FDEC98FC8A
:10220E009002C4127D9BE4FFFEFDFC9002C4E0F838
:10221E00A3E0F9A3E0FAA3E0FBC3127D4E50030244
:10222E0023D59002C4E0FCA3E0FDA3E0FEA3E024CE
:10223E000AFFE43EFEE43DFDE43CFCE47B14FAF9C7
:10224E00F812E4A9900385127D9B900183E0602B28
:10225E00E47F04FEFDFC9002C4E0F8A3E0F9A3E0E5
:10226E00FAA3E0FBD3127D4E500975322075330070
:10227E00022596E4F532F533022596E47F14FEFD31
:10228E00FC900010E0F8A3E0F9A3E0FAA3E0FB1243
:10229E007C23C004C005C006C00790003FE0FEA32B
:1022AE00E0FFE4FCFDF8F9AA06AB07D007D006D094
:1022BE0005D00412E4A99002C4E0F8A3E0F9A3E06B
:1022CE00FAA3E0FBC3127D4E40769002C4E0FCA35D
:1022DE00E0FDA3E0FEA3E0FFC004C005C006C007FA
:1022EE00E47F14FEFDFC900010E0F8A3E0F9A3E0FB
:1022FE00FAA3E0FB127C23C004C005C006C0079001
:10230E00003FE0FEA3E0FFE4FCFDF8F9AA06AB07F0
:10231E00D007D006D005D00412E4A9A804A905AAB6
:10232E0006AB07D007D006D005D004C3EF9BFFEE57
:10233E009AFEED99FDEC98FC9002C4127D9B805C98
:10234E00E47F14FEFDFC900010E0F8A3E0F9A3E09A
:10235E00FAA3E0FB127C23C004C005C006C00790A0
:10236E00003FE0FEA3E0FFE4FCFDF8F9AA06AB0790
:10237E00D007D006D005D00412E4A99002C4E0F82C
:10238E00A3E0F9A3E0FAA3E0FBC3EF9BFFEE9AFEF6
:10239E00ED99FDEC98FC9002C4127D9BE47F04FE47
:1023AE00FDFC9002C4E0F8A3E0F9A3E0FAA3E0FB81
:1023BE00D3127D4E5009753220753300022596E4F6
:1023CE00F532F5330225969002C4E0FCA3E0FDA39E
:1023DE00E0FEA3E024F6FFEE34FFFEED34FFFDEC4D
:1023EE0034FFFCE47B14FAF9F812E4A99003851289
:1023FE007D9B9002C4E0FCA3E0FDA3E0FEA3E0FF02
:10240E0074FFFBFAF9F8127C239002C4127D9B90A4
:10241E000183E0602BE47F04FEFDFC9002C4E0F833
:10242E00A3E0F9A3E0FAA3E0FBD3127D4E500975A9
:10243E003220753300022596E4F532F533022596E7
:10244E00E47F14FEFDFC900010E0F8A3E0F9A3E099
:10245E00FAA3E0FB127C23C004C005C006C007909F
:10246E00003FE0FEA3E0FFE4FCFDF8F9AA06AB078F
:10247E00D007D006D005D00412E4A99002C4E0F82B
:10248E00A3E0F9A3E0FAA3E0FBC3127D4E407690E1
:10249E0002C4E0FCA3E0FDA3E0FEA3E0FFC004C085
:1024AE0005C006C007E47F14FEFDFC900010E0F8A6
:1024BE00A3E0F9A3E0FAA3E0FB127C23C004C0055D
:1024CE00C006C00790003FE0FEA3E0FFE4FCFDF86D
:1024DE00F9AA06AB07D007D006D005D00412E4A99E
:1024EE00A804A905AA06AB07D007D006D005D004CC
:1024FE00C3EF9BFFEE9AFEED99FDEC98FC9002C4A3
:10250E00127D9B805CE47F14FEFDFC900010E0F8D1
:10251E00A3E0F9A3E0FAA3E0FB127C23C004C005FC
:10252E00C006C00790003FE0FEA3E0FFE4FCFDF80C
:10253E00F9AA06AB07D007D006D005D00412E4A93D
:10254E009002C4E0F8A3E0F9A3E0FAA3E0FBC3EF26
:10255E009BFFEE9AFEED99FDEC98FC9002C4127D65
:10256E009BE47F04FEFDFC9002C4E0F8A3E0F9A317
:10257E00E0FAA3E0FBD3127D4E500875322075337E
:10258E00008005E4F532F533E4FFFEFDFC90038593
:10259E00E0F8A3E0F9A3E0FAA3E0FBC3127D4E50EE
:1025AE000890076A7401F08005E490076AF09000C5
:1025BE003FE0FEA3E0FFE4FCFD900385E0F8A3E01E
:1025CE00F9A3E0FAA3E0FB127C23900389127D9B12
:1025DE00900010E0F8A3E0F9A3E0FAA3E0FB90036B
:1025EE0089E0FCA3E0FDA3E0FEA3E0C39BFFEE9A0F
:1025FE00FEED99FDEC98FC9001F3127D9B90076B1C
:10260E00E0FFE4FCFDFE9001F3E0F8A3E0F9A3E0A7
:10261E00FAA3E0FBD3127D4E500AE490000FF09027
:10262E00075904F0E4FFFEFDFC9001F3E0F8A3E08F
:10263E00F9A3E0FAA3E0FBC3127D4E5033D20A9009
:10264E0001F3E0FCA3E0FDA3E0FEA3E0FF74FFFBBB
:10265E00FAF9F8127C239001F3127D9B90076974AE
:10266E0001F0E490000FF090079AE054FDF0800E18
:10267E00C20AE4900769F090079AE04402F09007CE
:10268E006AE0601D900389E0FCA3E0FDA3E0FEA3D9
:10269E00E0FF74FFFBFAF9F8127C23900389127D98
:1026AE009B900183E0602190076AE060089000141F
:1026BE007401F08005E4900014F0E4F52EF52F90EF
:1026CE00079AE04401F08038900769E060089000B6
:1026DE00147401F08005E4900014F0752E20752F0F
:1026EE00009001F3E0FCA3E0FDA3E0FEA3E0FFEC0D
:1026FE004D4E4F700490000FF090079AE054FEF08C
:10270E009002D7E070030229239002D2E0FFC39417
:10271E00024003022923EF14700302288D04600384
:10272E00022923C3900768E0941E900767E0940087
:10273E0050030227EBE4F0A3741FF0E47B1EFAF9BA
:10274E00F8900793E0FCA3E0FDA3E0FEA3E0FF12E8
:10275E00E4A99001F3127D9B90003FE0FEA3E0FF01
:10276E00E4FCFDF8F9AA06AB079001F3E0FCA3E048
:10277E00FDA3E0FEA3E0FF12E4A9AF03900763EA16
:10278E00F0A3EFF09001F3E0FCA3E0FDA3E0FEA3C5
:10279E00E0FFC004C005C006C007900763E0FEA3BB
:1027AE00E0FFE4FCFDAA06AB07D007D006D005D0AB
:1027BE0004C3EF9BFFEE9AFEED9400FDEC9400FC3B
:1027CE009001F3127D9B9001F3E0FCA3E0FDA3E0EA
:1027DE00FEA3E0FF900389127D9B02292390001433
:1027EE00E06028E49002D7F090075404F090086F50
:1027FE00127DA700000000E4900767F0A3F0900799
:10280E0093127DA700000000022923900768E004C0
:10281E00F07006900767E004F0900793E0FCA3E0E9
:10282E00FDA3E0FEA3E0FF9001F3E0F8A3E0F9A31F
:10283E00E0FAA3E0FBEF2BFFEE3AFEED39FDEC38AC
:10284E00FC900793127D9B900767E07004A3E064F1
:10285E000170097BFF7AE1792912E569900767E03B
:10286E00FEA3E0FFC3941EEE940040030229237CD6
:10287E00007D05127B8274502FF876BF02292390BB
:10288E000014E06027E49002D7F090075404F09013
:10289E00086F127DA700000000E4900767F0A3F018
:1028AE00900793127DA700000000806990086FE0EA
:1028BE00FCA3E0FDA3E0FEA3E0FF9001F3E0F8A38C
:1028CE00E0F9A3E0FAA3E0FBD3127D4E4014900191
:1028DE00F3E0FCA3E0FDA3E0FEA3E0FF90086F127F
:1028EE007D9B900776E0FCA3E0FDA3E0FEA3E0FF56
:1028FE00900389E0F8A3E0F9A3E0FAA3E0FBD3127A
:10290E007D4E501190086FE0FCA3E0FDA3E0FEA306
:10291E00E0FF12D903900380E0FCA3E0FDA3E0FEEC
:10292E00A3E0FF900786127D9B900024E06008755F
:10293E0030207531008005E4F530F5319002D7E096
:10294E006008752C20752D008005E4F52CF52D9072
:10295E00003FE0FEA3E0FFE4FCFD900385E0F8A35A
:0B296E00E0F9A3E0FAA3E0FB127C23D9
:10297900900776E0F8A3E0F9A3E0FAA3E0FBC3121D
:102989007D4E5054E4F526F527F528F529F52AF565
:102999002BF52CF52DF52EF52FF530F531F532F512
:1029A900337BFF7AE1793112E5697FC47E0912E749
:1029B900877FA07E0F12E52FD20BE49002D7F0900B
:1029C900086F127DA7000000009007547401F09071
:1029D900079AE04420F08048C20B90079AE054DF40
:1029E900F09002D7E0600FC3900768E0941F90074A
:1029F90067E09400402A900183E06013900389E026
:102A0900FCA3E0FDA3E0FEA3E0FF12D9038011902F
:102A190001F3E0FCA3E0FDA3E0FEA3E0FF12D9036C
:102A29009001EEE06404600E90000EE0B40107D25C
:102A3900B412B372C2B4900392E024FE7003022D63
:102A49008F04600302327190079AE054BFF090FE40
:102A590042F090FEE3E4F07FA07E867D01FC9001C8
:102A6900F3E0F8A3E0F9A3E0FAA3E0FBC3127D4E7B
:102A7900500C9007B5127DA700000000801F7BA0B5
:102A89007A86790178009001F3E0FCA3E0FDA3E0E8
:102A9900FEA3E0FF12E4A99007B5127D9B7BA07A03
:102AA90086790178009001F3E0FCA3E0FDA3E0FE44
:102AB900A3E0FF12E4A9AC00AD01AE02AF03900799
:102AC9009D127D9BE47F107E27FDFC90079DE0F819
:102AD900A3E0F9A3E0FAA3E0FBC3127D64500C90D4
:102AE90007B1127DA700000000801EE47B107A2741
:102AF900F9F890079DE0FCA3E0FDA3E0FEA3E0FF49
:102B0900127CAE9007B1127D9BE47B107A27F9F80D
:102B19009001F3E0FCA3E0FDA3E0FEA3E0FF12E4D3
:102B2900A9AC00AD01AE02AF0390079D127D9BE4F5
:102B39007FE87E03FDFC90079DE0F8A3E0F9A3E0A0
:102B4900FAA3E0FBC3127D64500C9007AD127DA778
:102B590000000000801EE47BE87A03F9F890079DE5
:102B6900E0FCA3E0FDA3E0FEA3E0FF127CAE90072A
:102B7900AD127D9BE47BE87A03F9F89001F3E0FC60
:102B8900A3E0FDA3E0FEA3E0FF12E4A9AC00AD01C0
:102B9900AE02AF0390079D127D9BE47F64FEFDFCAE
:102BA90090079DE0F8A3E0F9A3E0FAA3E0FBC312C4
:102BB9007D64500C9007A9127DA700000000801DBC
:102BC900E47B64FAF9F890079DE0FCA3E0FDA3E03B
:102BD900FEA3E0FF127CAE9007A9127D9BE47B6403
:102BE900FAF9F89001F3E0FCA3E0FDA3E0FEA3E00D
:102BF900FF12E4A9AC00AD01AE02AF0390079D122C
:102C09007D9BE47F0AFEFDFC90079DE0F8A3E0F9B7
:102C1900A3E0FAA3E0FBC3127D64500C9007A51250
:102C29007DA700000000801DE47B0AFAF9F89007EF
:102C39009DE0FCA3E0FDA3E0FEA3E0FF127CAE90C3
:102C490007A5127D9BE47B0AFAF9F89001F3E0FCF1
:102C5900A3E0FDA3E0FEA3E0FF12E4A9AC00AD01EF
:102C6900AE02AF0390079D127D9BE47F01FEFDFC40
:102C790090079DE0F8A3E0F9A3E0FAA3E0FBC312F3
:102C89007D64500C9007A1127DA7000000008012FE
:102C990090079DE0FCA3E0FDA3E0FEA3E0FFA312E3
:102CA9007D9B9007A5E0FCA3E0FDA3E0FEA3E0FF68
:102CB9007804127D88EF54F0FBE49007A1E0FCA3AF
:102CC900E0FDA3E0FEA3E0540FFFE4EB4FFFE49027
:102CD9000797EFF09007ADE0FCA3E0FDA3E0FEA3AA
:102CE900E0FF7804127D88EF54F0FBE49007A9E037
:102CF900FCA3E0FDA3E0FEA3E0540FFFE4EB4FFFCC
:102D0900E4900798EFF09007B5E0FCA3E0FDA3E09D
:102D1900FEA3E0FF7804127D88EF54F0FBE49007EE
:102D2900B1E0FCA3E0FDA3E0FEA3E0540FFFE4EB58
:102D39004FFFE4900799EFF090045FE0700E900761
:102D490097E0F4F0A3E0F4F0A3E0F4F0900797E043
:102D590090FE42F090FEE0E4F0900798E090FE4289
:102D6900F090FEE1E4F0900799E090FE42F090FEC9
:102D7900E2E4F090079AE04440F090FE42F090FEC1
:102D8900E3E4F0023271900723E06016900389E0D2
:102D9900FCA3E0FDA3E0FEA3E0FF9007A1127D9B49
:102DA90080149001F3E0FCA3E0FDA3E0FEA3E0FFA3
:102DB9009007A1127D9B90077EE0FCA3E0FDA3E0B4
:102DC900FEA3E0FF9007A5127D9BE47FFF7EFFFD38
:102DD900FC90017DE0F8A3E0F9A3E0FAA3E0FB127F
:102DE9007C23E47BC07A5DF9F8127CAE9007B912B6
:102DF9007D9BE47FFF7EFFFDFC9001EAE0F8A3E004
:102E0900F9A3E0FAA3E0FB127C23E47BC07A5DF925
:102E1900F8127CAE9007BD127D9B9007B9E0FCA328
:102E2900E0FDA3E0FEA3E0FFA3E0F8A3E0F9A3E03F
:102E3900FAA3E0FBC3127D64500302308F9007B9F7
:102E4900E0F8A3E0F9A3E0FAA3E0FBA3E0FCA3E028
:102E5900FDA3E0FEA3E09BFFEE9AFEED99FDEC9841
:102E6900FCA3127D9B900723E0FF600690076AE0B0
:102E79007031EF6003022F56900014E07025900323
:102E890089E0FCA3E0FDA3E0FEA3E0FF900010E0D1
:102E9900F8A3E0F9A3E0FAA3E0FBC3127D4E5003C7
:102EA900022F569007A1E0FCA3E0FDA3E0FEA3E0FA
:102EB900FF9007C1E0F8A3E0F9A3E0FAA3E0FB1251
:102EC9007C239007A5E0F8A3E0F9A3E0FAA3E0FBCF
:102ED900127CAE9007B9E0F8A3E0F9A3E0FAA3E009
:102EE900FBC3127D64405A9007A1E0FCA3E0FDA357
:102EF900E0FEA3E0FF9007C1E0F8A3E0F9A3E0FA40
:102F0900A3E0FB127C239007A5E0F8A3E0F9A3E076
:102F1900FAA3E0FB127CAEA804A905AA06AB0790A8
:102F290007B9E0FCA3E0FDA3E0FEA3E0C39BFFEE2D
:102F39009AFEED99FDEC98FC9007A9127D9B022F52
:102F4900C99007A9127DA70000000080739007A10E
:102F5900E0FCA3E0FDA3E0FEA3E0FF9007C1E0F8D9
:102F6900A3E0F9A3E0FAA3E0FB127C239007A5E014
:102F7900F8A3E0F9A3E0FAA3E0FB127CAE9007B94D
:102F8900E0F8A3E0F9A3E0FAA3E02FFFEA3EFEE9A7
:102F99003DFDE83CFC9007A9127D9BE47FFF7EFF85
:102FA900FDFC9007A9E0F8A3E0F9A3E0FAA3E0FB90
:102FB900D3127D64400A9007A9127DA70000FFFF84
:102FC9009007B9E0FCA3E0FDA3E0FEA3E0FFA3E0C6
:102FD900F8A3E0F9A3E0FAA3E0FBC3127D64600360
:102FE9000232377FFF7EFFFDFC9007A1E0F8A3E0E6
:102FF900F9A3E0FAA3E0FB127C239007A5E0F8A36C
:10300900E0F9A3E0FAA3E0FB127CAE9007A9127DD8
:103019009B900723E0601290076AE0603E9007A941
:10302900127DA7000000008032900389E0FCA3E034
:10303900FDA3E0FEA3E0FF900010E0F8A3E0F9A3F0
:10304900E0FAA3E0FBC3127D4E500690076AE060E8
:103059000A9007A9127DA700000000E47FFF7EFF08
:10306900FDFC9007A9E0F8A3E0F9A3E0FAA3E0FBCF
:10307900D3127D6450030232379007A9127DA7004D
:1030890000FFFF0232379007B9E0FCA3E0FDA3E09F
:10309900FEA3E0FFA3E0F8A3E0F9A3E0FAA3E0FBB5
:1030A900C3127D6440030232379007BDE0F8A3E004
:1030B900A3E0A3E09007B9E0FCA3E0FDA3E0FEA331
:1030C900E0C39BFFEE9AFEED99FDEC98FC9007C1D9
:1030D900127D9B900723E0FF600690076AE0702E3F
:1030E900EF6003023190900014E07022900389E0B0
:1030F900FCA3E0FDA3E0FEA3E0FF900010E0F8A32D
:10310900E0F9A3E0FAA3E0FBC3127D4E40799007F2
:10311900A1E0FCA3E0FDA3E0FEA3E0FF9007C1E06E
:10312900F8A3E0F9A3E0FAA3E0FB127C239007A53A
:10313900E0F8A3E0F9A3E0FAA3E0FB127CAE900764
:10314900B9E0F8A3E0F9A3E0FAA3E02FFFEA3EFE15
:10315900E93DFDE83CFC9007A9127D9BE47FFF7ED9
:10316900FFFDFC9007A9E0F8A3E0F9A3E0FAA3E0CA
:10317900FBD3127D6450030232379007A9127DA751
:103189000000FFFF0232379007A1E0FCA3E0FDA396
:10319900E0FEA3E0FF9007C1E0F8A3E0F9A3E0FA9D
:1031A900A3E0FB127C239007A5E0F8A3E0F9A3E0D4
:1031B900FAA3E0FB127CAE9007B9E0F8A3E0F9A30B
:1031C900E0FAA3E0FBC3127D6440599007A1E0FC3B
:1031D900A3E0FDA3E0FEA3E0FF9007C1E0F8A3E0B0
:1031E900F9A3E0FAA3E0FB127C239007A5E0F8A37A
:1031F900E0F9A3E0FAA3E0FB127CAEA804A905AAB2
:1032090006AB079007B9E0FCA3E0FDA3E0FEA3E04D
:10321900C39BFFEE9AFEED99FDEC98FC9007A9126D
:103229007D9B800A9007A9127DA700000000E4FB9E
:103239007A01F9F89007A9E0FCA3E0FDA3E0FEA359
:10324900E0FF127CAE900181EFF09007A9E0FCA3AA
:10325900E0FDA3E0FEA3E0FFE4900182EFF0E4903B
:103269000042F0A3F012DDEA900004E06404700368
:1032790002374B90071DE0600302374B90076BE064
:10328900FFE4FCFDFE9001F3E0F8A3E0F9A3E0FA06
:10329900A3E0FBD3127D4E50227F0112E60B900072
:1032A90004E070057F0412E63F900004E0640270B8
:1032B90024900758E0FF12E63F801A900769E06002
:1032C9000F900004E0B40208900758E0FF12E63FAF
:1032D9007F0112E63F9002CEE0FCA3E0FDA3E0FEF1
:1032E900A3E0FF900377E0F8A3E0F9A3E0FAA3E0F5
:1032F9002FFFEA3EFEE93DFDE83CFCE4FBFAF9F864
:10330900C3127D4E400D7F0212E63F7F0312E63F56
:1033190002374B900004E01470030233E414700385
:1033290002353A1470030235B42403600302374BA3
:103339009002CAE0F8A3E0F9A3E0FAA3E0FB900247
:10334900CEE0FCA3E0FDA3E0FEA3E0C39BFFEE9A61
:10335900FEED99FDEC98FC9001F3E0F8A3E0F9A3E8
:10336900E0FAA3E0FBC3127D4E40637F0212E60B35
:10337900900372E0F8A3E0F9A3E0FAA3E0FB90035D
:1033890077E0FCA3E0FDA3E0FEA3E0C39BFFEE9A78
:10339900FEED99FDEC98FC9001F3E0F8A3E0F9A3A8
:1033A900E0FAA3E0FBC3127D4E40167F0312E60B41
:1033B9009002D8E0700302374B7F0412E60B023704
:1033C9004B7F0312E63F7F0412E63F02374B7F0231
:1033D90012E63F7F0312E63F02374B900769E06030
:1033E900169007597401F0C200E4900757F0A3E062
:1033F900FF12E63F02374B900759E0700302374B43
:10340900900757E0602190003BE07002A3E0600361
:1034190002374B900758E0FF12E63FE4900757F058
:10342900900759F002374B30003790003BE07002AB
:10343900A3E0600302374B900758E0FF12E60B90B8
:1034490007577401F0C200900035E0FEA3E0FF7C4D
:10345900007DC8127B7090003BEEF0A3EFF00237BD
:103469004B9002D8E0700302351E90076BE0FFE431
:10347900FCFDFE9001F3E0F8A3E0F9A3E0FAA3E074
:10348900FBD3127D4E500302351E9001F174FFF0FB
:10349900900769E060099007587401F002374B9072
:1034A90002CEE0FCA3E0FDA3E0FEA3E0FF9001F360
:1034B900E0F8A3E0F9A3E0FAA3E0FBC3127D4E50C4
:1034C900089007587402F08030900377E0FCA3E07D
:1034D900FDA3E0FEA3E0FF9001F3E0F8A3E0F9A368
:1034E900E0FAA3E0FBD3127D4E400890075874031D
:1034F900F080069007587404F0D20090002FE0FE87
:10350900A3E0FF7C007DC8127B7090003BEEF0A326
:10351900EFF002374B90002FE0FEA3E0FF7C007D27
:10352900C8127B7090003BEEF0A3EFF0C2000237A7
:103539004B9002CEE0FCA3E0FDA3E0FEA3E0FF90E8
:1035490001F3E0F8A3E0F9A3E0FAA3E0FBC3127DDD
:103559004E50127F0212E60B7F0312E63F7F0412E0
:10356900E63F02374B900377E0FCA3E0FDA3E0FEC2
:10357900A3E0FF9001F3E0F8A3E0F9A3E0FAA3E0E8
:10358900FBD3127D4E40127F0212E63F7F0312E603
:103599000B7F0412E63F02374B7F0212E63F7F039F
:1035A90012E63F7F0412E60B02374B9002CAE0FC99
:1035B900A3E0FDA3E0FEA3E0FF900377E0F8A3E01A
:1035C900F9A3E0FAA3E0FBC3127D4E500302374B87
:1035D9009002CEE0FCA3E0FDA3E0FEA3E0FF900390
:1035E90077E0F8A3E0F9A3E0FAA3E0FBC3127D4E6C
:1035F900500302374B90076BE0FFE4FCFDFE90019E
:10360900F3E0F8A3E0F9A3E0FAA3E0FBD3127D4EBF
:10361900500DE49007DAF07F0412E63F02374B9031
:1036290007D9E0700302372090076BE0FFE4FCFD47
:10363900FE9001F3E0F8A3E0F9A3E0FAA3E0FBD3DD
:10364900127D4E403F9002CAE0F8A3E0F9A3E0FAE8
:10365900A3E0FB9002CEE0FCA3E0FDA3E0FEA3E023
:103669009BFFEE9AFEED99FDEC98FC9001F3E0F8D2
:10367900A3E0F9A3E0FAA3E0FBC3127D4E40057F66
:103689000212E63F900372E0F8A3E0F9A3E0FAA37F
:10369900E0FB900377E0FCA3E0FDA3E0FEA3E0C319
:1036A9009BFFEE9AFEED99FDEC98FC9001F3E0F892
:1036B900A3E0F9A3E0FAA3E0FBC3127D4E40587FD3
:1036C9000312E63F9007DAE0701790002FE0FEA39F
:1036D900E0FF7C007DC8127B7090003BEEF0A3EF09
:1036E900F0D390003CE0940090003BE0940050211E
:1036F9007F0412E60B900035E0FEA3E0FF7C007D1D
:10370900C8127B7090003BEEF0A3EFF0E49007D96C
:10371900F09007DA7401F09007DAE060259007D994
:10372900E0701FD390003CE0940090003BE09400CF
:1037390050107F0412E63FE490003BF0A3F090079D
:0B374900DAF0900753E0700302040068
:013754002252
:10B37200E4F567C26990000EE0B402099002D8E0D9
:10B38200700302B6999002D8E0600F200B0C7F5335
:10B3920012E4ED7F5412E4ED80229002D8E0700FA7
:10B3A200200B0C7F5512E4ED7F5312E4ED800D303B
:10B3B2000B0A7F4F12E4ED7F4C12E4ED7F2C12E476
:10B3C200ED900183E0600C7F4712E4ED7F5312E4BD
:10B3D200ED800A7F4E12E4ED7F5412E4ED7F2C12D1
:10B3E200E4ED7568FF9002D8E060035368BFE4B5EE
:10B3F2002908E528B420035368DFE4B52B08E52AC1
:10B40200B420035368EF9002D7E060035368F790CB
:10B412000183E070035368FB900024E060035368EB
:10B42200FDE4B5330CE532B420075368FED26980DF
:10B4320002C2699002DDE02430FF12E4EDAF68122F
:10B44200E4ED7F2C12E4ED9002D7E060509002D23E
:10B45200E0604A900183E0602E900010E0FCA3E0DF
:10B46200FDA3E0FEA3E0FF90086FE0F8A3E0F9A3DC
:10B47200E0FAA3E02FFFEA3EFEE93DFDE83CFC9046
:10B48200036E127D9B804690086FE0FCA3E0FDA353
:10B49200E0FEA3E0FF90036E127D9B80309001835B
:10B4A200E070169001F3E0FCA3E0FDA3E0FEA3E050
:10B4B200FF90036E127D9B8014900389E0FCA3E051
:10B4C200FDA3E0FEA3E0FF90036E127D9BC20C90F1
:10B4D2000014E060077F2D12E4ED80057F2012E466
:10B4E200EDC201E4FFFEFDFC90036EE0F8A3E0F97B
:10B4F200A3E0FAA3E0FBC3127D4E7002D2019001D9
:10B50200F2E0600302B5C5754C07E54CB401087F53
:10B512002012E4ED02B5B67BA07A8679017800901C
:10B52200036EE0FCA3E0FDA3E0FEA3E0FF12E4A9AA
:10B532008F67E5676002D20C9001F2E02401FFE41C
:10B5420033FED3E54C9FEE6480F874809840192056
:10B552000C16E54CB4020A3001077F3012E4ED808C
:10B562000F7F2012E4ED8008E5672430FF12E4ED3E
:10B5720090036EE0FCA3E0FDA3E0FEA3E0FF7BA04E
:10B582007A867901780012E4A9AC00AD01AE02AF6F
:10B592000390036E127D9B90036EE0FCA3E0FDA37B
:10B5A200E0FEA3E0FFE47B0AFAF9F8127C239003A1
:10B5B2006E127D9B154CE54CD39400400302B50CF2
:10B5C20002B680754C07E54C14FF9001F2E0B50716
:10B5D200057F2E12E4EDE54C14FF9001F2E06F704E
:10B5E2000302B6747BA07A867901780090036EE03C
:10B5F200FCA3E0FDA3E0FEA3E0FF12E4A98F67E550
:10B60200676002D20C9001F2E02402FFE433FED321
:10B61200E54C9FEE6480F8748098400A200C077F06
:10B622002012E4ED8008E5672430FF12E4ED900378
:10B632006EE0FCA3E0FDA3E0FEA3E0FF7BA07A8620
:10B642007901780012E4A9AC00AD01AE02AF03901B
:10B65200036E127D9B90036EE0FCA3E0FDA3E0FE6F
:10B66200A3E0FFE47B0AFAF9F8127C2390036E123E
:10B672007D9B154CE54CD39400400302B5C87F2056
:10B6820012E4ED7F6B12E4ED7F6712E4ED7F0D12A1
:07B69200E4ED7F0A12E4ED74
:01B69900228E
:10DDEA00900043E090FE42F090FEE0E4F0FBE4FE97
:10DDFA0074812BF582E43401F583E0FD30E713905A
:10DE0A000043E04404F0E090FE42F090FEE0E4F0CB
:10DE1A008014E4900042F0A3E054FBF0E090FE424C
:10DE2A00F090FEE0E4F0900043E04402F0E090FE5F
:10DE3A0042F090FEE0E4F0900042F0A3E054FCF0DF
:10DE4A00E090FE42F090FEE0E4F074812BF582E46B
:10DE5A003401F583ED25E0F00EEEB408930BEB6484
:10DE6A0002708B900042E4F0A304F0E090FE42F0CE
:05DE7A0090FEE0E4F061
:01DE7F002280
:08E7C000204348203035200001
:0EE23D0090083FEBF0A3EAF0A3E9F0A3EDF0A8
:10E24B009001EEE0B401197F1C12E2B07F2612E2BE
:10E25B00B07F1C12E2B07F7412E2B07F0112E2B009
:10E26B00E4900843F0900842E0FFA3E0FEC39F5008
:10E27B001F90083FE0FBA3E0FAA3E0F98E827583C1
:10E28B0000127B31FF12E2B0900843E004F080D51E
:10E29B009001EEE0B4010A7F1C12E2B07F2E12E275
:04E2AB00B012E6C502
:01E2AF00224C
:05E2B000900844EFF0AE
:10E2B500E4A3F0A3F074FFA3F0A3F09001EEE060F7
:10E2C5005A24FC7009900844E0FF12E4ED2290FE08
:10E2D50002E030E52D900845E475F001127C0DFE55
:10E2E500D3E5F09420EE944E40E47BFF7AE779C0C5
:10E2F50012E5697FC47E0912E7877FA07E0F12E5CC
:10E305002F22900844E090FE00F0A3741FF07F0ACE
:0BE315007E0012E52F90FE01743FF027
:01E3200022DA
:10E6C5009001EEE024FC600A240270117F0D12E235
:10E6D500B0227F0D12E2B07F0A12E2B0227F0A1249
:03E6E500E2B0227E
:10E3F2009001EEE024FC601C2402702790FE007461
:10E4020011F0A3741FF07F0A7E0012E52F90FE0127
:10E41200743FF0229000417403F012D9D5E49000C9
:10E422000EF02290FE00741BF0A3741FF07F0A7E90
:10E432000012E52F90FE01743FF090FE0004F0A35D
:10E44200741FF07F0A7E0012E52F90FE01743FF0E8
:01E4520022A7
:10D9D5009007E5127DA700002580C2ACE4FFFE7E1E
:10D9E5006490011774FFF0A3DEFC7E007F647598D8
:10D9F5005075C834900041E014601714602024FE6F
:10DA05006028240470309007E5127DA7000004B05B
:10DA1500802E9007E5127DA70000096080229007FF
:10DA2500E5127DA7000012C080169007E5127DA7BC
:10DA350000004B00800A9007E5127DA700002580B5
:10DA4500E47F20FEFDFC9007E5E0F8A3E0F9A3E004
:10DA5500FAA3E0FB127C23A804A905AA06AB077F5D
:10DA6500007E247DF47C00127CAEC3E49FFFE49E1F
:10DA7500F5CB85CBCDEFF5CA85CACCE490038FF005
:0ADA8500900468F0900390F0D2AC1A
:01DA8F002274
:10E4ED00756B01E4F56D8F6AF56CE56A556B60022D
:10E4FD00056DE56B25E0F56B056CE56CB407EB90F0
:10E50D000648E0601514700AE56D30E00D436A8031
:10E51D008008E56D20E003436A808F993099FDC234
:01E52D009954
:01E52E0022CA
:10E777007F4912E4ED7F0D12E4ED7F0A12E4ED22EA
:10C1C400205445535420200054204520532054002B
:10C1D400554E3134303130002031202D20392000AB
:10C1E400205445535420004D4F444520200025320F
:10C1F400642020202532640054455354312000200B
:10C20400484559202000202055464420200054450C
:10C214005354322000205546442020002020202062
:10C224002020200054455354332000414E414C4FAC
:10C2340036005445535434200053455249414C0070
:10C244002D2D2D2D2D2D2D002054455354352000FA
:10C2540054455354352000205052314E540020543C
:10C26400455354362000544553543620002052413F
:10C274004D2020002020436F6D707574657220413D
:10C284006E642053656E736F72202000202043413A
:10C294005320436F72706F726174696F6E20202037
:10C2A400202020002020687474703A2F2F7777772D
:10C2B4002E6361732E636F2E6B7220002020544511
:10C2C4004C2038322D313537372D3535373820204D
:10C2D4002020200020204641582038322D322D3491
:10C2E40037352D343636392020202000202054457F
:10C2F4005354204F4B202020202020202020202079
:10C304002020200020202020202020202020202049
:10C3140020202020202020202020200020364F4FC5
:10C32400442020002E2E2E2E2E2E2E005445535403
:10C334003720002052454C415900494E304F555446
:10C344003000494E2531644F555425316400205442
:10C354004553543820005445535438200042434434
:10C364004F55540020204F4E2020200020204F46BF
:10C37400462020002054455354392000544553543A
:10C384003920002041444F55540020205A45524F33
:10C39400200020204849364820002054455354208A
:01C3A4003167
:10CEE400E4900753F012DB4A7BFF7AC179C412E560
:10CEF400697FA07E0F12E52F7BFF7AC179CC12E502
:10CF0400697FA07E0F12E52F7BFF7AC179C412E5F9
:10CF1400697FA07E0F12E52F125B218F4CE54CF444
:10CF2400700302CFD990017CE54CF0E490003EF010
:10CF340090003EE0600302CFF490017CE024BA60EC
:10CF4400742446B40A00507990CF53F82828730209
:10CF5400CF7102CF8C02CF9102CF9602CF9B02CF2A
:10CF6400A002CFA002CFAA02CFAF02CFB47BFF7A38
:10CF7400C179D412E5697FA07E0F12E52F12E7264E
:10CF840090003E7401F0804212C550803D12C85991
:10CF9400803812BBC3803312DA90802E90017CE07B
:10CFA400FF12D22D802412CC80801F12DE80801AC2
:10CFB40012C6D880159007537401F090003EF0809B
:10CFC4000912E72690003E7401F07F0712000E124A
:10CFD400DB4A02CF347BFF7AC179DC12E5697BFF3F
:10CFE4007AC179E412E59F7BFF7AC179EB12E5D52A
:09CFF400900753E0700302CF1C0A
:01CFFD002211
:10C5500078547C077D017BFF7AC3799E7E007F073C
:10C56000127AF2E490075CF012DB4A7B017A0779D9
:10C570005412E56990FE41E090075DF0540FF0120F
:10C580005B218F4CE54CB4FF0B90075DE0640F70AE
:10C590000302C6BC90075B7463F090075DE024F96A
:10C5A000604024FA601414601E24037041754C0826
:10C5B0007FC47E0912E78702C667754C097FC47E77
:10C5C0000912E78702C6679002C8E0FF7003754C46
:10C5D00007EFB40103754C037FC47E0912E787029D
:10C5E000C667754C017FC47E0912E7878079E54CE8
:10C5F0006401600BE54C64066005E54CB4080890E6
:10C60000075BE54CF08060E54C64046005E54CB4E4
:10C610000909E54C0490075BF0804CE54C6403602D
:10C6200005E54CB40509E54C1490075BF08038E54E
:10C630004C64076005E54CB40B0AE54C24029007F6
:10C640005BF08023E54CB40207E490075BF08017B1
:10C65000E54C700890075B740CF0800BE54CB4302F
:10C660000690075B740EF090084274FFF0A374C14B
:10C67000F0A374F2F0A3E4F0A3E54CF090075BE0C4
:10C68000FF900847E4F0A3EFF07B017A077954129A
:10C69000A77FE54C24BA70187B017A07795412E51C
:10C6A000697FA07E0F12E52F90075C7401F080096E
:10C6B0007B017A07795412E56912DB4A7BFF7AC164
:10C6C00079FC12E59F7BFF7AC2790312E5D59007CA
:07C6D0005CE0700302C57479
:01C6D7002240
:10C85900E4900754F012DB4A7BFF7AC2790A12E5A9
:10C86900697BFF7AC2791212E59F7BFF7AC2791937
:10C8790012E5D5125B218F4CE54CF4700302C99681
:10C88900E54C24BA600302C91AE4900755F09007F1
:10C8990055E0FFC39407502074502FF8E4F6EF25B4
:10C8A900E02426F876200876007FB87E0B12E52F63
:10C8B900900755E004F080D69007557407F090076B
:10C8C90055E0FFC3940D501574502FF8E4F67FB866
:10C8D9007E0B12E52F900755E004F080E190075593
:10C8E900740DF0900755E0FFC39413501574502F41
:10C8F900F8E4F67FB87E0B12E52F900755E004F0B7
:10C9090080E17F587E1B12E52F9007547401F08057
:10C9190079E4900755F0900755E0FFC3940750203C
:10C9290074502FF8E4F6EF25E02426F876200876EF
:10C93900007FB87E0B12E52F900755E004F080D6F2
:10C949009007557407F0900755E0FFC3940D5015F3
:10C9590074502FF8E4F67FB87E0B12E52F90075537
:10C96900E004F080E1900755740DF0900755E0FF61
:10C97900C39413501574502FF8E4F67FB87E0B1248
:10C98900E52F900755E004F080E112DB4A90075447
:10C99900E0700302C87C7BFF7AC2792012E569E462
:10C9A900900755F0900755E0FFC39407500FEF2506
:0DC9B900E02426F8E4F608F6E004F080E73C
:01C9C600224E
:10BBC300E4900758F0A3F0A3F0A3F0A3127DA7001D
:10BBD300000000900760127DA7000000009007643A
:10BBE300127DA70000000012DB4A7BFF7AC279288E
:10BBF30012E59F7BFF7AC2792F12E5D590064FE0BD
:10BC0300FF900754E4F0A3EFF0900116E0FF9007D4
:10BC130056E4F0A3EFF09001167405F012DF117FE4
:10BC2300C87E0012E52FE490075BF09001F0E0245A
:10BC330002FFE433FE90075BE0C39FEE6480F87479
:10BC43008098501F12C9C790075BE025E025E024C8
:10BC530069F582E43404F583127D9B90075BE0046D
:10BC6300F080C8125B218F4CE54CF4700302BD18C1
:10BC7300E54C605B14607124F9603B24FD60212472
:10BC8300C56079243F600302BD0F9001F0E0D394B7
:10BC930009400512E72680779001F0E004F0806FF9
:10BCA3009001F0E0D39401500512E72680619001E2
:10BCB300F0E014F0805990064FE0C394034005125E
:10BCC300E726804B90064FE004F012DF118040908E
:10BCD300064FE0D39400500512E726803290064FBA
:10BCE300E014F012DF11802790075CE0FCA3E0FD75
:10BCF300A3E0FEA3E0FFA3127D9B801390075A7479
:10BD030001F0900755E090064FF0800312E72612EA
:10BD1300DB4A02BDB612CB2E90075C127D9B9007C7
:10BD230060E0FCA3E0FDA3E0FEA3E0FF90075CE07E
:10BD3300F8A3E0F9A3E0FAA3E0FBC3127D4E40337E
:10BD4300E4900014F0900760E0F8A3E0F9A3E0FAB0
:10BD5300A3E0FB90075CE0FCA3E0FDA3E0FEA3E00F
:10BD63009BFFEE9AFEED99FDEC98FC900764127D23
:10BD73009B802F9000147401F090075CE0F8A3E01F
:10BD8300F9A3E0FAA3E0FBA3E0FCA3E0FDA3E0FE3C
:10BD9300A3E0C39BFFEE9AFEED99FDEC98FCA31282
:10BDA3007D9B900764E0FCA3E0FDA3E0FEA3E0FF1E
:10BDB30012D90390075AE0700302BC66900757E05C
:04BDC300900116F0E5
:01BDC7002259
:10DA9000E4900754F0A3F012DB4A7BFF7AC2793698
:10DAA00012E59F7BFF7AC2793D12E5D57FE87E03C0
:10DAB00012E52F12D9D5E4FF7F0B900117E4F0A3F4
:10DAC000DFFC7F0B7BFF7AC2794412E569D2AC128E
:10DAD0005B218F4CE54CF46036E54C24BA7008901D
:10DAE00007547401F08023D2B4E54C2430FF12E4D3
:10DAF000EDC2B4E54C75F00A84E5F090D7ED93F5EE
:10DB000056E54C75F00A8493F55512DB4A80329045
:10DB10000117E0F54CE54C6028E4900390F07FC4D9
:10DB20007E0912E787E54C75F00A84E5F090D7EDA1
:10DB300093F551E54C75F00A8493F550E490011784
:09DB4000F0900754E06088C2ACCB
:01DB490022B9
:05D22D00900754EFF032
:10D23200E4A3F0A3F012DB4A900754E0B4051D7B8F
:10D24200FF7AC2794C12E5697BFF7AC2795412E502
:10D252009F7BFF7AC2795B12E5D5801B7BFF7AC286
:10D26200796212E5697BFF7AC2796A12E59F7BFFD8
:10D272007AC2797112E5D5125B218F4CE54CF470BC
:10D282000302D336E54C24BA70099007557401F0B5
:10D2920002D336900754E06405706912E3F212E695
:10D2A200C57BFF7AC279787D1712E23D7BFF7AC295
:10D2B20079907D1712E23D7BFF7AC279A87D171221
:10D2C200E23D7BFF7AC279C07D1712E23D7BFF7A95
:10D2D200C279D87D1712E23D7BFF7AC279F07D17C1
:10D2E20012E23D7BFF7AC379087D1712E23D7BFF94
:10D2F2007AC379087D1712E23D7BFF7AC379201247
:10D30200E5698030E4900756F07BFF7AC3792812F2
:10D31200D3407BFF7AC2796A12E59F7BFF7AC2799A
:10D322007112E5D57BFF7AC3792012E5697F887E89
:0DD332001312E52F900755E0700302D27929
:01D33F0022CB
:10CC8000E4900754F0A3F0A3F012DB4A7BFF7AC3D1
:10CC9000793012E59F7BFF7AC3793712E5D57BFFA8
:10CCA0007AC3793E12E56990FE41E0900757F0544F
:10CCB0000FF0640F604AE024F9603824FA6016141B
:10CCC00060222403703A9007567402F07FC47E09F4
:10CCD00012E787802B9007567403F07FC47E0912F9
:10CCE000E787801C9007567404F07FC47E0912E722
:10CCF00087800D9007567401F07FC47E0912E78784
:10CD0000125B218F4CE54CF46069E54C1424FC5017
:10CD10000F603B14603F24FB604324C56047804D97
:10CD2000900755E54CF090FE40740FF0C3740595E4
:10CD30004C900757F014FF7401A807088002C33312
:10CD4000D8FC900757F0F4F090FE40F0802290FE5F
:10CD500040E4F0801B90FE4074FFF0801390075475
:10CD60007401F0800B9007547401F0800312E726E1
:10CD700012DB4A900754E0703A90084274FFF0A327
:10CD800074C3F0A37446F0900756E0FF900845E4A2
:10CD9000F0A3EFF0900755E0FF900847E4F0A3EF11
:10CDA000F07B017A07795812A77F7B017A077958BF
:10CDB00012E569900754E0700302CCA790FE40741E
:06CDC000FFF09001F1F00C
:01CDC600224A
:10DE8000E4900754F0A3F012DB4A7BFF7AC3795287
:10DE900012E5697BFF7AC3795A12E59F7BFF7AC34B
:10DEA000796112E5D5125B218F4CE54CF4605BE59E
:10DEB0004C24BA6047243B704B900754E020E01A92
:10DEC0007BFF7AC3796812E56990FE42E4F090FE28
:10DED000E0F0A3F0A3F0A3F0801A7BFF7AC379707F
:10DEE00012E56990FE4274FFF090FEE0E4F0A3F0CA
:10DEF000A3F0A3F0900754E004F0800B9007557452
:10DF000001F0800312E72612DB4A900755E0609586
:01DF100022EE
:10C6D800E4900754F0A3F0A3127DA7000000009097
:10C6E800075A127DA7000000007F007E007D007CB5
:10C6F8000012DB4A7BFF7AC3797812E5697BFF7AFF
:10C70800C3798012E59F7BFF7AC3798712E5D5E468
:10C718007FFF7EFFFDFC90017DE0F8A3E0F9A3E038
:10C72800FAA3E0FB127C23E47BC07A5DF9F8127C63
:10C73800AE900756127D9BE47FFF7EFFFDFC9001C3
:10C74800EAE0F8A3E0F9A3E0FAA3E0FB127C23E413
:10C758007BC07A5DF9F8127CAE90075A127D9B90E7
:10C768000756E0F8A3E0F9A3E0FAA3E0FBA3E0FC96
:10C77800A3E0FDA3E0FEA3E0C39BFFEE9AFEED99C4
:10C78800FDEC98FC4D4E4F70067FFF7EFFFDFC12BE
:10C798005B218F4CE54CF4700302C84FE54C24BA7A
:10C7A800700302C841243B600302C849900754E063
:10C7B80070447BFF7AC3798E12E569E4FB7A01F94C
:10C7C800F8900756E0FCA3E0FDA3E0FEA3E0FF120B
:10C7D8007CAE900181EFF0900756E0FCA3E0FDA34A
:10C7E800E0FEA3E0FFE4900182EFF012DDEA90079B
:10C7F800547401F0804E7BFF7AC3799612E569E4A0
:10C80800FB7A01F9F890075AE0FCA3E0FDA3E0FEEB
:10C81800A3E0FF127CAE900181EFF090075AE0FC94
:10C82800A3E0FDA3E0FEA3E0FFE4900182EFF01295
:10C83800DDEAE4900754F0800B9007557401F0800E
:10C848000312E72612DB4A900755E0700302C797E8
:01C8580022BD
:10BFC9003031202D20343900202053455420004D94
:10BFD9004F4445202000205245545259200020202A
:10BFE90020202020200020204630312000444154C8
:10BFF900452020002020463032200054494D45205C
:10C00900200020204630332000535045454420006D
:10C019002020463034200046494C54455200202007
:10C029004630352000535441424C450020204630CB
:10C03900362000413245524F20002020463037201B
:10C0490000424143485550002020463038200048DE
:10C059004F4C442020002020463039200052414EC8
:10C06900394520002020463130200032542D43200C
:10C079002000202046313120004C2D5459504500D4
:10C0890020204631322000382D394B4559002020D7
:10C0990046323020004241554420200020204632BB
:10C0A9003120005041524954590020204632322053
:10C0B9000053454E442020002020463233200044BE
:10C0C9004555494345002020463330200050524908
:10C0D9004E54200020204633312000464F524D2037
:10C0E900200020204633322000415052494E54004E
:10C0F900204633332049004E495449414C00202001
:10C109004633342000415343494920002020463317
:10C11900352000464545442020002046333620413D
:10C129000055544F435554002020463430200052C6
:10C13900454C415920002020463431200044454CCB
:10C14900415931002020463432200044454C4159A0
:10C159003200202046343320003252454C415900E8
:10C169002020463434200053454C454354002020B8
:10C1790046343520004F5054494F4E002020463454
:10C189003620005A45524F202000202046343720BF
:10C199000048493948202000202046343820002012
:10C1A9004E2D39202000202046343920004C4F36AE
:0BC1B900494320005020202D202020B2
:104B9100E4900753F0900757F0A3F0A3F0A3F0A31C
:104BA100F0A3F0A3F0A3F0A3F0A3F0A3F0A3F0A36C
:104BB100F0A3F0A3F0A3F0A3F0A3F0A3F0A3F0A35C
:104BC100F0A3F0A3F0A3F0A3F0A3F0A3F0A3F0A34C
:104BD100F0A3F0A3F0A3F0A3F090077AF0A3F09074
:104BE100077EF0A3F0A304F0A3127DA7000000004C
:104BF100900785127DA70000000012DB4A90078014
:104C0100E060097BFF7ABF79C912E5697BFF7ABF52
:104C110079D112E59F7BFF7ABF79D812E5D590074C
:104C21007FE0605DE47FE87E03FDFC900781E0F8B2
:104C3100A3E0F9A3E0FAA3E0FBC3127D6450219045
:104C41000781E0FCA3E0FDA3E0FEA3E02401FFE473
:104C51003EFEE43DFDE43CFC900781127D9B8021FA
:104C61007BFF7ABF79DF12E56912E726900780742E
:104C710001F0E490077FF0900781127DA70000000A
:104C810000125B218F4CE54CF47003025701E49054
:104C91000780F090017CE54CF0C3940A504B9007DB
:104CA1007FE0602490077EE075F00AA4254C900116
:104CB1007CF0E490003EF0E54C90D7ED93F5567F03
:104CC100A07E0F12E52F803390077EE54CF0A37490
:104CD10001F090003EF07BFF7ABF79E712E569E5CC
:104CE1004C90D7ED93F5558012E54CB40B0312E7C8
:104CF10026E54CB44605E490003EF090071DE060C7
:104D01001990017CE0FFC394284006EFD3942B4017
:104D110004EFB40C05E490017CF090003EE06003E8
:104D21000256FE90017CE0127DF84D95014DAF02D7
:104D31004DC9034E30044E86054ED5064F3F074FF1
:104D41007A084FBA094FFA0A50350B50780C50B80F
:104D51001450F81551381651781751B81E51F81FD3
:104D6100523820528B2152BF2252DD235333245318
:104D7100732853B32954012A544F2B548F2C54CFE9
:104D81002D550F2E55AF2F564F30568B3156C746E6
:104D9100000056D47BFF7ABF79EF12E59F7BFF7A43
:104DA100BF79F612E5D5E4FF12B69A0256EA7BFF07
:104DB1007ABF79FD12E59F7BFF7AC0790412E5D5B0
:104DC1007F0112B69A0256EA7BFF7AC0790B12E58F
:104DD1009F7BFF7AC0791212E5D5900025E0FF9004
:104DE1000755F0E4FCFDFE9007E97410F0127E1EF9
:104DF100900025EFF0C3940A5003740AF090002547
:104E0100E0D3943240037432F0900025E0FF900724
:104E110055E06F600690076D7401F07F327E0012DD
:104E2100E52F12DF117F647E0012E52F0256EA7B27
:104E3100FF7AC0791912E59F7BFF7AC0792012E5CC
:104E4100D59001F0E0FFFD900778E4F0A3EDF0E4E8
:104E5100FCFDFE9007E9740EF0127E1E9001F0EF4A
:104E6100F0C3940150037401F09001F0E0FF90074A
:104E710078E07003A3E06F70030256EA900758745C
:104E810001F00256EA7BFF7AC0792712E59F7BFF8A
:104E91007AC0792E12E5D590000AE0FEA3E0FF90DA
:104EA1000778EEF0A3EFF0E4FCFD9007E9740FF052
:104EB100127E1E7E0090000AEEF0A3EFF0900778BC
:104EC100E07003A3E06F70030256EA900759740182
:104ED100F00256EA7BFF7AC0793512E59F7BFF7AB3
:104EE100C0793C12E5D5900045E075F00AA4FF9029
:104EF1000027E02FFF900754F0A3F0E4FCFDFE90A3
:104F010007E97410F0127E1E900754EFF0A3E06FD2
:104F1100600890075A7401F0A3F0900754E0FF7500
:104F2100F00A84FD900044E4F0A3EDF0EF75F00A7F
:104F310084AFF0900026E4F0A3EFF00256EA7BFF85
:104F41007AC0794312E59F7BFF7AC0794A12E5D591
:104F510090064EE0900755F07B017A06794E12E3F8
:104F61002190064EE0FF900755E06F70030256EA6C
:104F710090075C7401F00256EA7BFF7AC079511206
:104F8100E59F7BFF7AC0795812E5D59002D2E0FF08
:104F9100900755F0E4FCFDFE9007E97414F0127ED1
:104FA1001E9002D2EFF0900755E06F70030256EAAF
:104FB1009007647401F00256EA7BFF7AC0795F12B0
:104FC100E59F7BFF7AC0796612E5D5900466E0FF24
:104FD100900755F0E4FCFDFE9007E97415F0127E90
:104FE1001E900466EFF0900755E06F70030256EAD9
:104FF1009007767401F00256EA7BFF7AC0796D1250
:10500100E59F7BFF7AC0797412E5D5900018E09096
:105011000755F07B017A00791812E321900018E01E
:10502100FF900755E06F70030256EA900762740122
:10503100F00256EA7BFF7AC0797B12E59F7BFF7A0B
:10504100C0798212E5D5900722E0FF900755F0E480
:10505100FCFDFE9007E97414F0127E1E900722EF0A
:10506100F0900755E06F70030256EA90076E7401E5
:10507100F012DF110256EA7BFF7AC0798912E59FAF
:105081007BFF7AC0799012E5D5900391E0FF9007FC
:1050910055F0E4FCFDFE9007E97414F0127E1E90B9
:1050A1000391EFF0900755E06F70030256EA900705
:1050B100757401F00256EA7BFF7AC0799712E59F79
:1050C1007BFF7AC0799E12E5D5900041E0FF900701
:1050D10055F0E4FCFDFE9007E97413F0127E1E907A
:1050E1000041EFF0900755E06F70030256EA900718
:1050F1005E7401F00256EA7BFF7AC079A512E59F42
:105101007BFF7AC079AC12E5D5900648E0FF9007A5
:1051110055F0E4FCFDFE9007E9740BF0127E1E9041
:105121000648EFF0900755E06F70030256EA9007CA
:105131006F7401F00256EA7BFF7AC079B312E59FE2
:105141007BFF7AC079BA12E5D590000EE0FF900797
:1051510055F0E4FCFDFE9007E97418F0127E1E90F4
:10516100000EEFF0900755E06F70030256EA9007CA
:10517100617401F00256EA7BFF7AC079C112E59FA2
:105181007BFF7AC079C812E5D59002DDE0FF900778
:1051910055F0E4FCFDFE9007E97422F0127E1E90AA
:1051A10002DDEFF0900755E06F70030256EA9007B9
:1051B100637401F00256EA7BFF7AC079CF12E59F52
:1051C1007BFF7AC079D612E5D59001EEE0FF90071A
:1051D10055F0E4FCFDFE9007E97412F0127E1E907A
:1051E10001EEEFF0900755E06F70030256EA900769
:1051F1005D7401F00256EA7BFF7AC079DD12E59F0A
:105201007BFF7AC079E412E5D5900384E0FF900733
:1052110055F0E4FCFDFE9007E97416F0127E1E9035
:105221000384EFF0900755E06F70030256EA900790
:10523100607401F00256EA7BFF7AC079EB12E59FB8
:105241007BFF7AC079F212E5D59002C9E0FF9007A1
:1052510055F0E4FCFDFE9007E9740DF0127E1EECA2
:105261004D4E4F60089002C97401F08005E4900230
:10527100C9F09002C9E0FF900755E06F7003025634
:10528100EA9007577401F00256EA7BFF7AC079F978
:1052910012E59F7BFF7AC1790012E5D5E4900756AC
:1052A100F07B017A07795612E321900756E07003EB
:1052B1000256EA900464E4F0A304F00256EA7BFF8C
:1052C1007AC1790712E59F7BFF7AC1790E12E5D584
:1052D10012C3A59007777401F00256EA7BFF7AC1E9
:1052E100791512E59F7BFF7AC1791C12E5D59006ED
:1052F1004DE0FFFD900778E4F0A3EDF0E4FCFDFE46
:105301009007E9740EF0127E1E90064DEFF0C394E3
:105311000150037401F090064DE0FF900778E070B2
:1053210003A3E06F70030256EA90076B7401F00269
:1053310056EA7BFF7AC1792312E59F7BFF7AC17917
:105341002A12E5D5900467E0FF900755F0E4FCFDD3
:10535100FE9007E9741AF0127E1E900467EFF09038
:105361000755E06F70030256EA90076C7401F00272
:1053710056EA7BFF7AC1793112E59F7BFF7AC179C9
:105381003812E5D5900004E0FF900755F0E4FCFDEC
:10539100FE9007E9741EF0127E1E900004EFF0905B
:1053A1000755E06F70030256EA9007677401F00237
:1053B10056EA7BFF7AC1793F12E59F7BFF7AC1797B
:1053C1004612E5D5900030E0900755F090002FE0AF
:1053D100FEA3E0FFE4FCFD9007E9741FF0127E1EBE
:1053E1007E0090002FEEF0A3EFF0900755E06F7074
:1053F10001E470030256EA9007707401F00256EA64
:105401007BFF7AC1794D12E59F7BFF7AC1795412F6
:10541100E5D5900036E0900755F0900035E0FEA309
:10542100E0FFE4FCFD9007E9741FF0127E1E7E0090
:10543100900035EEF0A3EFF0900755E06F7001E4B6
:1054410070030256EA9007717401F00256EA7BFF7D
:105451007AC1795B12E59F7BFF7AC1796212E5D54A
:10546100900017E0FF900755F0E4FCFDFE9007E97E
:105471007435F0127E1E900017EFF0900755E06F23
:0854810070030256EA9007686F
:105489007401F00256EA7BFF7AC1796912E59F7BC4
:10549900FF7AC1797012E5D59002C8E0FF900755EF
:1054A900F0E4FCFDFE9007E97436F0127E1E9002CE
:1054B900C8EFF0900755E06F70030256EA90076550
:1054C9007401F00256EA7BFF7AC1797712E59F7B76
:1054D900FF7AC1797E12E5D5900392E0FF900755D6
:1054E900F0E4FCFDFE9007E97423F0127E1E9003A0
:1054F90092EFF0900755E06F70030256EA90076942
:105509007401F00256EA7BFF7AC1798512E59F7B27
:10551900FF7AC1798C12E5D590017DE0FCA3E0FD0D
:10552900A3E0FEA3E0FF900785127D9B90017DE03B
:10553900FCA3E0FDA3E0FEA3E0FF9007E97409F0F6
:10554900127E1E90017D127D9BE47FC07E5DFDFC75
:1055590090017DE0F8A3E0F9A3E0FAA3E0FBD31200
:105569007D644014900785E0FCA3E0FDA3E0FEA361
:10557900E0FF90017D127D9B90017DE0FCA3E0FDA1
:10558900A3E0FEA3E0FF900785E0F8A3E0F9A3E01C
:10559900FAA3E0FBC3127D6470030256EA90077216
:1055A9007401F00256EA7BFF7AC1799312E59F7B79
:1055B900FF7AC1799A12E5D59001EAE0FCA3E0FDF2
:1055C900A3E0FEA3E0FF900785127D9B9001EAE02E
:1055D900FCA3E0FDA3E0FEA3E0FF9007E97409F056
:1055E900127E1E9001EA127D9BE47FC07E5DFDFC68
:1055F9009001EAE0F8A3E0F9A3E0FAA3E0FBD312F3
:105609007D644014900785E0FCA3E0FDA3E0FEA3C0
:10561900E0FF9001EA127D9B9001EAE0FCA3E0FD26
:10562900A3E0FEA3E0FF900785E0F8A3E0F9A3E07B
:10563900FAA3E0FBC3127D6470030256EA90077374
:105649007401F00256EA7BFF7AC179A112E59F7BCA
:10565900FF7AC179A812E5D5900723E0FF90075595
:10566900F0E4FCFDFE9007E97424F0127E1E900719
:1056790023EFF0900755E06F60679007747401F0AD
:10568900805F7BFF7AC179AF12E59F7BFF7AC17991
:10569900B612E5D590045FE0FF900755F0E4FCFDF4
:1056A900FE9007E97424F0127E1E90045FEFF090DB
:1056B9000755E06F602B90076A7401F0802390070B
:1056C900537401F0E490017BF080167BFF7ABF7977
:1056D900DF12E56990003E7401F0900780F012E74F
:1056E9002690003E7401F0900780F0E490077EF068
:1056F900A3F0024D1B12DB4A900753E07003024BE3
:10570900FE7BFF7ABF79E712E569900757E06018D9
:105719009002C9E0FFE4FCFDFE900842127D9B7DEA
:10572900637C007F0112B98690075FE060189003DF
:105739008DE0FFE4FCFDFE900842127D9B7D647CB8
:10574900007F0112B986900758E060189001F0E0D7
:10575900FFE4FCFDFE900842127D9B7D627C007F88
:105769000112B986900759E0601A90000AE0FEA379
:10577900E0FFE4FCFD900842127D9B7D617C007F87
:105789000112B98690075AE0601A900044E0FEA31E
:10579900E0FFE4FCFD900842127D9B7D607C007F68
:1057A9000112B98690075BE0601A900026E0FEA31B
:1057B900E0FFE4FCFD900842127D9B7D5F7C007F49
:1057C9000112B98690075CE0601890064EE0FFE48C
:1057D900FCFDFE900842127D9B7D5D7C007F0112DD
:1057E900B98690075DE060189001EEE0FFE4FCFDEA
:1057F900FE900842127D9B7D5C7C007F0112B98678
:1058090090075EE06018900041E0FFE4FCFDFE9027
:105819000842127D9B7D5B7C007F0112B98690074F
:1058290064E060189002D2E0FFE4FCFDFE900842BB
:10583900127D9B7D5A7C007F0112B986900760E03A
:105849006018900384E0FFE4FCFDFE900842127D9D
:105859009B7D597C007F0112B986900761E0601831
:1058690090000EE0FFE4FCFDFE900842127D9B7D56
:10587900587C007F0112B986900762E06018900099
:1058890018E0FFE4FCFDFE900842127D9B7D577CE9
:10589900007F0112B986900763E060189002DDE08D
:1058A900FFE4FCFDFE900842127D9B7D567C007F43
:1058B9000112B986900767E06018900004E0FFE4E0
:1058C900FCFDFE900842127D9B7D557C007F0112F4
:1058D900B986900768E06018900017E0FFE4FCFDC6
:1058E900FE900842127D9B7D537C007F0112B98690
:1058F900900769E06018900392E0FFE4FCFDFE90D8
:105909000842127D9B7D527C007F0112B986900767
:1059190065E060189002C8E0FFE4FCFDFE900842D3
:10592900127D9B7D517C007F0112B98690076AE048
:10593900601890045FE0FFE4FCFDFE900842127DD0
:105949009B7D507C007F0112B98690076BE060183F
:1059590090064DE0FFE4FCFDFE900842127D9B7D20
:105969006A7C007F0112B98690076CE06018900488
:1059790067E0FFE4FCFDFE900842127D9B7D727C8E
:10598900007F0112B98690076DE06018900025E04C
:10599900FFE4FCFDFE900842127D9B7D6B7C007F3D
:1059A9000112B98690076EE06018900722E0FFE4C3
:1059B900FCFDFE900842127D9B7D6C7C007F0112EC
:1059C900B986900775E06018900391E0FFE4FCFD4B
:1059D900FE900842127D9B7D707C007F0112B98682
:1059E90090076FE06018900648E0FFE4FCFDFE9028
:1059F9000842127D9B7D6D7C007F0112B98690075C
:105A090070E0601A90002FE0FEA3E0FFE4FCFD9037
:105A19000842127D9B7D6E7C007F0112B98690073A
:105A290071E0601A900035E0FEA3E0FFE4FCFD9010
:105A39000842127D9B7D547C007F0112B986900734
:105A490072E0601D90017DE0FCA3E0FDA3E0FEA3F0
:105A5900E0FF900842127D9B7D1C7C007F0412B9F7
:105A690086900773E0601D9001EAE0FCA3E0FDA3C6
:105A7900E0FEA3E0FF900842127D9B7D207C007F21
:105A89000412B986900774E06018900723E0FFE4D8
:105A9900FCFDFE900842127D9B7D6F7C007F011208
:105AA900B986900776E06018900466E0FFE4FCFD93
:105AB900FE900842127D9B7D687C007F0112B986A9
:105AC900900777E06051E490077CF0A3F090077CA1
:105AD900E0FEA3E0FFC39448EE9400503AEF247827
:105AE900FDE43EFCC004C005E02431F582E4340540
:105AF900F583E0FFE4FCFDFE900842127D9BD00592
:105B0900D0047F0112B98690077DE004F0700690F9
:075B1900077CE004F080B6F8
:015B20002262
:0BE32100900789EBF0A3EAF0A3E9F0FD
:10E32C00E4A3F0125B218F4CE54CF4602CE54C24FB
:10E33C00BA700890078C7401F0801B900789E0FB81
:10E34C00A3E0FAA3E0F9127B186006E4127B5E806E
:10E35C00057401127B5E12DB4A900789E0FBA3E097
:10E36C00FAA3E0F9127B18600B7556AB7555A375C3
:10E37C0054FF800975568E75558E7554A390078C75
:03E38C00E060A0AE
:01E38F00226B
:10C3A500E4900789F0A37402F0E4A3F0A3F0789079
:10C3B5007C077D017BFF7AC179BDFE7F07127AF28A
:10C3C500E4900797F0A3F090078BE02431F582E421
:10C3D5003405F583E090078CF0125B218F4CE54C1A
:10C3E500F4700302C493E54C24F6500D14606124E7
:10C3F500C5700302C48202C48A90078AE0248DF5C1
:10C4050082E43407F583E54CF090078EE075F00A79
:10C41500A4FFA3E075F064A42FFF90078DE02F9093
:10C42500078CF0D394FF401212E726E490078AF0B8
:10C4350090078CF0A3F0A3F0A3F090078AE0D394C3
:10C44500004005E014F0804090078A7402F08038BF
:10C4550090078BE0C394475005E004F08005E49015
:10C46500078BF090078BE02431F582E43405F583E2
:10C47500E090078CF090078A7402F0800B90078992
:10C485007401F0800312E72612DB4A02C5469007C5
:10C495008CE0FF90078BE0FB2431F582E43405F551
:10C4A50083EFF0EF75F0648490078FF0EF75F0641B
:10C4B50084AFF0EF75F00A8490078EF0EF75F00AFF
:10C4C50084AFF090078DEFF0FDEB75F00A84243012
:10C4D500900791F0EB75F00A84E5F02430A3F09015
:10C4E500078FE02430900794F090078EE024309079
:10C4F5000795F0ED2430A3F0A3E475F001127C0D4F
:10C50500FED3E5F09414EE9400402D90078AE0FFE9
:10C5150074069FFFE49400FE74902FF58274073E25
:10C52500F5837420F0D3900798E09428900797E05E
:10C5350094004004E4F0A3F07B017A07799012E5BA
:0AC5450069900789E0700302C3DE6D
:01C54F0022C9
:10A215002D2D2D2D2D2D2D2D2D2D2D2D2D2D2D2D69
:10A225002D2D2D2D2D00202020202053554220207E
:10A2350020544F54414C20202020200020444154DC
:10A245004520203A203230253032782E20253278AC
:10A255002E2025327800204441544520203A2031D3
:10A2650039253032782E202532782E202532780077
:10A275002054494D4520203A20202020202020250B
:10A285003032783A25303278002049442020202089
:10A295003A2020202020253464202020200020433F
:10A2A5004F554E54203A202020202025346420206C
:10A2B50020200020544F54414C203A202025366C54
:10A2C500642E2530316C64206B670020544F544157
:10A2D5004C203A202025356C642E2530326C6420C4
:10A2E5006B670020544F54414C203A202025346C94
:10A2F500642E2530336C64206B670020544F544125
:10A305004C203A202025386C64206B670020532DA3
:10A31500544F54414C203A25366C642E2530316C0F
:10A3250064206B670020532D544F54414C203A252F
:10A33500356C642E2530326C64206B670020532DFC
:10A34500544F54414C203A25346C642E2530336CDF
:10A3550064206B670020532D544F54414C203A25FF
:10A36500386C64206B67002020204F564552414CC5
:10A375004C202D20544F54414C20202000323025B4
:10A385003032782E202532782E2025327820202054
:10A39500253032783A253032780031392530327817
:10A3A5002E202532782E2025327820202025303287
:10A3B500783A2530327800253033642C2049445FC3
:10A3C500253032642C25346C642E2530316C6420A4
:10A3D5006B6700253033642C2049445F2530326497
:10A3E5002C25336C642E2530326C64206B67002578
:10A3F5003033642C2049445F253032642C25326C7F
:10A40500642E2530336C64206B6700253033642C53
:10A415002049445F253032642C25366C64206B67F7
:10A42500004E6F2E253033642020202025366C64A5
:10A435002E2530316C64206B67004E6F2E2530332E
:10A44500642020202025356C642E2530326C642054
:10A455006B67004E6F2E2530336420202020253475
:10A465006C642E2530336C64206B67004E6F2E258F
:10A475003033642020202025386C64206B6700472A
:10A48500726F7373203A20202025366C642E253098
:10A49500316C64206B670047726F7373203A20201C
:10A4A5002025356C642E2530326C64206B6700479F
:10A4B500726F7373203A20202025346C642E25306A
:10A4C500336C64206B670047726F7373203A2020EA
:10A4D5002025386C64206B67005461726520203A32
:10A4E50020202025366C642E2530316C64206B6766
:10A4F500005461726520203A20202025356C642E99
:10A505002530326C64206B67005461726520203AF7
:10A5150020202025346C642E2530336C64206B6735
:10A52500005461726520203A20202025386C642073
:10A535006B67004E65742020203A20202025366C5C
:10A54500642E2530316C64206B67004E65742020C5
:10A55500203A20202025356C642E2530326C64206D
:10A565006B67004E65742020203A20202025346C2E
:10A57500642E2530336C64206B67004E6574202093
:10A58500203A20202025386C64206B670025303266
:10A59500783A253032782C204E65743A25356C642E
:10A5A5002E2530316C64206B6700253032783A25D2
:10A5B5003032782C204E65743A25346C642E253063
:10A5C500326C64206B6700253032783A253032785A
:10A5D5002C204E65743A25336C642E2530336C641B
:10A5E500206B6700253032783A253032782C204EA2
:10A5F50065743A25376C64206B670049445F2530E4
:10A6050032642C4E65743A25366C642E2530316CD7
:10A6150064206B670049445F253032642C4E6574B5
:10A625003A25356C642E2530326C64206B67004901
:10A63500445F253032642C4E65743A25346C642EA3
:10A645002530336C64206B670049445F25303264E4
:10A655002C4E65743A25386C64206B6700253033C1
:10A66500642C20202020202025366C642E253031B6
:10A675006C64206B6700253033642C20202020205B
:10A685002025356C642E2530326C64206B670025DF
:10A695003033642C20202020202025346C642E2586
:10A6A50030336C64206B6700253033642C20202008
:10A6B50020202025386C64206B6700202020202076
:10A6C500202020202025366C642E2530316C642016
:10A6D5006B67002020202020202020202025356C9D
:10A6E500642E2530326C64206B67002020202020EA
:10A6F500202020202025346C642E2530336C6420E6
:10A705006B67002020202020202020202025386C69
:05A7150064206B6700E9
:10683E0012E13990071CE07003026F82900384E02E
:10684E0064067003026C7212E6C57BFF7AA279159C
:10685E007D1512E23D7BFF7AA2792B7D1512E23D6A
:10686E007BFF7AA279157D1512E23D900019E0FFAB
:10687E00C3945A503990084274FFF0A374A2F0A347
:10688E007441F0A3E4F0A3EFF0900005E0FF900850
:10689E0047E4F0A3EFF0900028E0FF900849E4F001
:1068AE00A3EFF07B017A0779E512A77F803E90086F
:1068BE004274FFF0A374A2F0A3745BF0900019E091
:1068CE00FF900845E4F0A3EFF0900005E0FF90087C
:1068DE0047E4F0A3EFF0900028E0FF900849E4F0C1
:1068EE00A3EFF07B017A0779E512A77F9008427437
:1068FE00FFF0A374A2F0A37475F0900029E0FF904E
:10690E000845E4F0A3EFF0900579E0FF900847E426
:10691E00F0A3EFF07B017A0779FB12A77F7B017A58
:10692E000779E57D1512E23D7B017A0779FB7D152E
:10693E0012E23D90084274FFF0A374A2F0A3748E8D
:10694E00F0900646E0FFA3E0900845CFF0A3EFF0ED
:10695E007B017A0779E512A77F7B017A0779E57DBE
:10696E001512E23D90084274FFF0A374A2F0A374D6
:10697E00A3F0900647E025E0FF900646E033FE7454
:10698E00842FF58274013EF583E0FFA3E090084565
:10699E00CFF0A3EFF07B017A0779E512A77F900184
:1069AE00F2E024FE7003026A88147003026B4C241A
:1069BE00026003026C0F90084274FFF0A374A2F001
:1069CE00A374B8F0900646E0FEA3E07802C333CE7F
:1069DE0033CED8F92493F58274033EF583E0FCA3FD
:1069EE00E0FDA3E0FEA3E0FFC004C005C006C007A3
:1069FE00900037E0FEA3E0FFEE3395E0FDFCF8F9E2
:106A0E00AA06AB07D007D006D005D004127CAE90F4
:106A1E000845127D9B900646E0FEA3E07802C33344
:106A2E00CE33CED8F92493F58274033EF583E0FC81
:106A3E00A3E0FDA3E0FEA3E0FFC004C005C006C0B6
:106A4E0007900037E0FEA3E0FFEE3395E0FDFCF883
:106A5E00F9AA06AB07D007D006D005D004127CAE3B
:106A6E00AC00AD01AE02AF03900849127D9B7B01D5
:106A7E007A0779FB12A77F026C5090084274FFF0E0
:106A8E00A374A2F0A374D0F0900646E0FEA3E078C3
:106A9E0002C333CE33CED8F92493F58274033EF578
:106AAE0083E0FCA3E0FDA3E0FEA3E0FFC004C0056D
:106ABE00C006C007900037E0FEA3E0FFEE3395E07E
:106ACE00FDFCF8F9AA06AB07D007D006D005D00416
:106ADE00127CAE900845127D9B900646E0FEA3E028
:106AEE007802C333CE33CED8F92493F58274033EA5
:106AFE00F583E0FCA3E0FDA3E0FEA3E0FFC004C02D
:106B0E0005C006C007900037E0FEA3E0FFEE339508
:106B1E00E0FDFCF8F9AA06AB07D007D006D005D0E9
:106B2E0004127CAEAC00AD01AE02AF039008491268
:106B3E007D9B7B017A0779FB12A77F026C50900830
:106B4E004274FFF0A374A2F0A374E8F0900646E03E
:106B5E00FEA3E07802C333CE33CED8F92493F58268
:106B6E0074033EF583E0FCA3E0FDA3E0FEA3E0FF8B
:106B7E00C004C005C006C007900037E0FEA3E0FFCA
:106B8E00EE3395E0FDFCF8F9AA06AB07D007D00668
:106B9E00D005D004127CAE900845127D9B9006461F
:106BAE00E0FEA3E07802C333CE33CED8F92493F5BA
:106BBE008274033EF583E0FCA3E0FDA3E0FEA3E0B8
:106BCE00FFC004C005C006C007900037E0FEA3E07A
:106BDE00FFEE3395E0FDFCF8F9AA06AB07D007D01F
:106BEE0006D005D004127CAEAC00AD01AE02AF03F0
:106BFE00900849127D9B7B017A0779FB12A77F8053
:106C0E004190084274FFF0A374A3F0A37400F090B7
:106C1E000646E0FEA3E07802C333CE33CED8F92485
:106C2E0093F58274033EF583E0FCA3E0FDA3E0FE42
:106C3E00A3E0FF900845127D9B7B017A0779FB123A
:106C4E00A77F7B017A0779E57D1512E23D7B017AFC
:106C5E000779FB7D1512E23D12E6C512E6C512E676
:106C6E00C5026F2C7BFF7AA279157D1512E23D903D
:106C7E0001F2E024FE7003026D59147003026E1DC2
:106C8E0024026003026EE090084274FFF0A374A326
:106C9E00F0A37412F0900646E0FEA3E07802C33330
:106CAE00CE33CED8F92493F58274033EF583E0FCFF
:106CBE00A3E0FDA3E0FEA3E0FFC004C005C006C034
:106CCE0007900037E0FEA3E0FFEE3395E0FDFCF801
:106CDE00F9AA06AB07D007D006D005D004127CAEB9
:106CEE00900845127D9B900646E0FEA3E07802C315
:106CFE0033CE33CED8F92493F58274033EF583E078
:106D0E00FCA3E0FDA3E0FEA3E0FFC004C005C006A7
:106D1E00C007900037E0FEA3E0FFEE3395E0FDFCE8
:106D2E00F8F9AA06AB07D007D006D005D004127C1E
:106D3E00AEAC00AD01AE02AF03900849127D9B7B55
:106D4E00017A0779FB12A77F026F2190084274FF28
:106D5E00F0A374A3F0A3742AF0900646E0FEA3E01D
:106D6E007802C333CE33CED8F92493F58274033E22
:106D7E00F583E0FCA3E0FDA3E0FEA3E0FFC004C0AA
:106D8E0005C006C007900037E0FEA3E0FFEE339586
:106D9E00E0FDFCF8F9AA06AB07D007D006D005D067
:106DAE0004127CAE900845127D9B900646E0FEA331
:106DBE00E07802C333CE33CED8F92493F582740330
:106DCE003EF583E0FCA3E0FDA3E0FEA3E0FFC004DC
:106DDE00C005C006C007900037E0FEA3E0FFEE330B
:106DEE0095E0FDFCF8F9AA06AB07D007D006D00552
:106DFE00D004127CAEAC00AD01AE02AF03900849D8
:106E0E00127D9B7B017A0779FB12A77F026F21907F
:106E1E00084274FFF0A374A3F0A37442F0900646E8
:106E2E00E0FEA3E07802C333CE33CED8F92493F537
:106E3E008274033EF583E0FCA3E0FDA3E0FEA3E035
:106E4E00FFC004C005C006C007900037E0FEA3E0F7
:106E5E00FFEE3395E0FDFCF8F9AA06AB07D007D09C
:106E6E0006D005D004127CAE900845127D9B90068C
:106E7E0046E0FEA3E07802C333CE33CED8F9249396
:106E8E00F58274033EF583E0FCA3E0FDA3E0FEA3D0
:106E9E00E0FFC004C005C006C007900037E0FEA3A7
:106EAE00E0FFEE3395E0FDFCF8F9AA06AB07D0073C
:106EBE00D006D005D004127CAEAC00AD01AE02AF50
:106ECE0003900849127D9B7B017A0779FB12A77FFD
:106EDE00804190084274FFF0A374A3F0A3745AF09B
:106EEE00900646E0FEA3E07802C333CE33CED8F947
:106EFE002493F58274033EF583E0FCA3E0FDA3E04A
:106F0E00FEA3E0FF900845127D9B7B017A0779FB7B
:106F1E0012A77F7B017A0779FB7D1512E23DE49083
:106F2E000811F090064DE0FF900811E0C39F500B42
:106F3E0012E6C5900811E004F080E8900646E0FAEB
:106F4E00A3E0FBAE027802C333CE33CED8F924933E
:106F5E00F58274033EF583127DA700000000EB2539
:106F6E00E0FFEA33FE74842FF58274013EF583E46C
:106F7E00F0A3F0229001F7E070030274A290038454
:106F8E00E06406700302727412E6C57BFF7AA27982
:106F9E00157D1512E23D7BFF7AA3796C7D1512E209
:106FAE003D7BFF7AA279157D1512E23D900019E026
:106FBE00FFC3945A503990084274FFF0A374A2F0A4
:106FCE00A37441F0A3E4F0A3EFF0900005E0FF906E
:106FDE000847E4F0A3EFF0900028E0FF900849E4A2
:106FEE00F0A3EFF07B017A0779E512A77F803E9040
:106FFE00084274FFF0A374A2F0A3745BF090001922
:10700E00E0FF900845E4F0A3EFF0900005E0FF905C
:10701E000847E4F0A3EFF0900028E0FF900849E461
:10702E00F0A3EFF07B017A0779E512A77F90084273
:10703E0074FFF0A374A2F0A37475F0900029E0FF22
:10704E00900845E4F0A3EFF0900579E0FF90084733
:10705E00E4F0A3EFF07B017A0779FB12A77F7B01A7
:10706E007A0779E57D1512E23D7B017A0779FB7D82
:10707E001512E23D90084274FFF0A374A2F0A374BF
:10708E00A3F0900039E0FFA3E0900845CFF0A3EF06
:10709E00F07B017A0779E512A77F9001F2E024FEDA
:1070AE0070030271381470030271B024026003027F
:1070BE00722790084274FFF0A374A2F0A374B8F084
:1070CE00900037E0FEA3E0FFEE3395E0FDFCF8F90B
:1070DE00AA06AB079002D9E0FCA3E0FDA3E0FEA355
:1070EE00E0FF127CAE900845127D9B900037E0FECB
:1070FE00A3E0FFEE3395E0FDFCF8F9AA06AB07908E
:10710E0002D9E0FCA3E0FDA3E0FEA3E0FF127CAEFB
:10711E00AC00AD01AE02AF03900849127D9B7B011E
:10712E007A0779FB12A77F02725290084274FFF021
:10713E00A374A2F0A374D0F0900037E0FEA3E0FF9A
:10714E00EE3395E0FDFCF8F9AA06AB079002D9E004
:10715E00FCA3E0FDA3E0FEA3E0FF127CAE90084589
:10716E00127D9B900037E0FEA3E0FFEE3395E0FD2D
:10717E00FCF8F9AA06AB079002D9E0FCA3E0FDA348
:10718E00E0FEA3E0FF127CAEAC00AD01AE02AF0399
:10719E00900849127D9B7B017A0779FB12A77F022B
:1071AE00725290084274FFF0A374A2F0A374E8F038
:1071BE00900037E0FEA3E0FFEE3395E0FDFCF8F91A
:1071CE00AA06AB079002D9E0FCA3E0FDA3E0FEA364
:1071DE00E0FF127CAE900845127D9B900037E0FEDA
:1071EE00A3E0FFEE3395E0FDFCF8F9AA06AB07909D
:1071FE0002D9E0FCA3E0FDA3E0FEA3E0FF127CAE0B
:10720E00AC00AD01AE02AF03900849127D9B7B012D
:10721E007A0779FB12A77F802B90084274FFF0A3A8
:10722E0074A3F0A37400F09002D9E0FCA3E0FDA3D8
:10723E00E0FEA3E0FF900845127D9B7B017A077963
:10724E00FB12A77F7B017A0779E57D1512E23D7B64
:10725E00017A0779FB7D1512E23D12E6C512E6C5ED
:10726E0012E6C50274347BFF7AA279157D1512E2FF
:10727E003D9001F2E024FE700302730F14700302BE
:10728E007387240260030273FE90084274FFF0A31A
:10729E0074A2F0A374B8F0900037E0FEA3E0FFEE06
:1072AE003395E0FDFCF8F9AA06AB079002D9E0FC95
:1072BE00A3E0FDA3E0FEA3E0FF127CAE9008451212
:1072CE007D9B900037E0FEA3E0FFEE3395E0FDFCE2
:1072DE00F8F9AA06AB079002D9E0FCA3E0FDA3E003
:1072EE00FEA3E0FF127CAEAC00AD01AE02AF039088
:1072FE000849127D9B7B017A0779FB12A77F0274E6
:10730E002990084274FFF0A374A2F0A374D0F090F9
:10731E000037E0FEA3E0FFEE3395E0FDFCF8F9AA9E
:10732E0006AB079002D9E0FCA3E0FDA3E0FEA3E0CC
:10733E00FF127CAE900845127D9B900037E0FEA3B5
:10734E00E0FFEE3395E0FDFCF8F9AA06AB079002DC
:10735E00D9E0FCA3E0FDA3E0FEA3E0FF127CAEACFF
:10736E0000AD01AE02AF03900849127D9B7B017AFE
:10737E000779FB12A77F02742990084274FFF0A3CD
:10738E0074A2F0A374E8F0900037E0FEA3E0FFEEE5
:10739E003395E0FDFCF8F9AA06AB079002D9E0FCA4
:1073AE00A3E0FDA3E0FEA3E0FF127CAE9008451221
:1073BE007D9B900037E0FEA3E0FFEE3395E0FDFCF1
:1073CE00F8F9AA06AB079002D9E0FCA3E0FDA3E012
:1073DE00FEA3E0FF127CAEAC00AD01AE02AF039097
:1073EE000849127D9B7B017A0779FB12A77F802BC0
:1073FE0090084274FFF0A374A3F0A37400F09002FF
:10740E00D9E0FCA3E0FDA3E0FEA3E0FF9008451247
:10741E007D9B7B017A0779FB12A77F7B017A077927
:10742E00FB7D1512E23DE4900811F090064DE0FF51
:10743E00900811E0C39F500B12E6C5900811E004AE
:10744E00F080E89002D9127DA700000000E49000C1
:10745E0039F0A3F0900015F0A304F0E4900811F0B9
:10746E00900811E0FB25E025E02493F582E4340337
:10747E00F583127DA700000000EB25E02484F58241
:10748E00E43401F583E4F0A3F0900811E004F0E099
:07749E00B433CD2212375573
:0174A50022C4
:10375500300A03024B909001EEE0700B12E7267FD2
:10376500B87E0B12E52F2212E139900015E07004A6
:10377500A3E0640170749001EEE0B405197F1C129A
:10378500E2B07F2612E2B07F1C12E2B07F7412E233
:10379500B07F0112E2B0900531E06420703B9008E3
:1037A50012F0900812E0FFC39448502D74312FF5A4
:1037B50082E43405F583E0B4FF0512E6C5801A906E
:1037C5000812E02431F582E43405F583E0FF12E2C6
:1037D500B0900812E004F080C99001EEE0B4050A4B
:1037E5007F1C12E2B07F2E12E2B0900019E0FFC3F9
:1037F500945A505390084274FFF0A374A3F0A37435
:1038050082F0A3E4F0A3EFF0900005E0FF900847F5
:10381500E4F0A3EFF0900028E0FF900849E4F0A35E
:10382500EFF0900029E0FF90084BE4F0A3EFF09053
:103835000579E0FF90084DE4F0A3EFF07B017A08ED
:10384500792912A77F805890084274FFF0A374A3CA
:10385500F0A3749FF0900019E0FF900845E4F0A3F1
:10386500EFF0900005E0FF900847E4F0A3EFF0903B
:103875000028E0FF900849E4F0A3EFF0900029E06C
:10388500FF90084BE4F0A3EFF0900579E0FF900876
:103895004DE4F0A3EFF07B017A08792912A77F9018
:1038A5000384E0B407004003024A449038B7F8287F
:1038B50028730238CC023B13023D1E02424E0244DD
:1038C5008502469002488F900015E07004A3E064DD
:1038D50001700B7B017A0879297D1512E23D900173
:1038E500F2E024FE7003023991147003023A272492
:1038F500026003023ABC90084274FFF0A374A3F07F
:10390500A374BCF0900015E0FFA3E0900845CFF04C
:10391500A3EFF0900646E0FFA3E0900847CFF0A3A1
:10392500EFF0900037E0FEA3E0FFEE3395E0FDFCFD
:10393500F8F9AA06AB079001F3E0FCA3E0FDA3E0CC
:10394500FEA3E0FF12E4A9900849127D9B90003781
:10395500E0FEA3E0FFEE3395E0FDFCF8F9AA06AB27
:10396500079001F3E0FCA3E0FDA3E0FEA3E0FF1256
:10397500E4A9AC00AD01AE02AF0390084D127D9BEA
:103985007B017A08791312A77F023B0590084274E0
:10399500FFF0A374A3F0A374D8F0900015E0FFA383
:1039A500E0900845CFF0A3EFF0900646E0FFA3E0D6
:1039B500900847CFF0A3EFF0900037E0FEA3E0FFBB
:1039C500EE3395E0FDFCF8F9AA06AB079001F3E0AC
:1039D500FCA3E0FDA3E0FEA3E0FF12E4A9900849E3
:1039E500127D9B900037E0FEA3E0FFEE3395E0FDEE
:1039F500FCF8F9AA06AB079001F3E0FCA3E0FDA3F0
:103A0500E0FEA3E0FF12E4A9AC00AD01AE02AF03F6
:103A150090084D127D9B7B017A08791312A77F02CE
:103A25003B0590084274FFF0A374A3F0A374F4F06F
:103A3500900015E0FFA3E0900845CFF0A3EFF090CC
:103A45000646E0FFA3E0900847CFF0A3EFF0900013
:103A550037E0FEA3E0FFEE3395E0FDFCF8F9AA069A
:103A6500AB079001F3E0FCA3E0FDA3E0FEA3E0FFBC
:103A750012E4A9900849127D9B900037E0FEA3E06F
:103A8500FFEE3395E0FDFCF8F9AA06AB079001F3CC
:103A9500E0FCA3E0FDA3E0FEA3E0FF12E4A9AC0077
:103AA500AD01AE02AF0390084D127D9B7B017A08F4
:103AB500791312A77F804990084274FFF0A374A47C
:103AC500F0A37410F0900015E0FFA3E0900845CF37
:103AD500F0A3EFF0900646E0FFA3E0900847CFF093
:103AE500A3EFF09001F3E0FCA3E0FDA3E0FEA3E06B
:103AF500FF900849127D9B7B017A08791312A77FF5
:103B05007B017A0879137D1512E23D024A44900043
:103B150015E07004A3E06401700B7B017A08792934
:103B25007D1512E23D9001F2E024FE7003023BC9CF
:103B3500147003023C5024026003023CD6900842F4
:103B450074FFF0A374A4F0A37426F0900464E0FF5E
:103B5500A3E0900845CFF0A3EFF0900037E0FEA377
:103B6500E0FFEE3395E0FDFCF8F9AA06AB079001FE
:103B7500F3E0FCA3E0FDA3E0FEA3E0FF12E4A990BF
:103B85000847127D9B900037E0FEA3E0FFEE3395DA
:103B9500E0FDFCF8F9AA06AB079001F3E0FCA3E011
:103BA500FDA3E0FEA3E0FF12E4A9AC00AD01AE0267
:103BB500AF0390084B127D9B7B017A08791312A7FE
:103BC5007F023D1090084274FFF0A374A4F0A37423
:103BD5003FF0900464E0FFA3E0900845CFF0A3EF29
:103BE500F0900037E0FEA3E0FFEE3395E0FDFCF832
:103BF500F9AA06AB079001F3E0FCA3E0FDA3E0FE04
:103C0500A3E0FF12E4A9900847127D9B900037E0DE
:103C1500FEA3E0FFEE3395E0FDFCF8F9AA06AB073D
:103C25009001F3E0FCA3E0FDA3E0FEA3E0FF12E4B6
:103C3500A9AC00AD01AE02AF0390084B127D9B7B92
:103C4500017A08791312A77F023D1090084274FF8C
:103C5500F0A374A4F0A37458F0900464E0FFA3E00B
:103C6500900845CFF0A3EFF0900037E0FEA3E0FF0A
:103C7500EE3395E0FDFCF8F9AA06AB079001F3E0F9
:103C8500FCA3E0FDA3E0FEA3E0FF12E4A990084732
:103C9500127D9B900037E0FEA3E0FFEE3395E0FD3B
:103CA500FCF8F9AA06AB079001F3E0FCA3E0FDA33D
:103CB500E0FEA3E0FF12E4A9AC00AD01AE02AF0344
:103CC50090084B127D9B7B017A08791312A77F80A0
:103CD5003A90084274FFF0A374A4F0A37471F090B5
:103CE5000464E0FFA3E0900845CFF0A3EFF0900156
:103CF500F3E0FCA3E0FDA3E0FEA3E0FF900847127C
:103D05007D9B7B017A08791312A77F7B017A08795D
:103D1500137D1512E23D024A447B017A0879297D1B
:103D25001512E23D9001F2E024FE7003023DB91444
:103D35007003023E3124026003023EA890084274DB
:103D4500FFF0A374A4F0A37484F0900037E0FEA301
:103D5500E0FFEE3395E0FDFCF8F9AA06AB0790030A
:103D650089E0FCA3E0FDA3E0FEA3E0FF12E4A99037
:103D75000845127D9B900037E0FEA3E0FFEE3395EA
:103D8500E0FDFCF8F9AA06AB07900389E0FCA3E087
:103D9500FDA3E0FEA3E0FF12E4A9AC00AD01AE0275
:103DA500AF03900849127D9B7B017A08791312A70E
:103DB5007F023ED390084274FFF0A374A4F0A3746D
:103DC5009CF0900037E0FEA3E0FFEE3395E0FDFCAC
:103DD500F8F9AA06AB07900389E0FCA3E0FDA3E090
:103DE500FEA3E0FF12E4A9900845127D9B900037E1
:103DF500E0FEA3E0FFEE3395E0FDFCF8F9AA06AB83
:103E050007900389E0FCA3E0FDA3E0FEA3E0FF1219
:103E1500E4A9AC00AD01AE02AF03900849127D9B49
:103E25007B017A08791312A77F023ED3900842746A
:103E3500FFF0A374A4F0A374B4F0900037E0FEA3E0
:103E4500E0FFEE3395E0FDFCF8F9AA06AB07900319
:103E550089E0FCA3E0FDA3E0FEA3E0FF12E4A99046
:103E65000845127D9B900037E0FEA3E0FFEE3395F9
:103E7500E0FDFCF8F9AA06AB07900389E0FCA3E096
:103E8500FDA3E0FEA3E0FF12E4A9AC00AD01AE0284
:103E9500AF03900849127D9B7B017A08791312A71D
:103EA5007F802B90084274FFF0A374A4F0A374CC18
:103EB500F0900389E0FCA3E0FDA3E0FEA3E0FF9002
:103EC5000845127D9B7B017A08791312A77F7B0138
:103ED5007A0879137D1512E23D9001F2E024FE7017
:103EE50003023F6E147003023FE6240260030240A2
:103EF5005D90084274FFF0A374A4F0A374DEF09003
:103F05000037E0FEA3E0FFEE3395E0FDFCF8F9AAEB
:103F150006AB07900010E0FCA3E0FDA3E0FEA3E0E4
:103F2500FF12E4A9900845127D9B900037E0FEA39F
:103F3500E0FFEE3395E0FDFCF8F9AA06AB0790002B
:103F450010E0FCA3E0FDA3E0FEA3E0FF12E4A9ACB2
:103F550000AD01AE02AF03900849127D9B7B017A4B
:103F650008791312A77F02408890084274FFF0A3D6
:103F750074A4F0A374F6F0900037E0FEA3E0FFEE22
:103F85003395E0FDFCF8F9AA06AB07900010E0FCBC
:103F9500A3E0FDA3E0FEA3E0FF12E4A9900845120B
:103FA5007D9B900037E0FEA3E0FFEE3395E0FDFC3E
:103FB500F8F9AA06AB07900010E0FCA3E0FDA3E02A
:103FC500FEA3E0FF12E4A9AC00AD01AE02AF039081
:103FD5000849127D9B7B017A08791312A77F02405D
:103FE5008890084274FFF0A374A5F0A3740EF090B6
:103FF5000037E0FEA3E0FFEE3395E0FDFCF8F9AAFB
:1040050006AB07900010E0FCA3E0FDA3E0FEA3E0F3
:10401500FF12E4A9900845127D9B900037E0FEA3AE
:10402500E0FFEE3395E0FDFCF8F9AA06AB0790003A
:1040350010E0FCA3E0FDA3E0FEA3E0FF12E4A9ACC1
:1040450000AD01AE02AF03900849127D9B7B017A5A
:1040550008791312A77F802B90084274FFF0A37490
:10406500A5F0A37426F0900010E0FCA3E0FDA3E00A
:10407500FEA3E0FF900845127D9B7B017A0879132A
:1040850012A77F7B017A0879137D1512E23D900115
:10409500F2E024FE700302412314700302419B24C5
:1040A50002600302421290084274FFF0A374A5F067
:1040B500A37438F0900037E0FEA3E0FFEE3395E0FF
:1040C500FDFCF8F9AA06AB079001F3E0FCA3E0FDBF
:1040D500A3E0FEA3E0FF12E4A9900845127D9B90A2
:1040E5000037E0FEA3E0FFEE3395E0FDFCF8F9AA0A
:1040F50006AB079001F3E0FCA3E0FDA3E0FEA3E01F
:10410500FF12E4A9AC00AD01AE02AF03900849125D
:104115007D9B7B017A08791312A77F02423D9008A7
:104125004274FFF0A374A5F0A37450F0900037E03B
:10413500FEA3E0FFEE3395E0FDFCF8F9AA06AB0718
:104145009001F3E0FCA3E0FDA3E0FEA3E0FF12E491
:10415500A9900845127D9B900037E0FEA3E0FFEE95
:104165003395E0FDFCF8F9AA06AB079001F3E0FCF6
:10417500A3E0FDA3E0FEA3E0FF12E4A9AC00AD01BE
:10418500AE02AF03900849127D9B7B017A08791333
:1041950012A77F02423D90084274FFF0A374A5F078
:1041A500A37468F0900037E0FEA3E0FFEE3395E0DE
:1041B500FDFCF8F9AA06AB079001F3E0FCA3E0FDCE
:1041C500A3E0FEA3E0FF12E4A9900845127D9B90B1
:1041D5000037E0FEA3E0FFEE3395E0FDFCF8F9AA19
:1041E50006AB079001F3E0FCA3E0FDA3E0FEA3E02E
:1041F500FF12E4A9AC00AD01AE02AF03900849126D
:104205007D9B7B017A08791312A77F802B9008424A
:1042150074FFF0A374A5F0A37480F09001F3E0FCA3
:10422500A3E0FDA3E0FEA3E0FF900845127D9B7B84
:10423500017A08791312A77F7B017A0879137D1516
:1042450012E23D12E6C5024A44900015E07004A34F
:10425500E06401700B7B017A0879297D1512E23D36
:104265009001F2E024FE700302430F147003024331
:10427500A12402600302443290084274FFF0A37443
:10428500A5F0A37492F0900029E0FF900845E4F0B2
:10429500A3EFF0900579E0FF900847E4F0A3EFF075
:1042A500900037E0FEA3E0FFEE3395E0FDFCF8F962
:1042B500AA06AB079001F3E0FCA3E0FDA3E0FEA393
:1042C500E0FF12E4A9900849127D9B900037E0FEBB
:1042D500A3E0FFEE3395E0FDFCF8F9AA06AB0790E5
:1042E50001F3E0FCA3E0FDA3E0FEA3E0FF12E4A9D7
:1042F500AC00AD01AE02AF0390084D127D9B7B0172
:104305007A08791312A77F02447790084274FFF068
:10431500A374A5F0A374AFF0900029E0FF900845C1
:10432500E4F0A3EFF0900579E0FF900847E4F0A3EF
:10433500EFF0900037E0FEA3E0FFEE3395E0FDFCE3
:10434500F8F9AA06AB079001F3E0FCA3E0FDA3E0B2
:10435500FEA3E0FF12E4A9900849127D9B90003767
:10436500E0FEA3E0FFEE3395E0FDFCF8F9AA06AB0D
:10437500079001F3E0FCA3E0FDA3E0FEA3E0FF123C
:10438500E4A9AC00AD01AE02AF0390084D127D9BD0
:104395007B017A08791312A77F024477900842744B
:1043A500FFF0A374A5F0A374CCF0900029E0FF9072
:1043B5000845E4F0A3EFF0900579E0FF900847E4A5
:1043C500F0A3EFF0900037E0FEA3E0FFEE3395E0B9
:1043D500FDFCF8F9AA06AB079001F3E0FCA3E0FDAC
:1043E500A3E0FEA3E0FF12E4A9900849127D9B908B
:1043F5000037E0FEA3E0FFEE3395E0FDFCF8F9AAF7
:0644050006AB079001F375
:10440B00E0FCA3E0FDA3E0FEA3E0FF12E4A9AC00F7
:10441B00AD01AE02AF0390084D127D9B7B017A0874
:10442B00791312A77F804590084274FFF0A374A5FF
:10443B00F0A374E9F0900029E0FF900845E4F0A3A5
:10444B00EFF0900579E0FF900847E4F0A3EFF090D0
:10445B0001F3E0FCA3E0FDA3E0FEA3E0FF9008491D
:10446B00127D9B7B017A08791312A77F7B017A0857
:10447B0079137D1512E23D024A44900015E0700459
:10448B00A3E06401700B7B017A0879297D1512E298
:10449B003D9001F2E024FE700302453B14700302D1
:1044AB0045C22402600302464890084274FFF0A301
:1044BB0074A6F0A37400F0900646E0FFA3E090080A
:1044CB0045CFF0A3EFF0900037E0FEA3E0FFEE3313
:1044DB0095E0FDFCF8F9AA06AB079001F3E0FCA30D
:1044EB00E0FDA3E0FEA3E0FF12E4A9900847127DD4
:1044FB009B900037E0FEA3E0FFEE3395E0FDFCF868
:10450B00F9AA06AB079001F3E0FCA3E0FDA3E0FEE4
:10451B00A3E0FF12E4A9AC00AD01AE02AF0390081B
:10452B004B127D9B7B017A08791312A77F0246827F
:10453B0090084274FFF0A374A6F0A3741AF09006CF
:10454B0046E0FFA3E0900845CFF0A3EFF0900037D3
:10455B00E0FEA3E0FFEE3395E0FDFCF8F9AA06AB15
:10456B00079001F3E0FCA3E0FDA3E0FEA3E0FF1244
:10457B00E4A9900847127D9B900037E0FEA3E0FF73
:10458B00EE3395E0FDFCF8F9AA06AB079001F3E0DA
:10459B00FCA3E0FDA3E0FEA3E0FF12E4A9AC00AD99
:1045AB0001AE02AF0390084B127D9B7B017A087919
:1045BB001312A77F02468290084274FFF0A374A6E1
:1045CB00F0A37434F0900646E0FFA3E0900845CFCB
:1045DB00F0A3EFF0900037E0FEA3E0FFEE3395E0A1
:1045EB00FDFCF8F9AA06AB079001F3E0FCA3E0FD94
:1045FB00A3E0FEA3E0FF12E4A9900847127D9B9075
:10460B000037E0FEA3E0FFEE3395E0FDFCF8F9AADE
:10461B0006AB079001F3E0FCA3E0FDA3E0FEA3E0F3
:10462B00FF12E4A9AC00AD01AE02AF0390084B1230
:10463B007D9B7B017A08791312A77F803A90084201
:10464B0074FFF0A374A6F0A3744EF0900646E0FF3F
:10465B00A3E0900845CFF0A3EFF09001F3E0FCA3AB
:10466B00E0FDA3E0FEA3E0FF900847127D9B7B01DA
:10467B007A08791312A77F7B017A0879137D1512BB
:10468B00E23D024A447B017A0879297D1512E23D0D
:10469B009001F2E024FE700302473A1470030247C4
:1046AB00C12402600302484790084274FFF0A374D0
:1046BB00A6F0A37462F0900015E0FFA3E09008450C
:1046CB00CFF0A3EFF0900037E0FEA3E0FFEE3395C1
:1046DB00E0FDFCF8F9AA06AB079001F3E0FCA3E0C0
:1046EB00FDA3E0FEA3E0FF12E4A9900847127D9B17
:1046FB00900037E0FEA3E0FFEE3395E0FDFCF8F908
:10470B00AA06AB079001F3E0FCA3E0FDA3E0FEA338
:10471B00E0FF12E4A9AC00AD01AE02AF0390084B71
:10472B00127D9B7B017A08791312A77F0248819037
:10473B00084274FFF0A374A6F0A3747BF0900015ED
:10474B00E0FFA3E0900845CFF0A3EFF0900037E037
:10475B00FEA3E0FFEE3395E0FDFCF8F9AA06AB07EC
:10476B009001F3E0FCA3E0FDA3E0FEA3E0FF12E465
:10477B00A9900847127D9B900037E0FEA3E0FFEE67
:10478B003395E0FDFCF8F9AA06AB079001F3E0FCCA
:10479B00A3E0FDA3E0FEA3E0FF12E4A9AC00AD0192
:1047AB00AE02AF0390084B127D9B7B017A08791305
:1047BB0012A77F02488190084274FFF0A374A6F001
:1047CB00A37494F0900015E0FFA3E0900845CFF0A0
:1047DB00A3EFF0900037E0FEA3E0FFEE3395E0FD92
:1047EB00FCF8F9AA06AB079001F3E0FCA3E0FDA3EC
:1047FB00E0FEA3E0FF12E4A9900847127D9B900016
:10480B0037E0FEA3E0FFEE3395E0FDFCF8F9AA06D6
:10481B00AB079001F3E0FCA3E0FDA3E0FEA3E0FFF8
:10482B0012E4A9AC00AD01AE02AF0390084B127DB0
:10483B009B7B017A08791312A77F803A9008427408
:10484B00FFF0A374A6F0A374ADF0900015E0FFA3E6
:10485B00E0900845CFF0A3EFF09001F3E0FCA3E06C
:10486B00FDA3E0FEA3E0FF900847127D9B7B017A3E
:10487B0008791312A77F7B017A0879137D1512E251
:10488B003D024A449001F2E024FE700302491F14DA
:10489B00700302499724026003024A0E9008427487
:1048AB00FFF0A374A6F0A374C0F0900037E0FEA352
:1048BB00E0FFEE3395E0FDFCF8F9AA06AB0790019B
:1048CB00F3E0FCA3E0FDA3E0FEA3E0FF12E4A9905C
:1048DB000845127D9B900037E0FEA3E0FFEE339579
:1048EB00E0FDFCF8F9AA06AB079001F3E0FCA3E0AE
:1048FB00FDA3E0FEA3E0FF12E4A9AC00AD01AE0204
:10490B00AF03900849127D9B7B017A08791312A79C
:10491B007F024A3990084274FFF0A374A6F0A37487
:10492B00D8F0900037E0FEA3E0FFEE3395E0FDFCFE
:10493B00F8F9AA06AB079001F3E0FCA3E0FDA3E0B6
:10494B00FEA3E0FF12E4A9900845127D9B9000376F
:10495B00E0FEA3E0FFEE3395E0FDFCF8F9AA06AB11
:10496B00079001F3E0FCA3E0FDA3E0FEA3E0FF1240
:10497B00E4A9AC00AD01AE02AF03900849127D9BD8
:10498B007B017A08791312A77F024A399008427487
:10499B00FFF0A374A6F0A374F0F0900037E0FEA331
:1049AB00E0FFEE3395E0FDFCF8F9AA06AB079001AA
:1049BB00F3E0FCA3E0FDA3E0FEA3E0FF12E4A9906B
:1049CB000845127D9B900037E0FEA3E0FFEE339588
:1049DB00E0FDFCF8F9AA06AB079001F3E0FCA3E0BD
:1049EB00FDA3E0FEA3E0FF12E4A9AC00AD01AE0213
:1049FB00AF03900849127D9B7B017A08791312A7AC
:104A0B007F802B90084274FFF0A374A7F0A3740867
:104A1B00F09001F3E0FCA3E0FDA3E0FEA3E0FF9028
:104A2B000845127D9B7B017A08791312A77F7B01C6
:104A3B007A0879137D1512E23DE4900812F0900686
:104A4B004DE0FF900812E0C39F500B12E6C5900893
:104A5B0012E004F080E8900006E0FCA3E0FDA3E088
:104A6B00FEA3E0FF9001F3E0F8A3E0F9A3E0FAA3C3
:104A7B00E0FBEF2BFFEE3AFEED39FDEC38FC90003E
:104A8B0006127D9B900646E0FEA3E07802C333CE70
:104A9B0033CED8F92493F58274033EF583C083C0DB
:104AAB0082E0FCA3E0FDA3E0FEA3E0FF9001F3E0B6
:104ABB00F8A3E0F9A3E0FAA3E0FBEF2BFFEE3AFE3D
:104ACB00ED39FDEC38FCD082D083127D9B9002D95E
:104ADB00E0FCA3E0FDA3E0FEA3E0FF9001F3E0F810
:104AEB00A3E0F9A3E0FAA3E0FBEF2BFFEE3AFEED18
:104AFB0039FDEC38FC9002D9127D9B900647E025DE
:104B0B00E0FF900646E033FE74842FF58274013E7D
:104B1B00F583E475F001127C0D90003AE004F0701F
:104B2B0006900039E004F0900465E004F070069004
:104B3B000464E004F0900016E004F0700690001599
:104B4B00E004F0D3900016E094E7900015E0940396
:104B5B004005E4F0A304F0D3900465E094E79004DF
:104B6B0064E094034005E4F0A304F0900464E0FED9
:104B7B00A3E0FFE4FCFD900842127D9B7D697C0065
:054B8B007F0112B98654
:014B90002202
:1074A60002785BE86480F8E933E83360110460F041
:1074B600ED33EC337009E8FCE9FDEAFEEBFF22044C
:1074C60060DED3EB9FEA9EE99DE8C2E78CF0C2F747
:1074D60095F0400CE8CCF8E9CDF9EACEFAEBCFFB13
:1074E60012782685D0F05804700320D5B3E80470CE
:1074F600075002B2D502786592D5EC0460F7E4CC69
:10750600C0E0C398F8603B94186008400DD0E0FBDB
:1075160002783DE4FBFAC9FC8028E830E406E4C9B9
:10752600FBE4CAFCE830E305E4C9CACBFCE854072F
:107536006010F8C3E913F9EA13FAEB13FBEC13FC3A
:10754600D8F130F52FC3E49CFCEF9BFFEE9AFEEDDD
:1075560099FDD0E0FBEF4E4D4C701222DB03027812
:1075660062EC2CFCEF33FFEE33FEED33FDED30E73E
:10757600EB02783DEF2BFFEE3AFEED39FDD0E0FB56
:1075860050130BBB0003027865ED13FDEE13FEEFFF
:0875960013FFEC13FC02783D29
:10759E00EC4D6011E8497017ED33EC3304600DE4E7
:1075AE00FCFFFEFD22E933E8330470F802785B122B
:1075BE00782658046009E4CC24815006285009022C
:1075CE007865284003027862C0E0EB4A7044B980C7
:1075DE0006D0E0FB027851EF4E701CBD8008EBFF29
:1075EE00EAFEE9FD80EBE98DF0A4FEE5F002768778
:1075FE00E9CDF9EAFEEBFFEF89F0A4FCE5F0CE89C8
:10760E00F0A42EFFE435F0CD89F0A42DFEE435F084
:10761E008067EF4E7005BD80D780C3EF8BF0A4ACB2
:10762E00F0EE8BF0A42CFCE435F0F8EF8AF0A42CED
:10763E00E5F038FCE433CB8DF0A42CFCE5F03BF800
:10764E00EE8AF0A42CFCE5F038F8E433CF89F0A4F0
:10765E002CFCE5F038CF3400CE89F0A42FFFE5F0F6
:10766E003EFEE433C98DF0A42EFEE5F039CD8AF04E
:10767E00A42FFFE5F03EFEE43DFD33D0E0FB5007C6
:10768E000BBB000F027865EC2CFCEF33FFEE33FEE4
:06769E00ED33FD02783D12
:1076A400027865EC5D046005E85904700302785BB8
:1076B400127826580460F6EC4860F2EC7004FDFE83
:1076C400FF22C860DB2481C85009C39860025006B9
:1076D4000278629850CAF582E9294B4A7005AB8258
:1076E40002785175F0007C1A7880C3EF9BEE9AED16
:1076F40099400DC3EF9BFFEE9AFEED99FDE842F031
:10770400DC23ACF0D0E0FFD0E0FED0E0FDAB822083
:10771400E7101BEB60BAEC2CFCEF33FFEE33FEED0D
:1077240033FD02783DE803F830E705C0F075F0005A
:10773400EF2FFFEE33FEED33FD40B830E7C280AAF1
:1077440074F8CC6480CCC86480C8F582046043C3F8
:10775400EB9FF5F0EA9E42F0E99D42F0E89C45F08B
:1077640060305018E5825FFFE582F42B5582FB50B0
:10777400210ABA001D09B90019088016E5825BFBCD
:10778400E582F42F5582FF50090EBE00050DBD00A1
:10779400010CC3EB9FF5F0EA9E42F0E99D42F0E84C
:0D77A4009C45F06007CC4820E701B3EC22C3
:1077B10075F020800E75F010800575F0087D007E53
:1077C100007F003392D530D503127D40EC33401059
:1077D100EF33FFEE33FEED33FDEC33FCD5F0ED225C
:0E77E100E5F0247EA2D513CC92E7CDCEFF2298
:1077EF00EDD2E7CD33EC3392D524814006E4FFFE92
:1077FF00FDFC22FCE4CFCECDCC24E0501174FF80F1
:10780F00EDC3CC13CCCD13CDCE13CECF13CF04708D
:07781F00F030D5DE027D40D0
:10A71A00E5672442F582E43408F583E00567229070
:10A72A00083F300803900842E475F001127DD80210
:10A73A007B182001E97F2ED2018018EF540F249054
:10A74A00D43440D4FF30050BEF24BFB41A005003B1
:10A75A002461FFE56860021568056BE56B70020508
:10A76A006A30080E90083FE475F001127DD8EF02B6
:10A77A007B5E02E69E7403D2088003E4C208F56792
:10A78A0090083F127DEFE4F568F56AF56BE56860BD
:10A79A00077F2012A75D80F57569FFC202C201C258
:10A7AA0003C204C206C207C20912A729FF700D30EC
:10A7BA0008057F0012A76EAF6BAE6A22B4255FC28E
:10A7CA00D5C20512A729FF24D0B40A00501A75F081
:10A7DA000A786830D50508B6FF0106C6A426F62011
:10A7EA00D5047002D20480D924CFB41A00EF5004E1
:10A7FA00C2E5D20502AA6ED20280C6D20180C0D2B8
:10A80A000380BCD2D580BAD20680B47F2012A75D5D
:10A81A002003077401B5680040F112A71AFF12A7B6
:10A82A005D02A797D209D207809512A71AFB12A731
:10A83A001AFA12A71AF94A4B7006796C7AAB7BFF9F
:10A84A0020033BE56860377E00E9C0E02EF9EAC0E4
:10A85A00E03400FA127B18F9D0E0FAD0E0C96006B9
:10A86A000EEE656970E3C2D5EBC0E0EAC0E0E9C06C
:10A87A00E0EE12AACFD0E0F9D0E0FAD0E0FB127BEA
:10A88A0018FF609DEBC0E0EAC0E0E9C0E012A75DF6
:10A89A00D0E02401F9D0E03400FAD0E0FBE5690405
:10A8AA0060DCD569D902A82BD203809412AAB160C0
:10A8BA00F7E569700104127870A969600DE56960AD
:10A8CA000914F56912AB59EF60F3EA30E702F404B0
:10A8DA00C3995079EAF425690430E701E404F5697B
:10A8EA00800D12AAB160C1EA05692569127870EA79
:10A8FA0090086EF030E701E4256904D56904200662
:10A90A00011412AACFE4C0E012AB5990086EE060BD
:10A91A001320E70714F012A745802204F0D0E014B0
:10A92A00C0E07F0012A745E569600712A73C1569D8
:10A93A00800B30060312A73CD0E002A797D0E004B0
:10A94A0080C412AAB1609EE5690412787090086EFC
:06A95A00EAF0E5692006A9
:10A9600002600104240412AACF74FF04C0E012ABF9
:10A970005912A745E569200602600312A73CD0E002
:10A98000B569E87F4512A74F90086EE07F2B30E74E
:10A99000047F2DF404C0E012A75DD0E075F00A84B6
:10A9A000C0F012A746D0E012A74602A79779108000
:10A9B000027908C207C2098008D2D5790A800479D1
:10A9C0000AC2D5E569047002F569E4FAFDFEFF12DA
:10A9D000A71AFC7B0820021312A71AFD7B10300176
:10A9E0000A12A71AFE12A71AFF7B20EC3382D59217
:10A9F000D55013C3E43001069FFFE49EFEE420021D
:10AA0000039DFDE49CFCE4CBF8C202EC700CCFCEBD
:10AA1000CDCCE824F8F870F38017C3EF33FFEE33A2
:10AA2000FEED33FDEC33FCEB33FB994002FB0FD81A
:10AA3000E9EB300205F8D0E0C448B202C0E00AEC0D
:10AA40004D4E4F78207B0070C2EAB5690040BCC013
:10AA5000E012AAD1D0F0D0E0200204C4C0E0C4B219
:10AA600002C0F012A746D0F0D5F0EB02A797127DF6
:10AA7000F8A83453A9AD58A8054CA80142A9B14F74
:10AA8000A9B944A9B949A81A43A9BF55A8EC46A930
:10AA90004C45A8B647AB8C50A8092DA80D2EA83060
:10AAA0002BA81123A82E20AB7A2AA7C9480000A8FA
:10AAB00028E569B4FF0375690612A71AFC12A71AE4
:10AAC000FD12A71AFE12A71AFF9008670278AD7947
:10AAD0000AA2D5200414300609B910020404B908EA
:10AAE0000104A2D52007025001042003689203B597
:10AAF00068005034C0E07F203004197F30A2037218
:10AB0000077206500F12AB28C203C207C206C20961
:10AB10007F30800F300603E9C0E012A75D300603E6
:10AB2000D0E0F9D0E0B568CC3006177F30B9100C12
:10AB300012A75D7F583005077F788003B90803129C
:10AB4000A75D3003057F2D02A75D7F202009F87FD8
:10AB50002B2007F322920380CF7F00B40700500B15
:10AB60002467F582E43408F583E0FF22286E756CD3
:10AB70006C29002D50434958D20212A71A3002F80E
:10AB8000C202786830D50108F602A7C912A71A24B4
:10AB900003B405004001E490AB739312A74E743ADE
:0BABA00012A74ED20475680402A9AD94
:10782600E9D2E7C933E833F892D5EDD2E7CD33ECA8
:0778360033FC5002B2D52221
:10783D00EC30E7100FBF000C0EBE00080DBD0004AC
:10784D000BEB6014A2D5EB13FCED92E7FD2274FF58
:10785D00FCFDFEFF22E480F8A2D574FF13FC7D80B1
:03786D00E480EFC5
:10787000F920E73624F950037907E4F42402FBE504
:1078800082158270021583DBF6E024FB501BE96051
:1078900014E4F0E582158270021583E004F0B40A66
:0D78A00008E4F0D9EE7401F00A22C2D522EE
:1078AD00ED33EC3392D5FA602AB4FF33EDC2E77BAA
:1078BD00FF60067A7879D2E4227A7879DB20D504D4
:1078CD007A7879D6224E614E002B494E46002D49CD
:1078DD004E4600E47A08F0A3DAFC7B00740722C060
:1078ED0083C082ECC0E0EDC0E0EEC0E0EFC0E0EAA6
:1078FD0075F010A4CAABF075F04DA42BFBE435F078
:10790D00FCEA2410FAEB34C5FBEC34D9FCEDC2E7EC
:10791D00FF75F056A4F42411C5F0F434C58FF0A40E
:10792D002AE5F03BE43CF020E7141279E2D0E0FFC9
:10793D00D0E0FED0E0FDD0E0FC1276A78014F40478
:10794D001279E2D0E0FFD0E0FED0E0FDD0E0FC12F5
:10795D00759ED082D083E0FAEDD2E7CD33EC33249F
:10796D0082FBE4C3CF33CFCE33CECD33CD33DBF378
:10797D007B0775F00A846004F0A31B0AE5F0F0A301
:10798D008FF0740AA4FFACF08EF0740AA42CFEAC38
:10799D00F050010C8DF0740AA42CFDE435F0F0A329
:0579AD00DBDE7407227F
:1079B2003F8000004120000042C80000447A0000DD
:1079C200461C400047C35000497424004B1896805F
:1079D2004CBEBC205A0E1BCA6753C21C749DC5AE56
:1079E200FB60065407601C2323127A10EB543860A4
:1079F200091279FC127A0B12759EECF8EDF9EEFA87
:107A0200EFCB22EB127A0B80F1543803241C9079CD
:107A1200B2FE93FC0EEE93FD0EEE930ECE93FF227A
:0300000002DF9D7F
:0CDF9D00787FE4F6D8FD75816D02DFE4AA
:107A2200E709F608DFFA8046E709F208DFFA803E46
:107A320088828C83E709F0A3DFFA8032E309F60833
:107A4200DFFA8078E309F208DFFA807088828C839B
:107A5200E309F0A3DFFA806489828A83E0A3F6084F
:107A6200DFFA805889828A83E0A3F208DFFA804C29
:107A720080D280FA80C680D4806980F28033801000
:107A820080A680EA809A80A880DA80E280CA803369
:107A920089828A83ECFAE493A3C8C582C8CCC583E1
:107AA200CCF0A3C8C582C8CCC583CCDFE9DEE780B1
:107AB2000D89828A83E493A3F608DFF9ECFAA9F030
:107AC200EDFB2289828A83ECFAE0A3C8C582C8CC86
:107AD200C583CCF0A3C8C582C8CCC583CCDFEADE9F
:107AE200E880DB89828A83E493A3F208DFF980CC01
:107AF20088F0EF60010E4E60C388F0ED2402B404FA
:107B02000050B9F582EB2402B4040050AF232345A0
:067B12008223907A7273D9
:107B1800BB010689828A83E0225002E722BBFE026B
:097B2800E32289828A83E493229E
:107B3100BB010CE58229F582E5833AF583E0225009
:107B410006E92582F8E622BBFE06E92582F8E22253
:0D7B5100E58229F582E5833AF583E493226D
:107B5E00BB010689828A83F0225002F722BBFE0106
:027B6E00F32200
:107B7000EF8DF0A4A8F0CF8CF0A428CE8DF0A42E29
:027B8000FE22E3
:107B8200BC000BBE0029EF8DF084FFADF022E4CCE7
:107B9200F875F008EF2FFFEE33FEEC33FCEE9DECB0
:107BA200984005FCEE9DFE0FD5F0E9E4CEFD22EDF6
:107BB200F8F5F0EE8420D21CFEADF075F008EF2F40
:107BC200FFED33FD4007985006D5F0F222C398FD31
:057BD2000FD5F0EA22CE
:107BD700C2D5EC30E709B2D5E4C39DFDE49CFCEEC9
:107BE70030E715B2D5E4C39FFFE49EFE127B82C344
:107BF700E49DFDE49CFC8003127B8230D507C3E43F
:067C07009FFFE49EFE2237
:107C0D00C5F0F8A3E028F0C5F0F8E5821582700202
:067C1D001583E038F0229F
:107C2300E88FF0A4CC8BF0A42CFCE98EF0A42CFC00
:107C33008AF0EDA42CFCEA8EF0A4CDA8F08BF0A47E
:107C43002DCC3825F0FDE98FF0A42CCD35F0FCEBDD
:107C53008EF0A4FEA9F0EB8FF0A4CFC5F02ECD39A2
:0F7C6300FEE43CFCEAA42DCE35F0FDE43CFC220F
:107C720075F008758200EF2FFFEE33FECD33CDCCC9
:107C820033CCC58233C5829BED9AEC99E58298404C
:107C92000CF582EE9BFEED9AFDEC99FC0FD5F0D629
:107CA200E4CEFBE4CDFAE4CCF9A88222B800C1B953
:107CB2000059BA002DEC8BF084CFCECDFCE5F0CB91
:107CC200F97818EF2FFFEE33FEED33FDEC33FCEBCA
:107CD20033FB10D703994004EB99FB0FD8E5E4F985
:107CE200FA227818EF2FFFEE33FEED33FDEC33FC72
:107CF200C933C910D7059BE99A4007EC9BFCE99A66
:107D0200F90FD8E0E4C9FAE4CCFB2275F010EF2FAA
:107D1200FFEE33FEED33FDCC33CCC833C810D707AA
:107D22009BEC9AE899400AED9BFDEC9AFCE899F8E5
:0E7D32000FD5F0DAE4CDFBE4CCFAE4C8F92278
:10E4A900C2D5E830E70FB2D5E4C39BFBE49AFAE49E
:10E4B90099F9E498F8EC30E717B2D512E4DF127C49
:10E4C900AEE4C39BFBE49AFAE499F9E498F8800373
:10E4D900127CAE30D50DE4C39FFFE49EFEE49DFDA2
:04E4E900E49CFC2291
:0E7D4000C3E49FFFE49EFEE49DFDE49CFC2254
:107D4E00EB9FF5F0EA9E42F0E99D42F0EC6480C8AC
:067D5E0064809845F0224C
:107D6400EB9FF5F0EA9E42F0E99D42F0E89C45F075
:017D740022EC
:107D7500E8600FECC313FCED13FDEE13FEEF13FFEC
:037D8500D8F12210
:107D8800E8600FEFC333FFEE33FEED33FDEC33FC59
:037D9800D8F122FD
:0C7D9B00ECF0A3EDF0A3EEF0A3EFF0225B
:107DA700A8828583F0D083D082127DBE127DBE1259
:107DB7007DBE127DBEE473E493A3C583C5F0C5837E
:107DC700C8C582C8F0A3C583C5F0C583C8C582C826
:017DD7002289
:107DD800F8E0FBA3A3E0F925F0F0E5821582700234
:077DE8001583E0FA38F022D8
:097DEF00EBF0A3EAF0A3E9F02295
:107DF800D083D082F8E4937012740193700DA3A31A
:107E080093F8740193F5828883E47374029368602D
:067E1800EFA3A3A380DF2D
:10E69E00EFB40A07740D12E6A9740A309811A899FE
:10E6AE00B8130CC2983098FDA899C298B811F630DC
:07E6BE0099FDC299F59922B4
:10E75200E4FFFE127B18600C0FEF70010E09E970E6
:05E76200F20A80EF2225
:10DFA900028EC9E493A3F8E493A34003F68001F237
:10DFB90008DFF48029E493A3F85407240CC8C33379
:10DFC900C4540F4420C8834004F456800146F6DF48
:10DFD900E4800B010204081020408090E390E47E65
:10DFE900019360BCA3FF543F30E509541FFEE4933D
:10DFF900A360010ECF54C025E060A840B8E493A304
:10E00900FAE493A3F8E493A3C8C582C8CAC583CA2E
:10E01900F0A3C8C582C8CAC583CADFE9DEE780BEE6
:01E3F100002B
:00000001FF
